:100000000C94192B0D94010F0D94D60E0D94AB0E7C
:100010000D94800E0D94550E0D942A0E0D94FF0D27
:100020000C9412CF0C944A2B0C944A2B0C944A2B10
:100030000C944A2B0C9470B50C944A2B0C944A2BBC
:100040000C944A2B0C9495C70C944A2B0C944A2B75
:100050000C944A2B0C944A2B0C94FCC50D942C0F39
:100060000C944A2B0C9458CE0C944A2B0C944A2B8B
:100070000C944A2B0C944A2B0C944A2B0C944A2B2C
:100080000C944A2B0C944A2B0C944A2B0C944A2B1C
:100090000C944A2B0C944A2B0C944A2B0C944A2B0C
:1000A0000C944A2B0C944A2B0C944A2B0C944A2BFC
:1000B0000C944A2B0C944A2B0C944A2B0C944A2BEC
:1000C0000C944A2B0C944A2B0C944A2B0C944A2BDC
:1000D0000C944A2B0C944A2B0C944A2B0C944A2BCC
:1000E0000C944A2BF44FF94FFE4F085012508B508E
:1000F0001C5024502C50365040504A505950635098
:100100008B506D50775081502B782B783278327825
:10011000327839783978397846784078407840783C
:100120008CCE92CEA3CEAECEB6CECBCEBACECBCEEA
:10013000BECEC2CECBCEC8CEF200F0000201D600B9
:100140000A01E2000001FE00F400D4000801D8001A
:10015000FC00EE00E200E400E800DC00084AD73BC7
:100160003BCE016E84BCBFFDC12F3D6C74319ABD86
:1001700056833DDA3D00C77F11BED9E4BB4C3E91AA
:100180006BAAAABE000000803F05A84CCDB2D44E99
:10019000B93836A9020C50B9918688083CA6AAAA9B
:1001A0002ABE000000803F000D94EA050D94CB05A7
:1001B0000D94F4050D94E1140D940A060D945E0C53
:1001C0000D94B9050D940F060D9402060D94890542
:1001D0000D9406060D9478050D947B050D94FC0591
:1001E0000D94D8050D94D5050D94E6050D949B133B
:1001F0000D94690A0D94BB050D94F8050D94E00566
:100200000D94DC050D94C7050D9477050D944F05ED
:100210000D94EE050D94D105434F4D4D554E494378
:100220004154494F4E0044525952554E0045525286
:100230004F525300494E464F004543484F002074EB
:100240006F6F206C6F6E6720657874727573696F5D
:100250006E2070726576656E7465640A0020636F47
:100260006C6420657874727573696F6E2070726546
:1002700076656E7465640A0047322F4733206261E9
:100280006420706172616D65746572730A00536CED
:100290006565702E2E2E00205A3A200020593A20F3
:1002A0000042656420583A20004C756C7A426F74A5
:1002B0002054415A20362072656164792E005265BF
:1002C00073756D696E67207072696E7400436C6936
:1002D000636B20746F20726573756D652E2E2E0012
:1002E0004E6F206D6F76652E00456E642066696CDA
:1002F00065206C6973740A00426567696E206669DF
:100300006C65206C6973740A004D313235005344BA
:10031000207072696E74696E67206279746520005E
:100320004E6F74205344207072696E74696E670A50
:100330000046696C652064656C657465643A0044C8
:10034000656C6574696F6E206661696C65642C20EC
:1003500046696C653A20006F70656E206661696C55
:1003600065642C2046696C653A2000256973002578
:10037000696D20256973002569682025696D202530
:10038000697300256964202569682025696D202529
:10039000697300256979202569642025696820250D
:1003A000696D20256973005072696E742074696DDF
:1003B000653A2000000125301D0C1824311C0B1754
:1003C000232F1B0A1E16040308060202222B1A41C1
:1003D00042033809FF3628294527444350726F7479
:1003E00065637465642050696E0A0045787472759F
:1003F000646572202573004C756C7A426F742054CA
:10040000415A20362072656164792E003902340227
:100410002D02260218026F66660044454255473A8F
:10042000006F6B00436F6F6C696E6720646F6E6561
:100430002E0048656174696E6720646F6E652E00DA
:1004400020573A00457874727564657220257300F0
:100450004C756C7A426F742054415A203620726574
:100460006164792E0042656420646F6E652E002001
:10047000573A004265642068656174696E672E00B2
:1004800042656420636F6F6C696E672E002F2F20AA
:10049000007A5F70726F62653A20007A5F6D6178F2
:1004A0003A20007A5F6D696E3A2000795F6D61785D
:1004B0003A2000795F6D696E3A2000785F6D61784F
:1004C0003A2000785F6D696E3A20005265706F7255
:1004D00074696E6720656E6473746F7020737461E5
:1004E0007475730A00426564204C6576656C696EAC
:1004F0006720004661696C656420746F20656E61D9
:10050000626C6520426564204C6576656C696E6737
:100510000A00426564204C6576656C20436F7272F8
:10052000656374696F6E204D61747269783A004E2C
:100530006F2063617365206C696768740A004163AA
:10054000746976652045787472756465723A200026
:10055000556E6B6E6F776E20636F6D6D616E643A72
:1005600020220020204E6F7A7A6C653A200020000D
:1005700066696C616D656E7420756E6C6F61640088
:100580005761697420666F72005052494E54205072
:1005900041555345440020204E6F7A7A6C653A20CD
:1005A000006368616E6765006F6620746865206629
:1005B000696C616D656E74005761697420666F7255
:1005C000207374617274005052494E54205041554A
:1005D0005345440020204E6F7A7A6C653A20002003
:1005E000004261636B004D696E696D756D205465E5
:1005F0006D70206973203132302E00486561746956
:100600006E67206661696C65640025753A25303235
:100610007500253032753A25303275002575642015
:10062000253032753A253032750000060900FE008B
:100630000000000001090008FE000005080806008F
:100640000040F0C88888987810050808060000C0A7
:10065000F88888888888F80505050600012030F8A4
:1006600030200508080600002070F820202020E037
:100670000509090600FF2070A8A8B8888870200521
:1006800009090600FFE080C0B0A828302828050925
:10069000090600FFF8A88888888888A8F8050A0A4B
:1006A0000600FE205050505088A8A888700303030D
:1006B00006000340A04000060900FE070192032146
:1006C00020FFFF08FF07FF000000060000010707EA
:1006D00006020080808080800080030202060105FF
:1006E000A0A00507070600005050F850F85050052C
:1006F00007070600002078A07028F02005070706ED
:100700000000C0C8102040981805070706000060C8
:1007100090A040A89068020303060104C040800333
:10072000070706010020408080804020030707065D
:1007300001008040202020408005050506000120A2
:10074000A870A8200505050600012020F820200239
:1007500003030602FFC04080050101060003F80202
:100760000202060200C0C0050505060001081020AF
:100770004080050707060000708888888888700315
:10078000070706010040C040404040E0050707065B
:100790000000708808708080F8050707060000F8E0
:1007A0001020100808F005070706000010305090D0
:1007B000F81010050707060000F880F00808887098
:1007C000050707060000708080F08888700507071D
:1007D000060000F80810202020200507070600006A
:1007E0007088887088887005070706000070888800
:1007F00078080870020505060200C0C000C0C002EB
:1008000006060602FFC0C000C040800407070600BD
:100810000010204080402010050303060002F8006D
:10082000F8040707060100804020102040800507DB
:100830000706000070880810200020050707060042
:100840000070880868A8A87005070706000070886F
:1008500088F8888888050707060000F08888F088EF
:1008600088F0050707060000708880808088700582
:100870000707060000F08888888888F005070706C3
:100880000000F88080F08080F8050707060000F877
:100890008080F0808080050707060000708880B89F
:1008A000888870050707060000888888F888888887
:1008B000010707060200808080808080800507078E
:1008C00006000038101010109060050707060000A1
:1008D0008890A0C0A090880507070600008080804F
:1008E000808080F805070706000088D8A8888888D7
:1008F000880507070600008888C8A8988888050723
:100900000706000070888888888870050707060039
:1009100000F08888F0808080050707060000708856
:100920008888A89068050707060000F08888F0A06E
:100930009088050707060000788080700808F00599
:100940000707060000F820202020202005070706C2
:100950000000888888888888700507070600008856
:1009600088888888502005070706000088888888BE
:1009700088A85005070706000088885020508888FE
:1009800005070706000088888850202020050707F3
:10099000060000F80810204080F803070706010051
:1009A000E08080808080E005050506000180402011
:1009B0001008030707060100E02020202020E005A2
:1009C0000303060004205088050101060000F80218
:1009D0000202060205804005050506000070087841
:1009E00088780507070600008080B0C88888F00571
:1009F0000505060000708080887005070706000066
:100A0000080868988888780505050600007088F849
:100A100080700507070600003048E0404040400570
:100A200006060600FF70888878087005070706002C
:100A3000008080B0C888888801070706020080000F
:100A400080808080800308080601FF20002020208D
:100A500020A040040707060000808090A0C0A0905E
:100A6000030707060100C04040404040E00505057F
:100A7000060000D0A8A8A8A8050505060000B0C873
:100A80008888880505050600007088888870050636
:100A9000060600FFF08888F080800506060600FF45
:100AA000788888780808050505060000B0C88080A9
:100AB0008005050506000070807008F00407070631
:100AC00000004040E0404040300505050600008839
:100AD00088889868050505060000888888502005E4
:100AE00005050600008888A8A85005050506000031
:100AF00088502050880506060600FF8888887808F8
:100B000070050505060000F8102040F803070706E9
:100B1000010020404080404020010707060200807D
:100B2000808080808080030707060100804040208D
:100B300040408005020206000268900000000600A6
:100B40000000000006000000000006000000000099
:100B50000600000000000600000000000600000083
:100B60000000060000000000060000000000060073
:100B70000000000006000000000006000000000069
:100B80000600000000000600000000000600000053
:100B90000000060000000000060000000000060043
:100BA0000000000006000000000006000000000039
:100BB0000600000000000600000000000600000023
:100BC0000000060000000000060000000000060013
:100BD0000000000006000000000006000000000009
:100BE00006000000000006000000000006000000F3
:100BF00000000600000000000600000000000600E3
:100C000000000000060000010707060200800080C7
:100C1000808080800507070600002070A8A0A870CB
:100C200020050707060000304040E04050A80505B9
:100C300005060000887050708805070706000088C8
:100C40005020F820F820010707060200808080006D
:100C50008080800508080600003048205050209011
:100C600060030101060107A0050707060000F888D8
:100C7000B8B8B888F80507070600017008788878C2
:100C800000F80505050600012850A05028050303BB
:100C9000060001F808080202020602064080050765
:100CA00007060000F888A88898A8F8050101060042
:100CB00006F8040404060003609090600507070628
:100CC00000002020F8202000F8040505060003603D
:100CD000902040F0030505060003E020E020E0023C
:100CE000020206020640800508080600FF88888880
:100CF0008898E8808005070706000078989878189B
:100D00001818020202060202C0C00202020602FF16
:100D1000408003050506000340C04040E00507078A
:100D2000060001708888887000F805050506000136
:100D3000A0502850A00507070600008890A858B8C2
:100D400008080507070600008890B848982038056D
:100D50000808060000C040C048D838080805070742
:100D6000060000200020408088700508080600006A
:100D70004020007088F888880508080600001020C8
:100D8000007088F888880508080600002050007068
:100D900088F888880508080600006890007088F8C0
:100DA00088880508080600005000708888F8888840
:100DB0000508080600002050207088F8888805077C
:100DC000070600003860A0B8E0A0B80508080600D3
:100DD000FF70888080887020600508080600004049
:100DE0002000F880F080F8050808060000081000D0
:100DF000F880F080F8050808060000205000F88010
:100E0000F080F80507070600005000F880F080F831
:100E1000030808060100804000E0404040E003086D
:100E200008060100204000E0404040E003080806BA
:100E3000010040A000E0404040E003070706010039
:100E4000A000E0404040E005070706000070484869
:100E5000E848487005080806000068900088C8A89F
:100E600098880508080600004020708888888870E7
:100E7000050808060000102070888888887005081A
:100E80000806000020500070888888700508080651
:100E900000006890007088888870050808060000C7
:100EA0005000708888888870050505060001885004
:100EB0002050880508080600FF1070A8A8A8A87090
:100EC000400508080600004020888888888870054A
:100ED000080806000010208888888888700508089F
:100EE00006000020500088888888700508080600E1
:100EF000005000888888888870050808060000105F
:100F0000208850202020200509090600FFC04070DD
:100F10004848704040E00408080601FF609090A037
:100F20009090E080050808060000402000700878D6
:100F30008878050808060000102000700878887876
:100F40000508080600002050007008788878050819
:100F50000806000068900070087888780507070682
:100F60000000500070087888780508080600002006
:100F700050207008788878050606060000D028788A
:100F8000A0A8500506060600FF7080887020600546
:100F900008080600004020007088F88070050808E6
:100FA0000600001020007088F88070050808060010
:100FB000002050007088F880700507070600005078
:100FC000007088F880700308080601008040004027
:100FD000C04040E003080806010020400040C04037
:100FE00040E003080806010040A00040C04040E087
:100FF000030707060100A00040C04040E0050707C6
:10100000060000A040A010788870050808060000BF
:10101000689000B0C888888805080806000040204D
:10102000007088888870050808060000102000708D
:10103000888888700508080600002050007088889D
:10104000887005080806000068900070888888701D
:1010500005070706000050007088888870050505A0
:101060000600012000F800200507070600FF1070A9
:10107000A8A8A8704005080806000040200088883D
:10108000889868050808060000102000888888985D
:1010900068050808060000205000888888986805C0
:1010A0000707060000500088888898680509090627
:1010B00000FF102000888888F808700407070601E0
:1010C000FFC04060506040E00508080600FF500087
:1010D0008888887808705A00590058000920000054
:1010E00000000000000000000000007FFFE00000A2
:1010F000000000000000000000007000E0000000A0
:1011000000000000000000000061F8600000000026
:10111000000000000000000041F820000000000076
:101120000000000000000040F0200000000000006F
:1011300000000000000040602000000000000000EF
:1011400000000000005801A07F80000000000000A7
:10115000004104005C63A0FFC0000000000000002C
:101160002082005EF7A0FFC0000000000000002009
:1011700082005EF7A0FFC0000000000000004104F4
:10118000005C63A07F800000000000000082080077
:101190005801A07F80000000000000010410004002
:1011A0006020FFC00000000000000104100040F0BB
:1011B00020FFC00000000000000082080041F8206D
:1011C000FFC00000000000000041040061F8603F23
:1011D00000000000000000000000007000E01E00A1
:1011E00000000000000001FFFF807FFFE00C000016
:1011F000000000000001FFFF800000000000000070
:1012000000000000000000007FFFE0000000000080
:10121000000000000000007000E00000000000007E
:10122000000000000000630C6000000000000000EF
:101230000000000000470E20000000000000000039
:10124000000000004F0F2000000000000000000020
:101250000000005F0FA00000000000000000000080
:1012600000005E07A07F8000000000000000410435
:1012700000406020FFC0000000000000002082004D
:1012800040F020FFC000000000000000208200406D
:10129000F020FFC00000000000000041040040609A
:1012A000207F80000000000000008208005E07A090
:1012B0007F80000000000000010410005F0FA0FF0D
:1012C000C0000000000000010410004F0F20FFC00C
:1012D00000000000000000820800470E20FFC00050
:1012E000000000000000410400630C603F000000AB
:1012F00000000000000000007000E01E0000000080
:1013000000000001FFFF807FFFE00C0000000000F4
:10131000000001FFFF8000000000002200250028DF
:10132000002B002E003100340002010000050108EE
:10133000010B0100000A0B02090C0D0E0807030443
:10134000010000000000000000000000000000009C
:10135000000000000000000000000000000000127B
:10136000111000000000000000000000000000005C
:1013700000000000000000000043290A0061626CC8
:10138000656420286D696E2074656D702000436F60
:101390006C64206578747275646573206172652071
:1013A0000045313A200045303A20005A3A20005991
:1013B0003A2000583A20004D53312C4D53322050E2
:1013C000696E730A002042002050006F6B00526566
:1013D00073656E643A20001000C90210012C0140B0
:1013E00001220170011801B0010E01F00104015049
:1013F00002FA00B002F0003003E600D003DC0090F7
:1014000004D2007005C800A006BE000008B400B0F9
:1014100009AA00D00BA000600E960060118C00009D
:1014200015820020197800C01D6E00A0226400B053
:10143000275A00902C500000314600E0343C001048
:10144000383200903A2800603C1E00A03D14008015
:101450003E0A00203F00004361703A454D45524727
:10146000454E43595F5041525345523A310A004369
:1014700061703A434153455F4C494748545F42527B
:10148000494748544E4553533A300A004361703A35
:10149000544F47474C455F4C49474854533A300AEC
:1014A000004361703A534F4654574152455F504F85
:1014B0005745523A300A004361703A4C4556454C04
:1014C000494E475F444154413A310A004361703A02
:1014D0005A5F50524F42453A310A004361703A41D7
:1014E00055544F4C4556454C3A310A004361703AC9
:1014F0005052494E545F4A4F423A310A004361709C
:101500003A50524F47524553533A300A00436170A4
:101510003A4155544F5245504F52545F54454D50E7
:101520003A310A004361703A454550524F4D3A31C5
:101530000A004649524D574152455F4E414D453A8A
:101540004D61726C696E20204649524D574152459B
:101550005F56455253494F4E3A312E312E352E3675
:10156000342045585452554445525F545950453AD9
:1015700053696E676C654578747275646572205343
:101580004F555243455F434F44455F55524C3A686F
:10159000747470733A2F2F636F64652E616C65707D
:1015A000686F626A656374732E636F6D2F6469661A
:1015B000667573696F6E2F4D41524C494E205052E3
:1015C0004F544F434F4C5F56455253494F4E3A315B
:1015D0002E30204D414348494E455F545950453ABD
:1015E0004C756C7A426F742054415A20362045580D
:1015F0005452554445525F434F554E543A3120554D
:101600005549443A38343566303033632D6165626C
:10161000642D346535332D613662392D37643039A8
:1016200038346664653630390A004D31343520531C
:101630003C696E6465783E206F7574206F66207219
:10164000616E67652028302D31290A0020706F7384
:101650006974696F6E206F7574206F662072616E99
:1016600067652E0A003F50726F626520001000AD62
:101670000330016A0150022B0170030A019004F546
:1016800000B005E500D006D800F007CE001009C56F
:1016900000300ABE00500BB700700CB100900DABCB
:1016A00000B00EA600D00FA200F0109D00101299FD
:1016B00000301395005014920070158E0090168B18
:1016C00000B0178700D0188400F0198100101B7E2D
:1016D00000301C7B00501D7900701E7600901F7337
:1016E00000B0207000D0216E00F0226B0010246941
:1016F0000030256600502663007027610090285E48
:1017000000B0295C00D02A5900F02B5600102D544F
:1017100000302E5100502F4E0070304B0090314859
:1017200000B0324500D0334200F0343E0010363B6A
:1017300000303737005038330070392E00903A2986
:1017400000B03B2300D03C1B00F03D1100103F01D6
:1017500000F03F000020204D383531205A005A2D2E
:1017600050726F6265204F666673657420286D6DD8
:10177000293A0A0020440020490020204D3330340B
:1017800020500020440020490020204D33303120DB
:1017900050005049442073657474696E67733A0A47
:1017A0000020460020420020480020204D313435E2
:1017B0002053004D6174657269616C2068656174C5
:1017C000757020706172616D65746572733A0A009C
:1017D00020204D3432302053004175746F20426513
:1017E00064204C6576656C696E673A0A00205A0081
:1017F00020590020204D323036205800486F6D654A
:10180000206F66667365743A0A00204500205A000E
:1018100020590020580020420020540020204D3242
:101820003035205300416476616E6365643A20531D
:101830003C6D696E5F66656564726174653E2054D7
:101840003C6D696E5F74726176656C5F6665656438
:10185000726174653E20423C6D696E5F7365676DB1
:10186000656E745F74696D655F6D733E20583C6D85
:1018700061785F78795F6A65726B3E205A3C6D6172
:10188000785F7A5F6A65726B3E20453C6D61785F78
:10189000655F6A65726B3E0A00205400205200208A
:1018A000204D323034205000416363656C657261B5
:1018B00074696F6E2028756E6974732F7332293ABC
:1018C00020503C7072696E745F616363656C3E208A
:1018D000523C726574726163745F616363656C3EF0
:1018E00020543C74726176656C5F616363656C3E25
:1018F0000A00204500205A0020590020204D323097
:10190000312058004D6178696D756D2041636365C4
:101910006C65726174696F6E2028756E6974732FBF
:101920007332293A0A00204500205A00205900202D
:10193000204D3230332058004D6178696D756D202F
:101940006665656472617465732028756E69747369
:101950002F73293A0A00204500205A002059002000
:10196000204D3932205800537465707320706572B1
:1019700020756E69743A0A0020204D3230302044C0
:10198000300A0020204D323030204400204469735A
:1019900061626C65640A0046696C616D656E7420F5
:1019A00073657474696E67733A0020204D31343961
:1019B0002043203B20556E69747320696E20436577
:1019C0006C736975730A0020204732312020202073
:1019D0003B20556E69747320696E206D6D0A003A64
:1019E00020007A5F6D696E3A20202D32207A5F6D7B
:1019F00061783A202035005A204F6666736574205E
:101A000000506C6561736520726573657400505297
:101A1000494E5445522048414C5445440050726947
:101A20006E7465722068616C7465642E206B696CDD
:101A30006C28292063616C6C6564210A006265640E
:101A40000A002C2073797374656D2073746F707045
:101A5000656421204865617465725F49443A2000DD
:101A6000544845524D414C2052554E415741592002
:101A700042454400546865726D616C2052756E6118
:101A800077617900544845524D414C2052554E41A2
:101A900057415920453100544845524D414C205240
:101AA000554E415741592045300048656174696E73
:101AB00067206661696C6564204245440048656141
:101AC00074696E67206661696C656400486561745D
:101AD000696E67206661696C656400486561746958
:101AE0006E67206661696C656420453000577269D5
:101AF00074696E6720746F2066696C653A20006FA8
:101B000070656E206661696C65642C2046696C6541
:101B10003A20006F70656E206661696C65642C20E8
:101B200046696C653A200046696C652073656C6592
:101B3000637465640A002053697A653A2000466937
:101B40006C65206F70656E65643A20006F70656E1D
:101B5000206661696C65642C2046696C653A2000DA
:101B60002066696C653A20004E6F77200022207055
:101B70006F73002220706172656E743A22005355B3
:101B800042524F5554494E452043414C4C207461BC
:101B9000726765743A22004B494C4C45442E200034
:101BA000747279696E6720746F2063616C6C207346
:101BB00075622D67636F64652066696C6573207755
:101BC00069746820746F6F206D616E79206C657622
:101BD000656C732E204D4158206C6576656C2069CC
:101BE000733A004572726F722077726974696E671A
:101BF00020746F20454550524F4D210A00486F6DAB
:101C0000652025732573257320666972737400201F
:101C100066697273740A005A0059005800486F6D63
:101C200065200000060900FE06018902FE20FFFE75
:101C300007FE06FE00000006000701060606020079
:101C4000808080800080030303060103A0A0A0051C
:101C500007070600FF5050F850F8505005090906D4
:101C600000FE2070A8A07028A870200608080600B2
:101C7000FF40A84810204854080507070600FF60E9
:101C800090906098906801030306020380808002B0
:101C900007070602FF408080808080400207070619
:101CA00002FF804040404040800505050600008856
:101CB00050F850880505050600002020F820200275
:101CC00004040602FEC0404080050101060002F83F
:101CD000020202060200C0C004060606010010103F
:101CE000204080800406060601006090909090607D
:101CF00003060606010040C0404040E00406060618
:101D000001006090102040F0040606060100F0205B
:101D1000601010E005060606000010305090F81024
:101D2000040606060100F080E01010E00406060636
:101D300001006080E0909060040606060100F0104B
:101D400010204040040606060100609060909060FC
:101D500004060606010060909070106002050506FA
:101D60000200C0C000C0C00207070602FEC0C000DB
:101D7000C040408005050506000018608060180519
:101D80000303060001F800F8050505060000C03051
:101D90000830C00407070601006090106040004052
:101DA0000506060600007090A8B0807005060606BD
:101DB0000000205088F88888050606060000F08894
:101DC000F08888F00406060601006090808090602C
:101DD000040606060100E090909090E004060606D6
:101DE0000100F080E08080F0040606060100F0802B
:101DF000E0808080040606060100609080B090605C
:101E00000406060601009090F090909003060606E6
:101E10000100E040404040E00506060600003810A2
:101E20001010906004060606010090A0C0A09090DB
:101E30000406060601008080808080F00506060604
:101E4000000088D8A8A8888804060606010090D05B
:101E5000B09090900506060600007088888888700B
:101E6000040606060100E09090E080800407070663
:101E700001FF609090D0B06010040606060100E0FB
:101E80009090E0909004060606010060904020903B
:101E900060050606060000F8202020202004060623
:101EA0000601009090909090600406060601009054
:101EB0009090F060600506060600008888A8A8D803
:101EC0008805060606000088502020508805060672
:101ED000060000888850202020040606060100F035
:101EE00010204080F0030606060100E0808080801C
:101EF000E00406060601008080402010100306065C
:101F0000060100E020202020E00503030600032056
:101F100050880501010600FEF80202020602048054
:101F20004004040406010070909070040606060147
:101F3000008080E09090E00404040601007080803E
:101F400070040606060100101070909070040404DE
:101F500006010060B0C07004060606010020504073
:101F6000E040400406060601FE6090907010600498
:101F700006060601008080E09090900306060601A8
:101F8000004000C04040E00308080601FE20006059
:101F9000202020A0400406060601008080A0C0A0EA
:101FA00090030606060100C040404040E0050404DE
:101FB000060000D0A8A888040404060100E0909060
:101FC0009004040406010060909060040606060177
:101FD000FEE09090E080800406060601FE7090907E
:101FE000701010040404060100A0D08080040404D2
:101FF00006010070C030E00406060601004040E023
:1020000040502004040406010090909070040404E1
:102010000601009090606005040406000088A8A8EE
:102020005004040406010090606090040606060156
:10203000FE909090709060040404060100F020402F
:10204000F0030707060100204040804040200107C0
:10205000070602FF808080808080800307070601DA
:10206000008040402040408004020206010350A04E
:10207000FFFFFFFFFFFFFFFFFFFFFFFFFFFFFFFF70
:10208000FFFFFFFFFFFFFFFFFFFFFFFFFFFFFFFF60
:10209000FF0000000600070106060602008000801F
:1020A0008080800406060601FF2070A0A070200535
:1020B00007070600FF304840F04040F805050506D8
:1020C0000000A8508850A80506060600008850F8B1
:1020D00020F8200107070602FF80808000808080B2
:1020E0000407070601FF708060906010E0030101A3
:1020F000060105A0060707060000788494A49484CE
:102100007803050506010160A06000E005050506ED
:1021100000002850A05028040303060100F010100E
:10212000040101060102F00607070600007884B4E6
:10213000A4A48478040101060105F0040303060148
:10214000026090600507070600FF2020F8202000AD
:10215000F803050506010140A02040E0030505063F
:102160000101C0204020C002020206020440800497
:1021700005050601FF9090B0D08005060606000018
:1021800078E8E868282801010106020280020202BC
:102190000602FE408003050506010140C04040E004
:1021A00003050506010140A04000E0050505060005
:1021B00000A0502850A00508080600FF40C040506D
:1021C000703078100508080600FF40C040506808CD
:1021D00010380508080600FFC0204030F0307810A5
:1021E00004070706010020002060809060050707B3
:1021F0000600004020205070888805070706000070
:102200001020205070888805070706000020502005
:1022100050708888050707060000285020507088F5
:1022200088050707060000500020507088880507C1
:10223000070600002050205070888805060606001A
:102240000078A0F0A0A0B80408080601FE60908005
:1022500080906020400407070601004020F080E0E5
:1022600080F00407070601002040F080E080F004C1
:1022700007070601002050F080E080F00407070601
:1022800001005000F080E080F003070706010080A5
:1022900040E0404040E00307070601002040E040E6
:1022A0004040E003070706010040A0E0404040E056
:1022B000030707060100A000E0404040E0050606D5
:1022C0000600007048E848487004070706010050FF
:1022D000A090D0B0909004070706010040206090C5
:1022E0009090600407070601002040609090906085
:1022F00004070706010020506090909060040707D3
:1023000006010050A060909090600407070601004D
:1023100050006090909060050505060000885020F0
:1023200050880408080601FF1070B0B0D0D0E080DB
:102330000407070601004020909090906004070772
:10234000060100204090909090600407070601006D
:102350002050909090906004070706010050009074
:1023600090909060050707060000102088502020FC
:102370002004060606010080E09090E08004060636
:102380000601006090A0A090A0040707060100408D
:102390002000709090700407070601002040007034
:1023A0009090700407070601002050007090907014
:1023B00004070706010050A0007090907004060604
:1023C000060100500070909070040707060100207D
:1023D00050207090907005040406000070A8B0783A
:1023E0000406060601FE7080807020400407070680
:1023F000010040200060B0C0700407070601002003
:10240000400060B0C0700407070601002050006063
:10241000B0C070040606060100500060B0C0700332
:102420000707060100804000C04040E003070706A0
:102430000100204000C04040E003070706010040C3
:10244000A000C04040E0030606060100A000C04016
:1024500040E00407070601003060107090906004AF
:10246000070706010050A000E090909004070706BF
:1024700001004020006090906004070706010020E2
:102480004000609090600407070601002050006043
:1024900090906004070706010050A00060909060D3
:1024A00004060606010050006090906005050506D0
:1024B00000002000F8002004040406010070B0D0E1
:1024C000E004070706010040200090909070040788
:1024D0000706010020400090909070040707060155
:1024E00000205000909090700406060601005000F5
:1024F000909090700409090601FE20400090909091
:102500007090600408080601FE8080E09090E080F2
:10251000800408080601FE50009090907090605270
:1025200065776970696E670050726F62696E6720C7
:102530006661696C65640050726F62696E672066DF
:1025400061696C65640050524F4245204641494CD8
:1025500020434C45414E204E4F5A5A4C450A00529A
:1025600065776970696E670A005265776970696E90
:10257000670050726F62696E67206661696C65649E
:102580000050726F62696E67206661696C656400F5
:1025900050524F4245204641494C20434C45414E04
:1025A000204E4F5A5A4C450A005265776970696E41
:1025B000670A0050726F62696E67206661696C65B8
:1025C000640A0050726F62696E67206661696C65AB
:1025D0006400205A3A200020593A200042656420C5
:1025E000583A20000A0A426564204C6576656C20E2
:1025F000436F7272656374696F6E204D61747269A6
:10260000783A00202B000A436F7272656374656428
:1026100020426564204865696768742076732E20BF
:1026200042656420546F706F6C6F67793A0A0020BE
:102630002B000A4265642048656967687420546FFE
:10264000706F6772617068793A0A2020202B2D2DF7
:102650002D204241434B202D2D2B0A2020207C2071
:10266000202020202020202020207C0A204C207C9C
:1026700020202020282B29202020207C20520A20C6
:1026800045207C20202020202020202020207C206D
:10269000490A2046207C20282D29204E20282B293D
:1026A000207C20470A2054207C202020202020202D
:1026B000202020207C20480A2020207C2020202050
:1026C000282D29202020207C20540A2020207C2016
:1026D000202020202020202020207C0A2020204F85
:1026E0002D2D2046524F4E54202D2D2B0A202830C0
:1026F0002C30290A004D65616E206F662073616D74
:10270000706C656420706F696E74733A2000206489
:102710003A200020623A200045716E20636F6566A2
:1027200066696369656E74733A20613A2000527578
:102730006E6E696E6720696E204452592D52554E57
:10274000206D6F64650A00473239204175746F202F
:10275000426564204C6576656C696E670A002842A4
:102760002961636B00284629726F6E740028522914
:102770006967687400284C29656674003F4E756D62
:10278000626572206F662070726F626520706F697B
:102790006E747320697320696D706C617573696202
:1027A0006C65202832206D696E696D756D292E0A61
:1027B000003F2856296572626F7365206C657665E7
:1027C0006C20697320696D706C61757369626C65EA
:1027D0002028302D34292E0A00534420636172646E
:1027E000206F6B0A006F70656E526F6F74206661A8
:1027F000696C65640A00766F6C756D652E696E692B
:1028000074206661696C65640A00534420696E69CE
:1028100074206661696C0A0043616E6E6F74206596
:102820006E746572207375626469723A2000022EBC
:102830002E004D61696E004D6F766520302E316D32
:102840006D004D6F766520316D6D004D6F766520A2
:1028500031306D6D004D6F7665206178697300458C
:1028600078747275646572004D6F7665205A004DFC
:102870006F76652059004D6F7665205800746F2083
:10288000726573756D65005761697420666F72209B
:102890007072696E74005052494E54205041555325
:1028A00045440045787472756465206D6F726500EB
:1028B000526573756D65207072696E740052455370
:1028C000554D45204F5054494F4E533A0020204E0D
:1028D0006F7A7A6C653A20002000506C65617365F0
:1028E00020776169742E2E2E0048656174696E67C9
:1028F000206E6F7A7A6C65005052494E54205041D8
:10290000555345440020204E6F7A7A6C653A20007A
:10291000200068656174206E6F7A7A6C652E0050B5
:102920007265737320627574746F6E20746F0050DB
:1029300052494E54205041555345440020204E6F7B
:102940007A7A6C653A2000200066696C616D656E6C
:1029500074206578747275646500576169742066C7
:102960006F72005052494E54205041555345440017
:1029700020204E6F7A7A6C653A2000200066696CE0
:10298000616D656E74206C6F6164005761697420BD
:10299000666F72005052494E542050415553454481
:1029A0000020204E6F7A7A6C653A2000746F2063A5
:1029B0006F6E74696E75652E2E2E00616E642070C8
:1029C0007265737320627574746F6E00496E7365FF
:1029D00072742066696C616D656E74005052494E68
:1029E000542050415553454400656E7175657565B9
:1029F000696E672022007C3C3E5E2B3D3F2F5B5D75
:102A00003B2C2A225C0043616E6E6F74206F7065F0
:102A10006E20737562646972200001050800FF066C
:102A20000121023520FFFF07FF06FF090050221693
:102A300056808080800080153353A0A0A002575795
:102A40005050F850F850500257572070A07028701E
:102A50002013355580A040A02002475740A0A04039
:102A6000A0A050251353808080122656408080807D
:102A7000804012265680404040408002455590607C
:102A8000F060900255552020F8202011335360400B
:102A900080044151F011335340E04002465610107B
:102AA0002040808012365640A0A0A0A0401236568A
:102AB00040C0404040E00246566090106080F00206
:102AC0004656F020601090600246562060A0F0202C
:102AD00020024656F080E01090600246566080E08A
:102AE000909060024656F01020204040024656600A
:102AF0009060909060024656609090701060122531
:102B000055C0C000C0C011365660600060408012E1
:102B10003656204080804020034353F000F01236A8
:102B20005680402020408012365640A02040004071
:102B3000015858304898A8A89040300246566090F6
:102B400090F09090024656E090E09090E002465659
:102B5000609080809060024656E090909090E002F5
:102B60004656F080E08080F0024656F080E080809B
:102B700080024656609080B090600246569090F079
:102B8000909090123656E040404040E00246567029
:102B9000202020A04002465690A0C0A0A09002464F
:102BA000568080808080F002465690F0F0909090A1
:102BB00002465690D0F0B0B0900246566090909089
:102BC0009060024656E09090E08080014757609008
:102BD00090D0B06010024656E09090E0909002468F
:102BE00056609040209060123656E0404040404091
:102BF0000246569090909090600246569090909029
:102C00006060024656909090F0F090024656909088
:102C100060609090025656888850202020024656C8
:102C2000F010204080F0123656E080808080E00274
:102C30004656808040201010123656E0202020207A
:102C4000E016325240A0014151F01622528040025B
:102C50004454709090700246568080E09090E0124C
:102C6000345460808060024656101070909070025C
:102C7000445460B0C060024656205040E0404001DD
:102C8000455560907010600246568080E0909090AC
:102C90001236564000C04040E01137572000202037
:102CA00020A040024656808090E09090123656C098
:102CB00040404040E0025454D0A8A8A8024454E048
:102CC00090909002445460909060014555E090E0EF
:102CD00080800145557090701010024454A0D0803F
:102CE0008012345460C020C00246564040E040503C
:102CF0002002445490909070123454A0A0A040023E
:102D0000545488A8A85002445490606090014555DE
:102D10009090709060024454F02040F00247573089
:102D20004020C02040302216568080808080800263
:102D30004757C02040304020C006425250A0FFFFFD
:102D4000FFFFFFFFFFFFFFFFFFFFFFFFFFFFFFFF93
:102D5000FFFFFFFFFFFFFFFFFFFFFFFFFFFFFF0979
:102D600000502216568000808080800146562070D8
:102D7000A0A070200246562050E04050A0025555B9
:102D800088705070880256568850F820F820221714
:102D900057808080008080800247577080E090706C
:102DA00010E0173151A002565670A8C8C8A8701478
:102DB000355560A06000E003435350A050123353D8
:102DC000E02020143151E002565670E8D8E8D8705F
:102DD000173151E015335340A04012355540E040C3
:102DE00000E014355540A02040E0143555C020C007
:102DF00020C01622524080014555909090E08002FC
:102E0000565678E8E868282824115180112252404B
:102E10008014355540C04040E014355540A0400076
:102E2000E0034353A050A0024757808080A060F089
:102E3000200247578080A0D0102070024757804062
:102E40008060A0F02012365640004080A04002472B
:102E50005740206090F0909002475720406090F0DB
:102E6000909002475760906090F0909002475750C2
:102E7000A06090F0909002475790006090F0909082
:102E800002475760906090F0909002465670A0A064
:102E9000F0A0B00147576090808090604002475793
:102EA0004020F080E080F00247572040F080E08032
:102EB000F00247576090F080E080F00247579000A2
:102EC000F080E080F01237578040E0404040E01250
:102ED00037572040E0404040E012375740A0E040E4
:102EE0004040E0123757A000E0404040E002565614
:102EF0007048E848487002475750A090D0B0909072
:102F000002475740206090909060024757204060F1
:102F10009090906002475760906090909060024758
:102F20005750A0609090906002475790006090903A
:102F30009060123353A040A002465670B0B0D0D07B
:102F4000E002475740209090909060024757204001
:102F5000909090906002475760909090909060029F
:102F600047579000909090906002575710208850DB
:102F700020202002465680E09090E0800246566075
:102F800090A0A090A002475740200070909070023F
:102F900047572040007090907002475720500070B3
:102FA00090907002475750A0007090907002465663
:102FB00050007090907002475760906070909070D1
:102FC000025454F068B0781135556080806040023A
:102FD000475740200060B0C0600247572040006063
:102FE000B0C06002475760900060B0C060024656B3
:102FF000500060B0C060123757804000C04040E0D1
:10300000123757204000C04040E012375740A00020
:10301000C04040E0123656A000C04040E002475792
:10302000A040A01070906002475750A000E0909020
:103030009002475740200060909060024757204020
:10304000006090906002475760900060909060022E
:10305000475750A0006090906002465690006090E4
:1030600090601235554000E0004002445470B0D0EA
:10307000E002475740200090909070024757204050
:10308000009090907002475760900090909070026E
:1030900046569000909090700148582040009090C3
:1030A0007090600147578080E090E0808001475732
:1030B0009000909070906001050700FE0500FB01F4
:1030C000F220FFFE05FE05FE02004002152580806D
:1030D000800080053242A0A002556550F850F8509B
:1030E0000146562070C030E0200255659010204007
:1030F000480255656080689068051222808002252C
:103100003540808080400225358040404080043337
:1031100043A040A003334340E040012232408004FA
:103120003141E002112180025565081020408002E3
:1031300045556090909060022535C0404040400267
:103140004555E0106080F0024555E0106010E00247
:1031500045552060A0F020024555F080E010E002C7
:1031600045556080E09060024555F01020404002D7
:103170004555609060906002455560907010600306
:1031800013238000800214248000808002354520B3
:1031900040804020033343E000E00235458040207A
:1031A0004080024555E0106000400255657088B8C7
:1031B000A870024555609090F090024555E090E06F
:1031C00090E00235456080808060024555E0909037
:1031D00090E0023545E080E080E0023545E080E0A7
:1031E00080800245557080B090700245559090F0F7
:1031F0009090023545E0404040E0024555301010C7
:10320000906002455590A0C0A09002354580808016
:1032100080E002556588D8A8888802455590D0B0CE
:1032200090900245556090909060024555E09090D6
:10323000E080014656609090906010024555E09005
:1032400090E09002455570806010E0023545E04006
:1032500040404002455590909090600245559090B6
:10326000A0A04002556588A8A8A850024555909096
:103270006090900245559090701060023545E020B6
:103280004080E0022535C0808080C00255658040C6
:10329000201008022535C0404040C005324240A001
:1032A000024151F0052232804002445470909070E7
:1032B00002455580E09090E00234446080806002D6
:1032C0004555107090907002445460B0C060023553
:1032D000452040E0404000465670909070106002DB
:1032E000455580E0909090021525800080808000F8
:1032F0002737400040404040800245558090A0E084
:10330000900215258080808080025464F0A8A8A8CF
:10331000024454E0909090024454609090600046C3
:1033200056E09090E08080004656709090701010AB
:10333000023444A0C0808002445470C030E00235A2
:103340004540E04040200244549090907002445424
:103350009090A040025464A8A85050023444A04069
:1033600040A0004656909090701060024454F020A7
:1033700040F0023545604080406002152580808025
:103380008080023545C0402040C005425250A0FF19
:10339000FFFFFFFFFFFFFFFFFFFFFFFFFFFFFFFF3D
:1033A000FFFFFFFFFFFFFFFFFFFFFFFFFFFFFFFF2D
:1033B000020040FFFFFFFFFFFFFFFFFFFFFFFFFFD8
:1033C000FFFFFFFFFFFFFFFFFFFFFFFFFFFFFFFF0D
:1033D000FFFFFFFFFFFFFFFFFFFFFFFFFFFFFFFFFD
:1033E000FFFFFFFFFFFFFFFFFFFFFFFFFFFFFFFFED
:1033F000FFFFFFFFFFFFFFFFFFFFFFFFFFFFFFFFDD
:10340000FFFFFFFFFFFFFFFFFFFFFFFFFFFFFFFFCC
:10341000FFFF01060D00FE09016602D620FFFE0B2C
:10342000FE0AFE0D00602219698080808080808005
:103430000080183363A0A0A00357675050F850F8DD
:1034400050500259692078A0A0702828F020025915
:103450006948A85010204050A89002586840A0A089
:1034600040A0989068281363808080113B6B2040B7
:10347000408080808080404020113B6B8040402015
:103480002020202040408006556520A870A82004F8
:1034900055652020F820201133636040800651617B
:1034A000F811336340E040025969080810102040C9
:1034B000408080025969205088888888885020027E
:1034C00059692060A02020202020F80259697088C6
:1034D000880810204080F8025969F8081020700808
:1034E000088870025969101030505090F81010027E
:1034F0005969F88080B0C8080888700259697088D6
:103500008080F088888870025969F808101020209F
:1035100040404002596970888888708888887002A5
:10352000596970888888780808887011386840E080
:1035300040000040E04011386840E040000060403A
:10354000800259690810204080402010080454640B
:10355000F80000F8025969804020100810204080CF
:10356000025969708888081020200020025969706B
:10357000888898A8A8B080780259692050888888DF
:10358000F8888888025969F048484870484848F0E7
:10359000025969708880808080808870025969F043
:1035A00048484848484848F0025969F8808080F007
:1035B000808080F8025969F8808080F08080808067
:1035C000025969708880808098888870025969885B
:1035D000888888F888888888123969E040404040A7
:1035E000404040E0025969381010101010109060EF
:1035F000025969888890A0C0A09088880259698083
:1036000080808080808080F80259698888D8A8A846
:103610008888888802596988C8C8A8A8989888881E
:10362000025969708888888888888870025969F08A
:10363000888888F080808080015A6A7088888888AD
:103640008888A87008025969F0888888F0A0908856
:1036500088025969708880807008088870025969EA
:10366000F82020202020202020025969888888887E
:1036700088888888700259698888888850505020C6
:103680002002596988888888A8A8A8A85002596982
:103690008888505020505088880259698888505036
:1036A0002020202020025969F80810102040408076
:1036B000F8113B6BE0808080808080808080E00219
:1036C0005969808040402010100808113B6BE020B1
:1036D0002020202020202020E00853632050880153
:1036E0005161F82A226280400256667008788898F4
:1036F00068025969808080F088888888F002566660
:1037000070888080887002596908080878888888DD
:1037100088780256667088F8808870025969304847
:103720004040F040404040005868708888887808E1
:103730008870025969808080B0C88888888812386B
:10374000684000C040404040E0004A6A100030102D
:1037500010101090906002596980808090A0C0A0E5
:103760009088123969C040404040404040E00256D5
:1037700066D0A8A8A8A888025666B0C88888888895
:10378000025666708888888870005868F088888833
:10379000F080808000586878888888780808080257
:1037A0005666B0C880808080025666708860108837
:1037B000700258684040F0404040483002566688E9
:1037C00088888898680256668888885050200256F3
:1037D000668888A8A8A8500256668850202050887D
:1037E0000058688888889868088870025666F810BB
:1037F000204080F8015B6B1820202020C020202072
:103800002018221969808080808080808080015B00
:103810006BC0202020201820202020C0085363489F
:10382000A890FFFFFFFFFFFFFFFFFFFFFFFFFFFF6E
:10383000FFFFFFFFFFFFFFFFFFFFFFFFFFFFFFFF98
:10384000FFFFFF0D0060221969800080808080806A
:1038500080800358682070A8A0A0A8702002596931
:1038600030484040E0404048B003566688705050B1
:10387000708802596988885050F820F82020221951
:1038800069808080800080808080124A6A60908099
:10389000609090601090601A3262A0A00359697025
:1038A00088A8D8C8D8A8887004576770087888781E
:1038B00000F80356662850A0A05028045363F80867
:1038C00008163161E00359697088E8D8D8E8D888CB
:1038D000700A5161F8174464609090600357672044
:1038E00020F8202000F807356540A02040E007358B
:1038F0006540A04020C02A22624080005868888825
:10390000888898E8808002596978E8E8E8E86828BB
:103910002828262161C0202262408007356540C0EA
:103920004040E0045767708888887000F803566646
:10393000A050282850A0025A6A40C04040E0081811
:10394000283808025A6A40C04040E0102808103861
:10395000025A6A40A04020A0481828380802596935
:10396000200020204080888870025A6A4020002071
:10397000508888F88888025A6A1020002050888869
:10398000F88888025A6A30480020508888F8888869
:10399000025A6A28500020508888F88888025A6A9B
:1039A00050500020508888F88888025A6A20502099
:1039B00020508888F8888802596958A0A0A0B0E0F3
:1039C000A0A0B8005B6B70888080808080887020A9
:1039D00040025A6A402000F88080F08080F8025A45
:1039E0006A102000F88080F08080F8025A6A30481F
:1039F00000F88080F08080F8025A6A505000F88009
:103A000080F08080F8123A6A804000E040404040F8
:103A100040E0123A6A204000E04040404040E0125E
:103A20004A6A609000E04040404040E0123A6AA09C
:103A3000A000E04040404040E0025969F04848485A
:103A4000E8484848F0025A6A2850008888C8A89870
:103A50008888025A6A4020007088888888887002A6
:103A60005A6A10200070888888888870025A6A30E4
:103A7000480070888888888870025A6A28500070C8
:103A8000888888888870025A6A50500070888888B0
:103A90008888700355658850205088015B6B0870DA
:103AA0009898A8A8A8C8C87080025A6A40200088C0
:103AB000888888888870025A6A10200088888888D8
:103AC000888870025A6A3048008888888888887098
:103AD000025A6A50500088888888888870025A6A1A
:103AE0001020008888502020202002596980F0880A
:103AF0008888F0808080025969609090A0A09088AA
:103B000088B0025969402000700878889868025986
:103B10006910200070087888986802596930480058
:103B20007008788898680259692850007008788869
:103B30009868025969505000700878889868025A4D
:103B40006A30483000700878889868025666702895
:103B500070A0A8500058687088808088702040024B
:103B600059694020007088F88088700259691020D7
:103B7000007088F88088700259693048007088F8B1
:103B80008088700259695050007088F880887012DF
:103B90003969804000C040404040E012396920400F
:103BA00000C040404040E0124969609000C0404081
:103BB0004040E0123969A0A000C040404040E0020F
:103BC0005A6A502060107088888888700259692865
:103BD0005000B0C8888888880259694020007088E1
:103BE00088888870025969102000708888888870D9
:103BF000025969304800708888888870025969289D
:103C00005000708888888870025969505000708808
:103C100088888870035767202000F800202001580A
:103C200068087098A8A8C870800259694020008868
:103C30008888889868025969102000888888889840
:103C400068025969304800888888889868025969EC
:103C5000505000888888889868005B6B1020008826
:103C600088889868088870005A6A8080B0C88888F8
:103C7000C8B08080005B6B505000888888986808C6
:103C8000887000000000000000000000000000003C
:103C90000000000000000000000000000000000024
:103CA00000000000000C000000000000000C0000FC
:103CB00000000000001200000000000000230000CF
:103CC000000000000021000000000000004C800007
:103CD00000000000005E8000000000000092400034
:103CE0000000000000A140000000000001212000B1
:103CF00000000000027F90000000000002001000A1
:103D00000000000007FFF8000000000004000800A9
:103D10000000000008000400000000000800060089
:103D2000000000001000020000000000301E010032
:103D300000000000207F81000000000041FFE080C3
:103D40000000000043FCF08000000000873B78404A
:103D5000000000018EDBFC60000000010FEBCC20B6
:103D6000000000021FEDB610000000021FDEB610BA
:103D70000000000439CD7F080000000436E0FF0891
:103D8000000000087EC0BB84000000187F005D8634
:103D9000000000107FC0ED82000000203CC07301D5
:103DA000000000203B337F01000000701BE77E0312
:103DB000800000C81DEEDE04C00000880FDEDC04B9
:103DC000400001240FDF3C092000012607DBF81921
:103DD0002000027203E7F0139000025101FFE0227D
:103DE00090000489007F802448000904801E004858
:103DF00024000BFE400000DFF400100040000080B3
:103E000002001FFFFFFFFFFFFE0000000000000098
:103E100000000000000000000000000000000000A2
:103E200000001022103C3C0E1F0010221004221132
:103E300004001022100822110400102210083C1166
:103E40000400102210102211040010221020221150
:103E500004001E1C1E3C3C0E04000000000000007C
:103E60000000000000000000000000000000000052
:103E70000000000000000000000000000000000042
:103E80000000000000000000000000000000000032
:103E90000000000000000000000000000000000022
:103EA0000000000000000000000000000000000012
:103EB0000000000000000000000000000000000002
:103EC0000A003B20454550524F4D20496E646578AD
:103ED0003A20005570646174696E67207A6F666677
:103EE00073657420696E20454550524F4D3A20004D
:103EF0000600060006000600060006000600060092
:103F000006003FC01F800F00060006000F001F8044
:103F10003FC0060006000600060006000600060078
:103F20000600060007F8000C0C001002002001003B
:103F30006001804000804003E04001C040008040BC
:103F400000004000006000002000001000000C0C89
:103F50000007F80001FE0003030004008008004091
:103F60001800601000207C00203800201000200085
:103F700000200000200000600000400000800303DB
:103F80000001FE00FFFFFF7F80FFC0FFC0FFC07F7A
:103F9000807F80FFC0FFC0FFC03F001E000C005AA2
:103FA000204F6666736574004D6F76652058004D2E
:103FB0006F76652059004D6F7665205A00457874FC
:103FC0007275646572000200002100240027002A37
:103FD000002D003000330001010000040107010A38
:103FE000010102102020080810204010204080020B
:103FF000010201080402010102040810204080802F
:1040000040201008040201800402018040201008B2
:10401000040201080402010102040810204080018A
:10402000020408102040800505050507050808085A
:1040300008020202020A0A08080404040401010139
:104040000101010101030303030303030304070741
:10405000070C0C0C0C0C0C0C0C02020202060606DF
:1040600006060606060B0B0B0B0B0B0B0B1FFFFFBD
:10407000FFFFFFFF600000000001FF4000000000A4
:1040800000FF8000000000007F83CF00000C303F65
:1040900087FF80000C301F867980000C000F8C3069
:1040A000C7838C30E78C30CFC7CC31F38C30DCEC5D
:1040B000EC33B98C30D86C6C33198C30D06C0C3339
:1040C000198C30D86C0C33198C30DC6C0E3B198C8D
:1040D00030CF7C079F198C30C77C038F19400000BC
:1040E00000000002600000000000061FFFFFFFFF4D
:1040F000FFF82020506C616E6E65724275666665D1
:104100007242797465733A20002046726565204DCD
:10411000656D6F72793A2000436F6D70696C6564EC
:104120003A2044656320313520323031370A00208F
:104130007C20417574686F723A2028416C65706804
:10414000204F626A6563747320496E632E2C204C85
:10415000756C7A426F7420476974205265706F7372
:1041600069746F7279290A00446563203135203201
:1041700030313731353A32313A303700204C6173C3
:104180007420557064617465643A2000312E312EBC
:10419000350A004D61726C696E0020536F6674774A
:1041A0006172652052657365740A002057617463FB
:1041B00068646F672052657365740A002042726FED
:1041C000776E206F75742052657365740A00204500
:1041D000787465726E616C2052657365740A005064
:1041E0006F77657255700A0073746172740A0065A6
:1041F00072726F722077726974696E6720746F20B3
:1042000066696C650A004572726F723A00456E64A9
:1042100073746F7073202563202563202563202528
:10422000630020503A00205A3A0020593A002058A2
:104230003A00656E6473746F7073206869743A2015
:10424000006563686F3A00446F6E6520736176693C
:104250006E672066696C652E0A004D323900004D8C
:104260003234005072696E74207061757365640039
:104270004D313235004D363030204230004D323431
:10428000004D3233202573006175746F25692E67E8
:10429000004578747275646572004D6F7665205ABA
:1042A000004D6F76652059004D6F76652058004DA2
:1042B0006F76656D656E74004D6F76652061786907
:1042C000730044697361626C652073746570706516
:1042D0007273004D383400426564204C6576656C1D
:1042E000696E67004732382058590A4D31303920FD
:1042F000533137350A473238205A0A4D3130392088
:10430000523134350A4731320A4732390A4D313099
:1043100034205330004175746F20686F6D6500471D
:104320003238004D61696E00290A00206279746597
:10433000733B20637263200053657474696E677306
:104340002053746F72656420280020496E76616C7A
:1043500069642065787472756465722000205A3A29
:104360000020593A0020436F756E7420583A00209F
:10437000453A00205A3A0020593A00583A00205A4B
:1043800000205900580020204D61783A2000205A22
:1043900000205900580020204D696E3A20004F6ED1
:1043A00020004F666600536F667420656E647374F8
:1043B0006F70733A200053657474696E672054728D
:1043C0006176656C20416363656C65726174696FC9
:1043D0006E3A200053657474696E6720526574727A
:1043E00061637420416363656C65726174696F6EAB
:1043F0003A200053657474696E67205072696E7458
:1044000020416363656C65726174696F6E3A200068
:1044100053657474696E67205072696E7420616EA2
:10442000642054726176656C20416363656C6572CB
:104430006174696F6E3A200020643A0020693A0086
:1044400020703A0020643A0020693A0020703A0057
:104450004B494C4C45442E200024F4D43050C38E9C
:1044600020C2A24017828B7011127A910D816CD9F3
:104470000AA861E108C7586607615143061E4B5DF3
:1044800005C145A7041A411104093D98037139314A
:10449000034036DB0265339102D4305402802E1D76
:1044A00002632CEE01752AC501B028A001102781F6
:1044B000018F2564012B244B01E0223401AC211F24
:1044C000018D200D01801FFC00841EED00971DDF73
:1044D00000B81CD200E61BC600201BBC00641AB248
:1044E00000B219A8000A19A0006A189900D1179102
:1044F0000040178B00B516840031167E00B3157985
:10450000003A157300C7146F0058146A00EE136662
:10451000008813630025135E00C7125B006C1257FE
:104520000015125400C111510070114F0021114BA0
:1045300000D61049008D104700461044000210427A
:1045400000C00F4000800F3E00420F3C00060F3BB2
:1045500000CB0E3800930E37005C0E3500270E346A
:1045600000F30D3200C10D3100900D3000600D2EB2
:1045700000320D2D00050D2C00D90C2B00AE0C299E
:1045800000850C29005C0C2700350C27000E0C263A
:1045900000E80B2400C40B2400A00B23007D0B2398
:1045A000005A0B2100390B2100180B2000F80A1FBC
:1045B00000D90A1E00BB0A1E009D0A1D00800A1DAC
:1045C00000630A1C00470A1B002C0A1B00110A1A70
:1045D00000F7091A00DD091900C4091900AB09190F
:1045E00000920917007B091800630917004C09168F
:1045F0000036091600200916000A091500F50815ED
:1046000000E0081400CC081400B8081400A4081432
:1046100000900813007D0812006B08130058081260
:104620000046081200340811002308110012081176
:104630000001081100F0071000E0071000D007107B
:1046400000C0071000B0070F00A107100091070E6F
:104650000083070F0074070F0065070E0057070E51
:104660000049070E003B070D002E070E0020070D26
:104670000013070D0006070D00F9060C00ED060DEE
:1046800000E0060C00D4060C00C8060C00BC060CAA
:1046900000B0060C00A4060B0099060C008D060B5A
:1046A0000082060B0077060B006C060B0061060A01
:1046B0000057060B004C060A0042060A0038060A9C
:1046C000002E060A0024060A001A060A001006092F
:1046D0000007060A00FD050900F4050900EB0509BD
:1046E00000E2050900D9050900D0050900C7050940
:1046F00000BE050900B5050800AD050800A50509BF
:10470000009C050800940508008C05080084050835
:10471000007C050800740508006C050700650508A5
:10472000005D050700560508004E05070047050710
:10473000004005080038050700310507002A050775
:1047400000230507001C050600160507000F0507D6
:10475000000805060002050700FB040600F5040733
:1047600000EE040600E8040600E2040700DB04068D
:1047700000D5040600CF040600C9040600C30406E1
:1047800000BD040600B7040600B1040500AC040631
:1047900000A6040600A00405009B0406009504057D
:1047A00000900406008A04050085040500800406C4
:1047B000007A04050075040500700405006B04050B
:1047C0000066040500610405005C0405005704054B
:1047D00000520405004D040500480405004304058B
:1047E000003E0404003A04050035040500300404CA
:1047F000002C04050027040400230405001E040403
:10480000001A04040016040500110404000D040439
:1048100000090405000404040000040400FC03046F
:1048200000F8030400F4030400F0030400EC0304A4
:1048300000E8030400E4030400E0030400DC0304D4
:1048400000D8030400D4030400D0030400CC030404
:1048500000C8030300C503030024F404D9201BC4CB
:104860000C5C0E9804C4095F0265077101F405F938
:1048700000FB04B30048048700C1036900580355D6
:104880000003034500BE023A008402310053022AAD
:10489000002902250004022000E4011C00C80119BF
:1048A00000AF01170098011400840113007101107A
:1048B000006101100051010E0043010D0036010B93
:1048C000002B010B0020010B00150109000C010950
:1048D0000003010800FB000800F3000800EB0007DC
:1048E00000E4000600DE000600D8000600D2000644
:1048F00000CC000500C7000500C2000500BD000493
:1049000000B9000400B5000400B1000400AD0004CB
:1049100000A9000400A5000300A20003009F0004FA
:10492000009B000300980003009500020093000321
:1049300000900003008D0002008B0003008800023D
:10494000008600020084000300810002007F000254
:10495000007D0002007B0002007900020077000168
:104960000076000200740002007200010071000273
:10497000006F0002006D0001006C0002006A00017F
:104980000069000200670001006600010065000187
:10499000006400020062000100610001006000018B
:1049A000005F0002005D0001005C0001005B00018F
:1049B000005A000100590001005800010057000191
:1049C0000056000100550001005400010053000092
:1049D000005300010052000100510001005000018D
:1049E000004F0001004E0000004E0001004D00018C
:1049F000004C0001004B0000004B0001004A000188
:104A00000049000100480000004800010047000183
:104A1000004600000046000100450000004500017E
:104A20000044000100430000004300010042000078
:104A3000004200010041000000410001004000016F
:104A4000003F0000003F0001003E0000003E00016A
:104A5000003D0000003D0001003C0000003C000063
:104A6000003C0001003B0000003B0001003A000058
:104A7000003A000100390000003900010038000050
:104A80000038000000380001003700000037000146
:104A9000003600000036000000360001003500003E
:104AA0000035000000350001003400000034000033
:104AB0000034000100330000003300000033000127
:104AC000003200000032000000320001003100001E
:104AD0000031000000310001003000000030000013
:104AE00000300001002F0000002F0000002F000008
:104AF000002F0001002E0000002E0000002E0001FB
:104B0000002D0000002D0000002D0000002D0001F0
:104B1000002C0000002C0000002C0000002C0001E4
:104B2000002B0000002B0000002B0000002B0001D8
:104B3000002A0000002A0000002A0000002A0001CC
:104B400000290000002900000029000000290000C1
:104B500000290001002800000028000000280000B3
:104B600000280000002800010027000000270000A6
:104B70000027000000270000002700010026000099
:104B8000002600000026000000260000002600018C
:104B90000025000000250000002500000025000081
:104BA0000025000000250001002400000024000072
:104BB0000024000000240000002400010023000065
:104BC0000023000000230000002300000023000059
:104BD000002300000023000100220000002200004A
:104BE000002200000022000000220000002200013C
:104BF0000021000000210000002100000021000031
:104C00000021000000210000002100010020000020
:104C10000020000000200000002000000020000014
:104C2000002000000020000000200001001F000004
:104C3000001F0000001F0000001F0000001F0000F8
:104C4000001F0000001F0001001E0000001E0000E9
:104C5000001E0000001E0000004D3834205820596E
:104C6000205A2045004572723A204D494E54454D18
:104C70005020424544004D494E54454D50207472D9
:104C800069676765726564004572723A204D494EE6
:104C900054454D50204531004572723A204D494EE1
:104CA00054454D50204530004572723A204D4158D0
:104CB00054454D5020424544004D415854454D50B7
:104CC00020747269676765726564004572723A2084
:104CD0004D415854454D50204531004572723A209F
:104CE0004D415854454D502045300020746F6F2081
:104CF0006C6F6E6720657874727573696F6E207063
:104D0000726576656E7465640A0020636F6C64205A
:104D1000657874727573696F6E2070726576656EF2
:104D20007465640A00436172642072656D6F766514
:104D300064004361726420696E7365727465640017
:104D40004D36303020486F74656E6420746F6F206C
:104D5000636F6C6420746F206368616E67652066A2
:104D6000696C616D656E740A004B64200023646594
:104D700066696E65202044454641554C545F004BA2
:104D800069200023646566696E65202044454641BC
:104D9000554C545F004B70200023646566696E6556
:104DA000202044454641554C545F00504944204121
:104DB00075746F74756E652066696E697368656475
:104DC000212050757420746865206C617374204BC9
:104DD000702C204B6920616E64204B6420636F6EE1
:104DE0007374616E74732066726F6D2062656C6F90
:104DF0007720696E746F20436F6E666967757261A4
:104E000074696F6E2E680A00504944204175746FB2
:104E100074756E65206661696C6564212074696DC6
:104E2000656F75740A00504944204175746F74753C
:104E30006E65206661696C6564212054656D7065DE
:104E400072617475726520746F6F20686967680A93
:104E500000204B643A2000204B693A2000204B7020
:104E60003A20000A20436C617373696320504944FF
:104E7000200A002054753A2000204B753A2000206B
:104E80006D61783A2000206D696E3A200020643A06
:104E9000200020626961733A2000526573746F725A
:104EA00065206661696C73616665004D3530320A54
:104EB0004D353030004C6F61642073657474696ED9
:104EC00067730053746F72652073657474696E67DD
:104ED0007300416476616E63656420536574746920
:104EE0006E6773004D61696E005072696E74206167
:104EF000626F727465640041626F757420466972F6
:104F00006D77617265004E6F205344206361726457
:104F1000005072696E742066726F6D2053440053A6
:104F2000746F70207072696E7400526573756D6570
:104F3000207072696E7400506175736520707269BB
:104F40006E74004368616E67652066696C616D65AB
:104F50006E7400436F6E66696775726174696F6E17
:104F60000054656D7065726174757265004D6F7681
:104F7000656D656E740054756E6500496E666F20D0
:104F800073637265656E00202F002042403A002056
:104F9000403A004E6F204C696E65204E756D62651B
:104FA00072207769746820636865636B73756D2C14
:104FB000204C617374204C696E653A200053544F45
:104FC000505045442E20005072696E7465722073F3
:104FD000746F707065642064756520746F206572ED
:104FE000726F72732E20466978207468652065722E
:104FF000726F7220616E6420757365204D39393986
:1050000020746F20726573746172742E2028546549
:105010006D70657261747572652069732072657355
:1050200065742E20536574206974206166746572FE
:105030002072657374617274696E67290A004E6F1D
:1050400020436865636B73756D2077697468206CA5
:10505000696E65206E756D6265722C204C6173748B
:10506000204C696E653A2000636865636B73756DEB
:10507000206D69736D617463682C204C61737420BA
:105080004C696E653A20004C696E65204E756D6204
:105090006572206973206E6F74204C617374204CAC
:1050A000696E65204E756D6265722B312C204C61E6
:1050B0007374204C696E653A20004D313130004DDB
:1050C0003331004D383420582059205A20450053A0
:1050D000442072656164206572726F720A00446FC9
:1050E0006E65207072696E74696E672066696C65A2
:1050F0000A004B494C4C45442E20004B494C4C2057
:10510000636175736564206279204B494C4C206261
:105110007574746F6E2F70696E0A004B494C4C4564
:10512000442E20004B494C4C20636175736564200C
:10513000627920746F6F206D75636820696E61639A
:10514000746976652074696D65202D2063757272AF
:10515000656E7420636F6D6D616E643A20004C75EE
:105160006C7A426F742054415A2036204F66662E66
:10517000004F6666004F6E2000456E6473746F705A
:105180002061626F72740053746570732F6D6D00CF
:105190004A65726B00416363656C65726174696F27
:1051A0006E0056656C6F63697479005A204F6666AD
:1051B00073657400416476616E6365642053657441
:1051C00074696E6773005654726176206D696E0063
:1051D0005654726176206D696E0056547261762065
:1051E0006D696E00566D696E00566D696E00566D84
:1051F000696E00566D6178204500566D61782045D6
:1052000000566D6178204500566D6178205A005631
:105210006D6178205A00566D6178205A00566D6194
:1052200078205900566D6178205900566D617820BC
:105230005900566D6178205800566D6178205800ED
:10524000566D61782058004D6F74696F6E0045731C
:10525000746570732F6D6D004573746570732F6D79
:105260006D005A73746570732F6D6D005A73746599
:1052700070732F6D6D005973746570732F6D6D00B1
:105280005973746570732F6D6D0058737465707306
:105290002F6D6D005873746570732F6D6D004D6FB9
:1052A00074696F6E0056652D6A65726B0056652DC8
:1052B0006A65726B0056652D6A65726B00567A2DB1
:1052C0006A65726B00567A2D6A65726B0056792D8D
:1052D0006A65726B0056792D6A65726B0056792D7E
:1052E0006A65726B0056782D6A65726B0056782D70
:1052F0006A65726B0056782D6A65726B004D6F742B
:10530000696F6E004F666673657473206170706CB0
:10531000696564004572723A20546F6F206661724D
:105320002100546F6F206661722066726F6D20726B
:1053300065666572656E636520706F696E740A00DC
:1053400048617264636F6465642044656661756C6E
:10535000742053657474696E6773204C6F61646563
:10536000640A0028230000282300006400000010C5
:1053700027000000009643000096430000404000D4
:1053800000C8410000C9420000C9420000C84400F2
:10539000804F44202863616C63756C617465642977
:1053A000210A0020213D2000454550524F4D204309
:1053B0005243206D69736D61746368202D202873DA
:1053C000746F726564292000290A0020627974656F
:1053D000733B2063726320002073746F72656420D6
:1053E00073657474696E677320726574726965762B
:1053F0006564202800204D61726C696E3D56343022
:10540000290A0028454550524F4D3D004545505210
:105410004F4D2076657273696F6E206D69736D6193
:105420007463682000000020002300260029002C5F
:10543000002F0032000001000003010601090100F5
:1054400000A0C10000A0C1000000000000964300C1
:10545000809743000087435A204F66667365740047
:10546000466C6F7700466C6F770046616E207370F4
:1054700065656420310046616E2073706565642047
:10548000310042656400426564004E6F7A7A6C6553
:10549000004E6F7A7A6C65005370656564005370D6
:1054A000656564004D61696E00416D61782045005D
:1054B000416D6178204500416D6178205A00416D51
:1054C0006178205A00416D6178205900416D617802
:1054D000205900416D6178205800416D6178205855
:1054E00000412D74726176656C00412D7472617695
:1054F000656C00412D7265747261637400412D7298
:1055000065747261637400416363656C0041636339
:10551000656C004D6F74696F6E000000A0C1008063
:105520009743000000005761726E696E673A204829
:105530006F6D696E672042756D702044697669737E
:105540006F72203C20310A000202040000A04000DB
:1055500000A040000000400000A0430080A14300E4
:1055600000874300004842000048420000404000DD
:10557000000000FF01FF5A2070726F6265206F7596
:10558000742E206265640A005A2070726F62652072
:105590006F75742E2062656400486F6D65205859E0
:1055A0002066697273740A00486F6D65205859202F
:1055B000666972737400436F6F6C646F776E004638
:1055C000616E20737065656420310046616E2073E2
:1055D0007065656420310042656400426564004E78
:1055E0006F7A7A6C65004E6F7A7A6C65004D6169EE
:1055F0006E004E414E494E495459494E46CDCCCC91
:105600003D0AD7233C17B7D13877CC2B329595E696
:10561000241FB14F0A000020410000C84200401C76
:105620004620BCBE4CCA1B0E5AAEC59D7400DA00A3
:10563000F3CE11241FBECFEFD1E2DEBFCDBF00E01D
:105640000CBF14E0A0E0B2E0E6E1F3E402E00BBF3F
:1056500002C007900D92AC31B107D9F725E1ACE15A
:10566000B4E001C01D92A931B207E1F716E5C0E32D
:10567000D6E500E006C022970109FE010BBF0F949A
:105680000B21CE32D10780E00807A9F70E9439B07C
:105690000D947A210C9400002F923F924F925F92CA
:1056A0006F927F928F929F92AF92BF92CF92DF9232
:1056B000EF92FF920F931F93CF93DF93CDB7DEB797
:1056C000C958D1090FB6F894DEBF0FBECDBF009107
:1056D000320920E6029F800111240E54184F809158
:1056E000840680FF1AC0E1E4F2E484917F013FEF79
:1056F000E31AF30A811102C0780104C00E944359E1
:10570000F701F3CFD7018D917D01882319F00E9415
:105710004359F8CF8AE00E94435910926E061092C6
:105720006D068FE3809383061092820610928106A5
:1057300010923604109237041092380410923904F3
:10574000F80180810F5F1F4F8032D1F38E34B1F4A6
:10575000818190ED980F9A3020F08D3211F08B32CC
:1057600069F43296DF0131962C9120532A30D0F320
:10577000CD01FC01019620812032D9F3F0937B0604
:10578000E0937A067F01BFEFEB1AFB0A10816AE211
:1057900070E0C7010F944B21009739F0DC0111979D
:1057A0008C918032E1F311961C921D3429F014354E
:1057B00019F0173409F0CAC0F7014E2F9F2F8191BD
:1057C0008032D9F380538A3008F0C0C0109383062A
:1057D0002091810630918206E42FF92F6AE0AF0113
:1057E0004F5F5F4F629FC001639F900D1124208126
:1057F00030E020533109820F931F218120532A303A
:1058000030F090938206809381069A0103C09C0138
:10581000FA01E5CFD9012F5F3F4F4C914032D1F3D0
:105820001D34D1F48E31910591F03CF4873191050E
:1058300071F08C31910581F40AC08537910564F0CF
:105840008737910524F0803AE3E09E0729F4B0936E
:105850006E06A0936D067AC010926E0610926D06C9
:10586000D0907A0641E050E0FD0131962C91222340
:1058700009F46CC02132A1F41D3491F480329105F9
:1058800079F4F0936E06E0936D0663E270E0CF0169
:105890000F944B21009709F459C0DC011C9256C0AB
:1058A0000FEB020F0A31A0F59F01F90160812F5F14
:1058B0003F4F6032D1F320ED260F2A3040F023ED28
:1058C000260F223020F06B3211F00C9457419F01CB
:1058D000602F70E0DB01B595A795B595A795B595B7
:1058E000A795AA5CBB4F07707A01002E01C0EE0C91
:1058F0000A94EAF7FC90FE28FC922115310511F07C
:105900002D1901C020E0DB01A45EBB4F2C930AC01F
:1059100020916D0630916E06232B21F4B0936E0614
:10592000A0936D06208121542A3110F4DF019CCF11
:10593000DF0131966C9160536A30D0F39D01F9011B
:105940002F5F3F4F60816032D1F3F0CF80918306AB
:105950008D3411F40C948935843511F40C94FA408B
:10596000873411F00C943A4180918106909182061F
:105970008A31910509F47CC7A4F48430910544F47C
:10598000823091050CF01FC197FF2BC00C9454413D
:105990008430910509F4E5C60C9709F427C70C94E7
:1059A00054418E31910511F40C94D7343CF48C3170
:1059B000910509F4E6C70CF462C7E8C78B35910579
:1059C00011F40C9480358C35910511F40C948535C7
:1059D0008A35910511F00C945441109280060C9474
:1059E000544180915702882311F40C9454410F9430
:1059F00028088BE394E00F94C9060F94270A80913E
:105A0000840683FD8FC0C0904704D0904804E09086
:105A10004904F0904A0420918C0730918D07409101
:105A20008E0750918F07C701B6010F94E3198823A1
:105A300009F478C080913A04811138C060910A025B
:105A400070910B02882777FD8095982F0F94E919A4
:105A50009B01AC01609164067091650680916606B9
:105A6000909167060F94E31987FF20C0C0928C07BE
:105A7000D0928D07E0928E07F0928F07E1E4F2E476
:105A800084918F010F5F1F4F882321F00E9443599B
:105A9000F801F6CFEDE5F2E084918F010F5F1F4F23
:105AA000882321F00E944359F801F6CFC0904704A3
:105AB000D0904804E0904904F0904A0420918C076B
:105AC00030918D0740918E0750918F07C701B60125
:105AD0000F94151E20E030E048E453E40F943C207E
:105AE000181604F5C0928C07D0928D07E0928E07AD
:105AF000F0928F07E1E4F2E484918F010F5F1F4F72
:105B0000882321F00E944359F801F6CFEEE3F2E03A
:105B100084918F010F5F1F4F882321F00E9443590A
:105B2000F801F6CF20913B0430913C0440913D04B4
:105B300050913E04609180077091810780918207A7
:105B4000909183070F94E31981111DC020913F04A8
:105B50003091400440914104509142046091840787
:105B60007091850780918607909187070F94E319BC
:105B7000811109C060910C0270910D0280910E029A
:105B800090910F021AC06091A6027091A702882717
:105B900077FD8095982F0F94E91920910C02309190
:105BA0000D0240910E0250910F020F94481A2AE004
:105BB00037ED43E25CE30F94481A0E94FBDE0F943A
:105BC00028070C94544120915702222311F40C947D
:105BD000544111E0029709F010E00F94280882E583
:105BE0000F941208882309F45CC10F9443066B01DB
:105BF0007C014090800750908107609082077090F0
:105C00008307209184073091850740918607509142
:105C1000870763962CAF3DAF4EAF5FAF6397809120
:105C20003B0490913C04A0913D04B0913E046796E2
:105C30008CAF9DAFAEAFBFAF679720913F0430915F
:105C4000400440914104509142046F962CAF3DAF07
:105C50004EAF5FAF6F9720E030E0A901C701B601FA
:105C60000F94E319882309F462C5A3019201679692
:105C70006CAD7DAD8EAD9FAD67970F94E31981112B
:105C800011C063962CAD3DAD4EAD5FAD63976F9681
:105C90006CAD7DAD8EAD9FAD6F970F94E3198823EA
:105CA00009F445C520E030E0A901C701B6010F9411
:105CB000E319881F8827881F181759F080E090E0A3
:105CC000A0E8BFEBAB968CAF9DAFAEAFBFAFAB97CD
:105CD0000AC020E030E040E85FE3AB962CAF3DAF78
:105CE0004EAF5FAFAB97A301920167966CAD7DADF0
:105CF0008EAD9FAD67970F94151EA3966CAF7DAFC9
:105D00008EAF9FAFA39763962CAD3DAD4EAD5FAD0B
:105D100063976F966CAD7DAD8EAD9FAD6F970F9411
:105D2000151EA7966CAF7DAF8EAF9FAFA797A396BA
:105D30002CAD3DAD4EAD5FADA397CA01B9010F9437
:105D4000481A4B015C01A7962CAD3DAD4EAD5FAD41
:105D5000A797CA01B9010F94481A9B01AC01C5016C
:105D6000B4010F94161E0F9481206B966CAF7DAF1B
:105D70008EAF9FAF6B9720E030E040E05FE30F9481
:105D8000481A4B015C01A7019601C701B6010F94A7
:105D9000481A6B017C01A5019401C501B4010F945F
:105DA000481A9B01AC01C701B6010F94151E0F9450
:105DB00081209B01AC01AB966CAD7DAD8EAD9FADEE
:105DC000AB970F94481A4B015C0167962CAD3DAD23
:105DD0004EAD5FAD6797C301B2010F94161E20E070
:105DE00030E040E05FE30F94481A6B017C01A79616
:105DF0006CAD7DAD8EAD9FADA79790586B962CADD9
:105E00003DAD4EAD5FAD6B970F94F21E9B01AC01A3
:105E1000C501B4010F94481A9B01AC01C701B6013A
:105E20000F94161EA30192010F94151E6B017C01A5
:105E30006F962CAD3DAD4EAD5FAD6F9763966CAD7B
:105E40007DAD8EAD9FAD63970F94161E20E030E0C0
:105E500040E05FE30F94481A2B013C016B962CAD98
:105E60003DAD4EAD5FAD6B97A3966CAD7DAD8EAD88
:105E70009FADA3970F94F21E9B01AC01C501B40125
:105E80000F94481A9B01AC01C301B2010F94161E76
:105E900063962CAD3DAD4EAD5FAD63970F94151E6F
:105EA00014C089E40F941208882329F00F94430644
:105EB0006B017C0103C0C12CD12C76018AE40F94C4
:105EC00012088823F9F00F9443066F966CAF7DAFEC
:105ED0008EAF9FAF6F9720E030E0A901C701B601F8
:105EE0000F94E31981111EC020E030E0A9016F96E4
:105EF0006CAD7DAD8EAD9FAD6F970F94E3198111A1
:105F000011C015C420E030E0A901C701B6010F940B
:105F1000E319882309F40BC46F961CAE1DAE1EAEA8
:105F20001FAE6F97D701C601B05863968CAF9DAF77
:105F3000AEAFBFAF63976F962CAD3DAD4EAD5FADCD
:105F40006F97505867962CAF3DAF4EAF5FAF6797D6
:105F50009C01AD01BC01CD010F94481A4B015C01BD
:105F600067962CAD3DAD4EAD5FAD6797CA01B901E7
:105F70000F94481A9B01AC01C501B4010F94161E81
:105F80000F948120EB966CAF7DAF8EAF9FAFEB97F8
:105F90008091800790918107A0918207B09183073B
:105FA000A3968CAF9DAFAEAFBFAFA397A7019601ED
:105FB000BC01CD010F94161EAB966CAF7DAF8EAFBA
:105FC0009FAFAB972091840730918507409186075A
:105FD00050918707A7962CAF3DAF4EAF5FAFA79705
:105FE0006F962CAD3DAD4EAD5FAD6F97A7966CAD86
:105FF0007DAD8EAD9FADA7970F94161EAF966CAF7B
:106000007DAF8EAF9FAFAF9780913B0490913C04E2
:10601000A0913D04B0913E04E3968CAF9DAFAEAF2E
:10602000BFAFE397AB962CAD3DAD4EAD5FADAB973B
:10603000BC01CD010F94151E6B017C0120913F0422
:10604000309140044091410450914204E7962CAFB6
:106050003DAF4EAF5FAFE797AF962CAD3DAD4EADC8
:106060005FADAF97E7966CAD7DAD8EAD9FADE79719
:106070000F94151E4B015C01809188079091890750
:10608000A0918A07B0918B07C158DF4F888399830D
:10609000AA83BB83CF57D0409C01AD0160914304DC
:1060A0007091440480914504909146040F94151E0C
:1060B0006B966CAF7DAF8EAF9FAF6B9720918C07C7
:1060C00030918D0740918E0750918F07CD57DF4F4C
:1060D000288339834A835B83C358D0406091470447
:1060E000709148048091490490914A040F94151EC0
:1060F000EF966CAF7DAF8EAF9FAFEF97A701960184
:1061000063966CAD7DAD8EAD9FAD63970F94481ACD
:106110002B013C01A501940167966CAD7DAD8EAD60
:106120009FAD67970F94481A9B01AC01C301B20160
:106130000F94161E2B013C01A501940163966CADD2
:106140007DAD8EAD9FAD63970F94481A4B015C01F6
:10615000A701960167966CAD7DAD8EAD9FAD67973B
:106160000F94481A9B01AC01C501B4010F94151E90
:10617000A30192010F94891E6B017C0120E030E0A5
:10618000A9010F94E31987FF0AC02BED3FE049EC0A
:1061900050E4C701B6010F94161E6B017C01112358
:1061A00051F02BED3FE049EC50E4C701B6010F94EC
:1061B000151E6B017C0120E030E0A901C701B6018A
:1061C0000F94E319811128C0E3962CAD3DAD4EAD7F
:1061D0005FADE397A3966CAD7DAD8EAD9FADA397FC
:1061E0000F94E319811118C0E7962CAD3DAD4EAD6B
:1061F0005FADE797A7966CAD7DAD8EAD9FADA797D0
:106200000F94E319811108C08BEDC82E8FE0D82EB2
:1062100089ECE82E80E4F82EEB962CAD3DAD4EAD2A
:106220005FADEB97C701B6010F94481A9B01AC0113
:106230000F94481A4B015C016B962CAD3DAD4EADF1
:106240005FAD6B97CA01B9010F94481A9B01AC016D
:10625000C501B4010F94161E0F9481204B015C01FF
:106260002FE632E143E85AE30F94E31987FD5BC25E
:10627000C501B4010F948B1F0F945F1F1B016115A3
:10628000710519F422242394312CB10180E090E0AF
:106290000F94E7194B015C019B01AC01C701B601EA
:1062A0000F94F21EA3966CAF7DAF8EAF9FAFA397F6
:1062B000A50194016B966CAD7DAD8EAD9FAD6B97D6
:1062C0000F94F21EEB966CAF7DAF8EAF9FAFEB9746
:1062D000A5019401EF966CAD7DAD8EAD9FADEF97AE
:1062E0000F94F21EEF966CAF7DAF8EAF9FAFEF971E
:1062F000A3962CAD3DAD4EAD5FADA397CA01B901DC
:106300000F94481A20E030E040E05FE30F94481A11
:106310009B01AC0160E070E080E89FE30F94151EE4
:10632000E3966CAF7DAF8EAF9FAFE397C158DF4F61
:1063300088819981AA81BB81CF57D04089879A876C
:10634000AB87BC87CD57DF4F288139814A815B817C
:10635000C358D0402D873E874F87588B6091A60247
:106360007091A702882777FD8095982F0F94E919DF
:1063700020910C0230910D0240910E0250910F02BB
:106380000F94481A2AE037ED43E25CE30F94481A71
:10639000E7966CAF7DAF8EAF9FAFE7970F941B0A68
:1063A000DC01CB0188539F4FAF4FBF4F6B968CAF33
:1063B0009DAFAEAFBFAF6B9760964FAC60976196E5
:1063C0005FAC619762966FAC629763967FAC6397A0
:1063D000A1E0B0E0A596BFAFAEAFA59719E1B12E91
:1063E000A5962EAD3FADA5972215330508F057C1F0
:1063F0000E942C6C0F941B0A6B962CAD3DAD4EADDC
:106400005FAD6B97621B730B840B950B97FD11C0EF
:106410000F941B0ADC01CB0188539F4FAF4FBF4F36
:106420006B968CAF9DAFAEAFBFAF6B9780E00E9415
:1064300054F1BA9409F44FC0E3962CAD3DAD4EAD86
:106440005FADE39767966CAD7DAD8EAD9FAD679701
:106450000F94481A6B017C01A3962CAD3DAD4EAD57
:106460005FADA397B201C3010F94481AA70196012B
:106470000F94161E162FA72E982E892EE3962CAD5C
:106480003DAD4EAD5FADE397B201C3010F94481A25
:106490006B017C01A3962CAD3DAD4EAD5FADA397D6
:1064A00067966CAD7DAD8EAD9FAD67970F94481A22
:1064B0009B01AC01C701B6010F94151E2B013C01D5
:1064C000812F9A2DA92DB82D67968CAF9DAFAEAFB9
:1064D000BFAF67975FC0A596AEADBFADA597BD0135
:1064E00080E090E00F94E719A3962CAD3DAD4EAD42
:1064F0005FADA3970F94481A4B015C010F94EF1EF8
:106500006B017C01C501B4010F9477204B015C0144
:10651000A701960163966CAD7DAD8EAD9FAD63977F
:106520000F94481A2B013C01A50194016F966CADA4
:106530007DAD8EAD9FAD6F970F94481A9B01AC0156
:10654000C301B2010F94161E2B013C01A501940159
:1065500063966CAD7DAD8EAD9FAD63970F94481A79
:106560004B015C01A70196016F966CAD7DAD8EADC0
:106570009FAD6F970F94481A9B01AC01C501B40100
:106580000F94151E67966CAF7DAF8EAF9FAF679768
:10659000B9E1BB2E9201A301AB966CAD7DAD8EAD82
:1065A0009FADAB970F94161E69837A838B839C8370
:1065B00067962CAD3DAD4EAD5FAD6797AF966CADB8
:1065C0007DAD8EAD9FADAF970F94161E6D837E830C
:1065D0008F839887EB962CAD3DAD4EAD5FADEB97BD
:1065E00069857A858B859C850F94161E69877A87C5
:1065F0008B879C87EF962CAD3DAD4EAD5FADEF9791
:106600006D857E858F8598890F94161E6D877E8790
:106610008F87988BCE0101960F94C906C09079069A
:1066200089819A81AB81BC8188A399A3AAA3BBA3CA
:106630008D819E81AF81B8858CA39DA3AEA3BFA39E
:1066400089859A85AB85BC8588A799A7AAA7BBA78A
:10665000AE01485D5F4FBE016C5D7F4FCE018096FD
:106660000E94D4A2E796ECACFDAC0EAD1FADE7974F
:106670009E01235F3F4FAE01485D5F4FBE016C5DE1
:106680007F4FCE0180960E943DCFA596EEADFFAD27
:10669000A5973196A596FFAFEEAFA597A1CEC09076
:1066A000790680913B0490913C04A0913D04B09107
:1066B0003E0488A399A3AAA3BBA380913F04909111
:1066C0004004A0914104B09142048CA39DA3AEA3C9
:1066D000BFA38091430490914404A0914504B091DC
:1066E000460488A799A7AAA7BBA7AE01485D5F4F3C
:1066F000BE016C5D7F4FCE0180960E94D4A2E796CA
:10670000ECACFDAC0EAD1FADE79727E434E0AE0175
:10671000485D5F4FBE016C5D7F4FCE0180960E9449
:106720003DCF0F9428070F94270A0C945441E6E0BC
:10673000F2E484918F010F5F1F4F882321F00E94A4
:106740004359F801F6CFE8E7F2E084918F010F5F3B
:106750001F4F882311F40C9454410E944359F801AF
:10676000F4CF80E50F941208882329F00E94A45AE0
:106770004B015C0103C0812C912C540183E50F94E3
:106780001208882361F00F94430620E030E04AE7C6
:1067900054E40F94481A0F945F1F4B015C010E9450
:1067A0007DFB80911002811105C060E08EE892E0CF
:1067B0000E942BA40F94270AC0905704D09058042D
:1067C000E0905904F0905A04C80CD91CEA1CFB1C38
:1067D0000F941B0A6C197D098E099F0997FD02C051
:1067E0000C94544180E00E9454F1F2CF0E94B076A4
:1067F00081110C94544180E50F941208882319F0FC
:106800000F94330601C060E06FAF83E50F94120868
:10681000882319F00F94330601C06CE06BAF84E558
:106820000F941208882319F00F94330601C063E017
:1068300068A382E50F941208882319F00F94430689
:1068400004C060E070E080ED90E469837A838B831C
:106850009C839E01205E3F4FAE014F5F5F4FBE01A4
:10686000655C7F4FCE01CF960E94A7E80C945441FF
:1068700081E080935702109278060C9454410E9454
:10688000B07681110C94544180E50F94120888234E
:1068900021F00F943306462F01C040E06091880735
:1068A0007091890780918A0790918B0700E010E032
:1068B00020E231EC09831A832B833C8300E010E84B
:1068C00022E933E40D831E832F83388700E010E034
:1068D00020EA31E409871A872B873C8700E010E023
:1068E00020EC3FE70D871E872F87388B413071F1F1
:1068F000423021F518A219A21AA21BA220E030E012
:1069000040EA51E40F94161E7B018C0120E030E038
:1069100047E853E40F943C20181624F4E12CF12CA2
:1069200007E813E4A701B8014BAF5CAF6DAF7EAFD2
:10693000BE01605E7F4FCE01CB9611C020E030E0FB
:1069400040EA51E40F94E31987FF0BC018A219A283
:106950001AA21BA2BE01605E7F4FCE0109960E9463
:10696000A0E818A219A21AA21BA2AE01405E5F4FB6
:10697000BE016B5F7F4FCE0101960E949CE80C9494
:10698000544180E00F9400110C94544181E08093B5
:10699000730724982C9A0898109A0E948F7C109262
:1069A0007307249A2C98089A10980C94544120E06C
:1069B00030E0A90160918007709181078091820782
:1069C000909183070F94161E182F88E5C957DF4F43
:1069D0006883C758D040C857DF4F7883C858D04025
:1069E000C757DF4F9883C958D0400F941208C95732
:1069F000DF4F6881C758D040C857DF4F7881C858EB
:106A0000D040C757DF4F9881C958D040882321F024
:106A10000F9443069B0102C09B01812FA901BC0179
:106A200048A359A36AA37BA320E030E0A9016091A9
:106A300084077091850780918607909187070F944E
:106A4000161E5B018C0189E50F941208882321F042
:106A50000F9443065B018C01A501B80149835A8359
:106A60006B837C8340904F0450905004609051049D
:106A70007090520420914B0430914C0440914D048D
:106A800050914E0468A179A18AA19BA10F94151E73
:106A90006B017C012CE032E040EA51EC0F943C2089
:106AA00087FF02C00C94544121E230E046E953E4F0
:106AB000C701B6010F94E319181614F40C9454414D
:106AC000A3019201B501C8010F94151E6B017C0151
:106AD0002CE032E040EA51EC0F943C2087FF02C0EA
:106AE0000C94544121E230E847E953E4C701B60170
:106AF0000F94E319181614F40C9454410C94684143
:106B000081E0809380060C9454410E9499EB0C9490
:106B1000544180918106909182068937910511F444
:106B20000C947F3E0CF0D5C08D34910509F4A1C5BD
:106B30000CF053C08931910509F4E1C21CF5843190
:106B4000910509F45AC27CF48131910509F44AC2D5
:106B50002CF4029708F4C3C10C945441429709F4F1
:106B600074C70C9454418631910509F48DC20CF41C
:106B700087C28731910509F48DC2489709F4A0C2F4
:106B80000C9454418F31910509F47EC47CF48B310F
:106B9000910509F4D0C20CF4C0C28C31910509F4FE
:106BA00006C34E9709F407C30C9454418A329105E9
:106BB00009F40AC52CF4809709F41EC40C945441BE
:106BC0008B34910509F452C58C34910511F00C9465
:106BD00054410E9407780C9454418B36910509F476
:106BE000A2C6ACF58535910509F460C7C4F48235B9
:106BF000910509F423C74CF48135910511F00C94EB
:106C000054410E9465FB0C9454418335910509F46D
:106C100018C78435910509F418C70C945441883677
:106C2000910509F429C54CF48C35910511F00C94AB
:106C300054410F940E030C9454418936910509F484
:106C4000E4C58A36910509F44BC60C945441833748
:106C5000910509F42EC7D4F48E36910509F458C570
:106C600034F48D36910509F411C60C9454418F36D5
:106C7000910509F45EC58237910511F00C945441D9
:106C80000E947DFB0E9492BF0C945441863791056F
:106C900009F412C774F48537910511F00C9454412E
:106CA00060E080916D0690916E060E941BA40C948A
:106CB00054418737910509F436C78837910511F09B
:106CC0000C94544181E080937207809371070C9477
:106CD0005441803331E0930711F40C94063F0CF0DB
:106CE00078C08D3C910511F40C948D3EACF58E3B33
:106CF000910509F4E3C5ACF48C38910509F482C51B
:106D000034F48D37910509F424C60C94544181392B
:106D1000910509F4F9C78B39910509F490C50C94D4
:106D20005441893C910509F4F2C74CF4883C910523
:106D300011F00C9454410E94FEC00C9454418B3CC1
:106D4000910509F4E7C78C3C910511F00C9454416E
:106D50000E949DBE0C945441823E910509F4E6C701
:106D6000DCF4833D910509F4DBC74CF48E3C9105BE
:106D700011F00C9454410F9403050C9454418C3D34
:106D8000910509F4D0C78D3D910511F00C94544143
:106D90000E944BC10C9454418D3251E0950711F47F
:106DA0000C94033F3CF48C32914011F40C94DA3E85
:106DB0000C9454418E32E1E09E0711F40C94093F8B
:106DC0008F32914011F00C9454410E9460DF0C947A
:106DD0005441853F21E0920711F40C94683F0CF078
:106DE00045C0813941E0940711F40C940C3FFCF448
:106DF0008F35A1E09A0711F40C947D404CF48E3548
:106E0000914011F00C9454410E940F4F0C94544146
:106E10008336F1E09F0711F40C94CF408039914004
:106E200011F00C9454410E947DFB0C945441843A1F
:106E300031E0930709F4F4C754F48239914011F01A
:106E40000C94544180E00E940AEB0C9454418C3A1B
:106E5000A1E09A0711F40C94653F843F914011F032
:106E60000C9454410E9483C10C9454418335E3E057
:106E70009E0711F40C94743FB4F4873F21E092070D
:106E800011F40C946E3F14F40C946B3F8C3142E07F
:106E9000940711F40C94713F8835924011F40C94CE
:106EA000773F0C9454418C38A3E09A0711F40C946A
:106EB0007A404CF48B38934011F00C9454410E946A
:106EC000305F0C945441803AF3E09F0709F4D0C23C
:106ED000873E934011F40C94E8400C945441009187
:106EE0006D0610916E0680E50F941208882369F0F4
:106EF0000E94A45A6B017C01BB24B39461157105F7
:106F00008105910531F4B12C04C0B12CC12CD12CD8
:106F1000760183E50F9412088823F9F00F94430655
:106F200020E030E04AE754E40F94481A0F945F1FC2
:106F30006B017C01B11013C06115710581059105CC
:106F400071F40115110559F0D8018C91882339F09D
:106F500061E0C8010E941BA407C0BB2091F360E060
:106F60008DEC92E00E942BA481E08093370A0E946E
:106F70007DFB0F94270AC114D104E104F104D1F080
:106F80008090570490905804A0905904B0905A04EF
:106F90008C0C9D1CAE1CBF1C0F941B0A6819790930
:106FA0008A099B0997FF1AC08091370A81110C94B6
:106FB000BE4114C08091370A882321F080E00E94EE
:106FC00054F1F8CF8091621260E0882319F08EEBC3
:106FD00092E002C089EA92E00E942BA41092370A44
:106FE0000C94544160E080EE92E00E942BA417982C
:106FF0001698159814980C945441E8EFF2E0849197
:107000008F010F5F1F4F882321F00E944359F80121
:10701000F6CF10920E1540E050E0BA018AEB92E1F3
:107020000E945F748BE1EAEBF2E1DE0115960190BC
:107030000D928A95E1F78091B8129091B9129C83D4
:107040008B8380E293E09A83898340E050E0BE0125
:107050006F5F7F4F80EC93E00E9428AECE010196D7
:107060000E948791E9EEF2E084918F010F5F1F4F3C
:10707000882311F40C9454410E944359F801F4CF31
:107080000E943A900C945441109262121092631232
:107090000C945441E0916D06F0916E068081882336
:1070A00029F0803209F410823196F8CF40E061E097
:1070B00080916D0690916E060E944A680C9454412E
:1070C00019821A821B821C8218A219A21AA21BA260
:1070D00080917706882341F040E0BE016F5F7F4FCB
:1070E000CE0180960E9414E480916312882319F0E7
:1070F00081E0809362120E9490770C945441109228
:1071000062120E94077889E093E09093BC0A809312
:10711000BB0A0E9455BA0C94544180916312882393
:1071200011F40C94544183E50F94120881110C94CE
:10713000C3410C94544180916312882351F1EEE0D5
:10714000F3E084918F010F5F1F4F882321F00E948D
:107150004359F801F6CF609105157091061580919D
:107160000715909108154AE00E94934C8FE20E9407
:10717000435960910115709102158091031590910A
:1071800004154AE00E94934C8AE00E9443590C94F3
:107190005441E0E2F3E084918F010F5F1F4F882399
:1071A00011F40C9454410E944359F801F4CF0E9409
:1071B00045BD0C94544180916312882311F40C94C2
:1071C000544184E594E10E94258C84E594E10E9479
:1071D00028901092611210926012E0906D06F0906B
:1071E0006E0680916312882311F40C9454410E941E
:1071F00030901D8218861C821B8280E293E09A8365
:10720000898386EB92E19093D6128093D512F70191
:1072100080818F3209F06AC06FE270E0C7010F947D
:107220004B218C010F5F1F4F9E012F5F3F4F590174
:107230000115110509F460C06FE270E0C8010F94F8
:107240004B216C01009709F458C00817190708F082
:1072500054C04C01801A910AA401B801CE01809655
:107260000F946B21E0E2F0E0EC0FFD1FE80DF91D3B
:1072700010828E01005E1F4FD8018D918D018823F1
:1072800019F00E944359F8CF8AE00E944359609157
:10729000D5127091D6126115710519F06C5F7F4F90
:1072A00002C060E070E021E0AE01405E5F4FCE01C1
:1072B00005960E942EAD811111C0BE01605E7F4F08
:1072C00087E593E00E94A49B8EE20E9443598AE0E6
:1072D0000E944359C5010E948791E6C7B092D61219
:1072E000A092D51286010F5F1F4FA2CF87ED92E1CA
:1072F0009093D6128093D51287016091D512709128
:10730000D6126115710519F06C5F7F4F02C060E005
:1073100070E018A21BA222E0A801CE0180960E9474
:107320002EADF82E882311F1CE0180960E94638C39
:10733000F82E8823D9F06CA57DA58EA59FA541E0E8
:107340000E94D670F82E882389F0E8A9B0E2EB9F5E
:10735000F0011124E55AFB4F309739F085EE808318
:107360001BA20E949870F82E01C0F12CCE018096CD
:107370000E948291FF2011F1A1E3EA2EA3E0FA2EF0
:10738000F7018491882331F0FFEFEF1AFF0A0E9482
:107390004359F6CFD8018D918D01882319F00E94B1
:1073A0004359F8CF8AE00E94435910920515109274
:1073B0000615109207151092081519C0FFE3EF2E5D
:1073C000F3E0FF2EF7018491882331F0FFEFEF1AED
:1073D000FF0A0E944359F6CFD8018D918D01882371
:1073E00019F00E944359F8CF8EE20E944359CE0112
:1073F00001960E94879158C78091621281110E9464
:107400007DFB00916D0610916E0680E50F94B1072B
:10741000882321F00E94315BF82E01C0F12C80916D
:107420006312882309F440C74F2D61E0C8010E9410
:107430004A6883E50F941208882381F00F9433067D
:10744000AB01BC01409305155093061560930715D9
:107450007093081584E594E10E945F748091631233
:10746000882319F081E080936212F1101DC743CE8A
:1074700080916D0690916E0621E02093611240E0AC
:1074800060E00E944A6810C70E945C77ECE3CE2E51
:10749000D12CE12CF12CA70196010F94B81D162FC9
:1074A000072FCA01B901A70196010F94B81DD62E66
:1074B000C72ECA01B90128E130E040E050E00F9446
:1074C000B81DFB01C9016DE671E00F94DE209B0140
:1074D0004D2D5C2DDE0111967D012115310599F0B0
:1074E0000F931F93CF92DF92FF93EF939F938F930E
:1074F0003F932F9383E993E09F938F93FF92AF93F2
:107500000F947D1912C00097B1F00F931F93CF9283
:10751000DF92FF93EF939F938F9383E893E09F9382
:107520008F93FF92AF930F947D190FB6F894DEBF3F
:107530000FBECDBF30C0309779F00F931F93CF921D
:10754000DF92FF93EF9387E793E09F938F93FF92F0
:10755000AF930F947D19E9CF452B69F00F931F93DB
:10756000CF92DF928FE693E09F938F93FF92AF933A
:107570000F947D19DACF0F931F938BE693E09F93BF
:107580008F93FF92AF930F947D190F900F900F90F0
:107590000F900F900F9060E0C7010E941BA4E1E4E0
:1075A000F2E484918F010F5F1F4F882321F00E9426
:1075B0004359F801F6CFB70187EA93E00E94A49BF4
:1075C0008AE00E94435970C683E50F94120888230D
:1075D00009F46AC60E941D5BE82E80E50F9412082C
:1075E000811112C081E0E11001C080E08093730737
:1075F000882329F024982C9A0898109A55C6249A22
:107600002C98089A109850C680E50F941208882389
:1076100031F00F94330677FD47C68B0102C00DE0B1
:1076200010E0802FE4EBF3E09491891731F031966C
:1076300093E0EC3DF907C1F7B7C6E6E0F2E48491C8
:107640008F010F5F1F4F882321F00E944359F801DB
:10765000F6CFECEDF3E084918F010F5F1F4F88238D
:1076600009F422C60E944359F801F5CF0E94907791
:107670001BC60E94477718C688E690E00E94BEC0ED
:10768000811112C68091840683FD0EC683E50F9496
:107690001208882309F408C60F9443060F945A1F52
:1076A0007093F70F6093F60F80E00E9413520F94CF
:1076B000430620E030E040E752E40F94E319181647
:1076C0003CF00E94477760E087EF93E00E942BA494
:1076D0000F9443062091640630916506409166063A
:1076E000509167060F943C2018160CF0DDC58EED06
:1076F00092E09F938F938BEE93E09F938F931F92D3
:107700000E9495760F900F900F900F900F90CCC520
:107710008EE40F941208882309F4C6C50F9433062B
:1077200060935B0670935C0680935D0690935E06A3
:10773000BBC583E50F941208882321F00E941D5BCE
:10774000C82E01C0C12CC0928406E1E4F2E4849109
:107750008F010F5F1F4F882321F00E944359F801CA
:10776000F6CFEAE1F4E084918F010F5F1F4F882389
:1077700021F00E944359F801F6CFCC2099F17CE02A
:10778000E72E74E0F72E00E010E020E0D12CC601D7
:10779000002E02C0959587950A94E2F780FF17C0E6
:1077A00099249394920E222319F08CE20E9443595B
:1077B000F70125913491F90184915901FFEFAF1A36
:1077C000BF0A882329F00E9443599501F4CF922ED5
:1077D0000F5F1F4F22E0E20EF11C0530110571F022
:1077E000292DD5CFE6E1F4E084918F010F5F1F4F83
:1077F000882321F00E944359F801F6CF8AE00E94C5
:10780000435952C50E949F924FC589E690E00E945D
:10781000BEC081110C943C45E1E2F4E084918F01FB
:107820000F5F1F4F882321F00E944359F801F6CFC4
:107830000E94C8F08AE00E9443590C943C4583E5BD
:107840000F941208882309F42FC50E941D5B8093B2
:1078500063068D3318F08CE3809363060F941B0A44
:107860006B017C012091630630E0A8EEB3E00F9439
:10787000061EC60ED71EE81EF91EC0925F06D092E5
:107880006006E0926106F09262060EC58DE690E019
:107890000E94BEC0811108C58091840683FD04C585
:1078A00083E50F94120860968FAF6097811199C598
:1078B00082E50F941208811194C5F6C48091840664
:1078C00083FDF2C483E50F9412086C968FAF6C971A
:1078D00081112AC782E50F941208811125C7E4C4DB
:1078E00083E50F941208882339F00F9433068B0137
:1078F0006F3F710519F010F00FEF10E080E50F9465
:107900001208882331F00E941D5B823008F0CCC43D
:1079100001C080E0E82FF0E0EE0FFF1FEC59FE4EB3
:1079200011830083C1C480E50F941208882339F0C5
:107930000F9433066230710508F0B6C402C060E0EF
:1079400070E0FB01EE0FFF1FEC59FE4E118210821A
:10795000ABC48CE40F94B107882319F00F9443064D
:1079600004C060E070E080E090EC27966CAF7DAFE3
:107970008EAF9FAF27978AE50F941208882319F0DE
:107980000F94430603C060E070E0CB0120E030E0DC
:1079900040E251E40F94161E23966CAF7DAF8EAF7C
:1079A0009FAF239788E50F941208882319F00F944E
:1079B000430603C060E070E0CB0120E030E040E22D
:1079C00051E40F94161E6BAF7CAF8DAF9EAF89E56F
:1079D0000F941208882319F00F94430603C060E047
:1079E00070E0CB0120E030E847E953E40F94161E25
:1079F00020E030E040E251E40F94151E68A379A323
:107A00008AA39BA319821A821B821C82809177060B
:107A100081114AC4C12CE12C8E010F5F1F4F9E01C2
:107A2000205E3F4FAE01455C5F4FBE01615C7F4F02
:107A3000CE018D5B9F4F0E943CE536C410927F06BD
:107A400033C481E080937F062FC483E50F9412082E
:107A5000882399F00F94430620E030E04AE754E48D
:107A60000F94481A0F945F1F60935302709354024F
:107A7000809355029093560217C488E50F94B1077E
:107A80008111D7C789E50F94B1078111D2C78AE563
:107A90000F94B1078111CDC785E40F94B10781110F
:107AA000C8C70E947DFB0F947A06FEC30F94FC07A3
:107AB000FBC30E94F359F8C385E40F94B1078823F0
:107AC00081F00E94315B882361F0E1E4F2E484916B
:107AD0008F010F5F1F4F882321F00E944359F80147
:107AE000F6CF81E40F94B107882381F00E94315BC7
:107AF000882361F0EDE8F4E084918F010F5F1F4F60
:107B0000882321F00E944359F801F6CF00916D06B9
:107B100010916E06D8018D918D01882309F46ECEE7
:107B20000E944359F7CF81E08093730724982C9AE1
:107B30000898109AEBECF4E084918F010F5F1F4FCF
:107B4000882321F00E944359F801F6CFE3ECF4E0DA
:107B500084918F010F5F1F4F882321F00E944359AA
:107B6000F801F6CF1E9B03C009EF12E002C004EF3C
:107B700012E0F80181918F01882319F00E94435986
:107B8000F8CF8AE00E944359EBEBF4E084918F0137
:107B90000F5F1F4F882321F00E944359F801F6CF51
:107BA000029B03C009EF12E002C004EF12E0D8010B
:107BB0008D918D01882319F00E944359F8CF8AE0F6
:107BC0000E944359E3EBF4E084918F010F5F1F4F54
:107BD000882321F00E944359F801F6CF1D9B03C072
:107BE00009EF12E002C004EF12E0F80181918F0169
:107BF000882319F00E944359F8CF8AE00E94435924
:107C0000EBEAF4E084918F010F5F1F4F882321F08E
:107C10000E944359F801F6CF019B03C009EF12E01F
:107C200002C004EF12E0D8018D918D01882319F074
:107C30000E944359F8CF8AE00E944359E3EAF4E0F6
:107C400084918F010F5F1F4F882321F00E944359B9
:107C5000F801F6CF1C9903C009EF12E002C004EF4F
:107C600012E0F80181918F01882319F00E94435995
:107C7000F8CF8AE00E944359EBE9F4E084918F0148
:107C80000F5F1F4F882321F00E944359F801F6CF60
:107C9000379B03C009EF12E002C004EF12E0D801E5
:107CA0008D918D01882319F00E944359F8CF8AE005
:107CB0000E944359E1E9F4E084918F010F5F1F4F67
:107CC000882321F00E944359F801F6CF009903C0A0
:107CD00009EF12E002C004EF12E0F80181918F0178
:107CE000882319F00E944359F8CF8AE00E94435933
:107CF00010927307249A2C98089A1098D5C2109263
:107D0000720710927107D0C20E948059CDC20E94A2
:107D10008658CAC20F94DF07C7C20E94B45AC4C2B1
:107D20000E9402BFC1C20F941E08BEC280E50F941C
:107D3000B107882309F4B8C20F943306F62E062F34
:107D4000172F83E50F941208882321F00F94330630
:107D50006B0103C0CC24CA94DC2C96012F5F3F4FEB
:107D60002330310508F0A0C217FD9EC20E947DFBA2
:107D7000FFEFCF16DF0631F0CA94CD2871F000E096
:107D800010E00DC08F2D0F94BE0931E020E0892B4B
:107D900009F030E0032F122F02C001E010E08F2D18
:107DA0000F94BE098017910709F47EC280E00E94FB
:107DB00054F1F5CF83E50F941208882319F00F943E
:107DC000330602C064E071E079A368A380E50F94F4
:107DD0001208882339F00F943306693833E17307AA
:107DE00030F402C068EE73E07A83698304C088E8E7
:107DF00093E19A838983BE01605E7F4FCE01019635
:107E00000E94BB6D51C20E9487BD4EC20E9421BE1E
:107E10004BC20E945A4F48C281E00E940AEB44C202
:107E200086E50F94B107882321F082E195E00E9456
:107E300051C083E50F94B107882321F00E94315B84
:107E4000182F01C010E083E50F94B107882319F0C3
:107E5000812F0E94E691F0906F06111103C0E1E4BA
:107E6000F2E41AC0F110FBCFE6E0F2E484918F0156
:107E70000F5F1F4F882321F00E944359F801F6CF6E
:107E8000E3EFF4E084918F010F5F1F4F882339F3F4
:107E90000E944359F801F6CF84918F010F5F1F4F65
:107EA000882321F00E944359F801F6CFFF2019F0F2
:107EB00063E073E002C067E073E085EE94E00E9447
:107EC000A49B8AE00E944359EFC10F94F503ECC1D3
:107ED0000E9426FEE9C10E94E0FCE6C10E944A64BD
:107EE000E3C10E94405BE0C10E94B95FDDC10E9416
:107EF000B076882319F081E00F94001185E40F9487
:107F0000B107882319F00F94430604C060E070E0C5
:107F100080E090EC2F966CAF7DAF8EAF9FAF2F9728
:107F20008AE50F941208882319F00F94430604C0C1
:107F300060E070E080E291E42B966CAF7DAF8EAF95
:107F40009FAF2B9788E50F941208882319F00F94A0
:107F5000430604C060E070E080E291E427966CAFD5
:107F60007DAF8EAF9FAF279789E50F9412088823C6
:107F700019F00F94430604C060E070E882E993E4CE
:107F800023966CAF7DAF8EAF9FAF239785E50F949F
:107F9000B107882319F00F94430604C060E070E035
:107FA00088EC92EC6BAF7CAF8DAF9EAF8CE40F94FE
:107FB000B107882319F00F94430603C060E070E016
:107FC000CB0168A379A38AA39BA382E40F94120830
:107FD000882321F00F943306F62E02C085E0F82E98
:107FE000D09053128091770681117EC0CC24C39427
:107FF000EF2C8E01055C1F4F9E01215C3F4FAE01AF
:108000004D5B5F4FBE01695B7F4FCE01855B9F4F2C
:108010000E943CE5882309F467C081E08093370A19
:1080200011E08091370A882309F44AC060E08F2D5F
:108030000E94316E809176068823F1F110937106CB
:1080400040E050E0BA0185EB96E90E94ECA68091F1
:10805000370A882321F081E00E9454F1F8CF109272
:1080600072061092730610927406109275061092A2
:1080700076060E9413520E9452F31093710640E05C
:1080800050E0BA018BE095E90E94ECA60F941B0A20
:10809000685370458F4F9F4F6093720670937306BD
:1080A0008093740690937506109276061093370AA3
:1080B00061E08F2D0E94316E81E00E9454F1B1CFBA
:1080C00000E010E028E432E409831A832B833C8328
:1080D00080917706882341F04F2DBE016F5F7F4F5F
:1080E000CE0180960E9414E441E0D412DDC00E94CB
:1080F0009077DAC00E94F45ED7C083E50F9412082F
:10810000882309F449C00E941D5B813039F0823018
:1081100009F042C008E213E0F12C23C008E213E0AA
:10812000F12CD8018D918D010F941208882339F01C
:108130000E941D5B4FEF682F8F2D0E944856F394CD
:10814000B4E0FB12EECF82E40F941208882321F1F1
:108150000E941D5B4FEF682F1CC0F394F4E0FF16E4
:1081600079F0F80181918F010F9412088823A9F307
:108170000E941D5B482F6FEF8F2D0E944856EDCF58
:1081800082E40F941208882339F00E941D5B482F67
:108190006FEF84E00E9448560E94634E85C0E6E07F
:1081A000F2E484918F010F5F1F4F882321F00E941A
:1081B0004359F801F6CFEFE2F5E084918F010F5FAC
:1081C0001F4F882309F470C00E944359F801F5CF6E
:1081D00081E0809357021092780683E50F94B107EF
:1081E000811103C00E94FB4D5FC00E94315B811171
:1081F0005BC0F8CFF0908106FF2021F1E1E4F2E4CA
:1082000084918F010F5F1F4F882321F00E944359F3
:10821000F801F6CF84E50E9443596F2D70E080E0AD
:1082200090E04AE00E94934C80E20E9443590BE0A8
:1082300013E0D8018D918D01882309F4DFCA0E94D3
:108240004359F7CF10927906E1E4F2E484918F016B
:108250000F5F1F4F882321F00E944359F801F6CF8A
:1082600060E070E08EE395E00E94414F8AE00E945A
:1082700043591AC0E1E4F2E484918F010F5F1F4F6C
:10828000882321F00E944359F801F6CF60917A06C5
:1082900070917B0680E595E00E94A49B82E20E949B
:1082A00043598AE00E9443590E94934DE5C32091AF
:1082B0006D0630916E06232B39F49F012150310950
:1082C00030936E0620936D0620E030E00C94682C0D
:1082D00080E00E94E6910F944A0A83E50F94B1076B
:1082E000882309F449C00E94315B21E0482FBE0178
:1082F0006F5F7F4FCE0180960E94B4786B017C0146
:108300009B01AC010F94C220811131C02CEA35ECE5
:1083100047E257E368A179A18AA19BA10F94161E99
:10832000AB01BC0181EA92E00E944DBD2CEA35EC24
:1083300047E257E369817A818B819C810F94161EF5
:10834000AB01BC018CE992E00E944DBD2CEA35ECFA
:1083500047E257E3C701B6010F94161EAB01BC01FB
:1083600087E992E00E944DBD8AE00E9443590F9434
:10837000310A0E9492BF98CF81E0B7CF80E00E947F
:1083800054F10C94CC370F943306AB01BC014093ED
:10839000051550930615609307157093081584E52D
:1083A00094E10E945F7480CF802F0E94B14F6E2DA8
:1083B000802F0F94E609F12CB701802F0E94D04F37
:1083C0000630110529F4F0926711E09266116CCF26
:1083D0000830110509F068CFF0926511E092641140
:1083E00063CF0F9443060F945A1F7093F70F609357
:1083F000F60F80E00E9413520F94430620E030E015
:1084000040E752E40F94E319181644F00E944777AE
:1084100060E080E594E00E942BA402C00E94907767
:108420006091F60F7091F70F882777FD8095982F50
:108430000F94E91920916406309165064091660613
:10844000509167060F943C2018160CF065C18EED14
:1084500092E09F938F9384E494E09F938F931F9275
:108460000E9495760F900F900F900F900F9081E0E3
:108470008093890267961CAE1DAE1EAE1FAE679735
:108480006B961CAE1DAE1EAE1FAE6B9710E0A09695
:108490001FAEA0973CE3A4963FAFA4974CE1A896EB
:1084A0004FAFA89756E4AC965FAFAC97D12CE12CB8
:1084B00060E8F62E0FEB812C912C54016091F60FA1
:1084C0007091F70F882777FD8095982F0F94E91901
:1084D000762E672E582E492E262F372F482F592FAC
:1084E0006D2D7E2D8F2D902F0F94E3198823D9F0B9
:1084F00020916406309165064091660650916706AA
:10850000672D762D852D942D0F94E319182F111FAB
:108510001127111F60968FAD6097882341F01123BA
:1085200031F011E0E7C07D2C6E2C5F2C402E0F94B3
:108530001B0A6B017C01DC01CB016B962CAD3DADC0
:108540004EAD5FAD6B97821B930BA40BB50BB7FDC4
:108550003BC0D701C60188519C4FAF4FBF4F6B96B0
:108560008CAF9DAFAEAFBFAF6B970E94C8F0E0E499
:10857000F4E084911F019FEF291A390A882321F022
:108580000E944359F101F5CF81149104A104B10473
:10859000A9F0C501B40168517C4F8F4F9F4F6C19F2
:1085A0007D098E099F0928EE33E040E050E00F94EA
:1085B000B81DCA01B9010E94044D03C08FE30E9497
:1085C00043598AE00E94435980E00E9454F10F947D
:1085D000270AA09164066C96AFAF6C972090650651
:1085E00030906606009167062A2F322D432D502FBA
:1085F000672D762D852D942D0F94151E9F7720E0E5
:1086000030E040E251E481149104A104B10429F462
:108610000F94E31987FD05C006C00F943C2018167F
:1086200014F446015701112309F44AC067962CAD92
:108630003DAD4EAD5FAD6797211531054105510543
:1086400041F0D701C601821B930BA40BB50BB7FDFC
:1086500037C06C962FAD6C97322D432D502FA096BE
:108660006FADA097A4967FADA497A8968FADA8975D
:10867000AC969FADAC970F94151E20E030E040EC17
:108680005FE30F94E31987FD4CCFD701C601805AF1
:108690009541AF4FBF4F67968CAF9DAFAEAFBFAFA9
:1086A00067976C969FAD6C97A0969FAFA097A49686
:1086B0002FAEA497A8963FAEA897AC960FAFAC97F5
:1086C000809189028823B1F081149104A104B1043E
:1086D00029F4D72CE62CF52C042DF0CEA8EECA1ADE
:1086E000A3E0DA0AE108F108C818D908EA08FB088B
:1086F000F7FCEFCF80918902882309F4D5CD60E0A3
:10870000112329F084E294E00E942BA4CDCD82E3D2
:1087100094E00E942BA4C8CD6096BFAD6097B111C4
:10872000A6CE89EE92E095CE0F9443060F945A1F81
:108730006739710514F066E970E07093F30F609388
:10874000F20F0E94C9510F94430620E030E040EA46
:1087500050E40F943C20181614F40E949077609116
:10876000F20F7091F30F882777FD8095982F0F9463
:10877000E919209168063091690640916A06509186
:108780006B060F94E31960E087FF03C080E894E074
:1087900002C083E794E00E942BA481E080938902C9
:1087A0008091790680936C0667961CAE1DAE1EAE56
:1087B0001FAE67976B961CAE1DAE1EAE1FAE6B97BD
:1087C00060961FAE6097A0961FAEA097BCE3A496DC
:1087D000BFAFA497ECE1A896EFAFA897F6E4AC96EC
:1087E000FFAFAC97C12CD12C40E8E42E5FEBF52E07
:1087F000812C912C54016091F20F7091F30F882716
:1088000077FD8095982F0F94E919162F072F782E52
:10881000692E262F372F482F592FB601C7010F94E5
:10882000E319882331F1209168063091690640915F
:108830006A0650916B06612F702F872D962D0F942D
:10884000E319881F8827881F60968FAF60976C9602
:108850002FAD6C97222389F0882379F080918902CB
:10886000882309F421CD60E085E694E00E942BA4E2
:108870001BCD1C2D0D2D7E2C6F2C0F941B0A6B0114
:108880007C01DC01CB016B962CAD3DAD4EAD5FADF7
:108890006B97821B930BA40BB50BB7FD3BC0D701A5
:1088A000C60188519C4FAF4FBF4F6B968CAF9DAFA9
:1088B000AEAFBFAF6B970E94C8F0EFE6F4E08491D3
:1088C0002F019FEF491A590A882321F00E9443592A
:1088D000F201F5CF81149104A104B104A9F0C501FE
:1088E000B40168517C4F8F4F9F4F6C197D098E09E1
:1088F0009F0928EE33E040E050E00F94B81DCA0114
:10890000B9010E94044D03C08FE30E9443598AE0DD
:108910000E94435980E00E9454F10F94270A20904E
:1089200068063090690640906A0650906B06910187
:10893000A201612F702F872D962D0F94151E9F7702
:1089400020E030E040EA50E481149104A104B10435
:1089500029F40F94E31987FD05C006C00F943C204D
:10896000181614F4460157016096AFAD6097AA231C
:1089700009F443C067962CAD3DAD4EAD5FAD679732
:10898000211531054105510541F0D701C601821B72
:10899000930BA40BB50BB7FD30C09101A201A096BB
:1089A0006FADA097A4967FADA497A8968FADA8971A
:1089B000AC969FADAC970F94151E20E030E040ECD4
:1089C0005FE30F94E31987FD49CFD701C601805AB1
:1089D0009541AF4FBF4F67968CAF9DAFAEAFBFAF66
:1089E0006797A0962FAEA097A4963FAEA497A8969F
:1089F0004FAEA897AC965FAEAC9780918902882362
:108A000009F42CCF81149104A104B10429F4C12EDE
:108A1000D02EE72CF62CEFCE98EEC91A93E0D90AA7
:108A2000E108F108C818D908EA08FB08F7FE16CFD4
:108A3000EECF0E947DFB88E50F94B107882319F0E3
:108A4000179A10926E0789E50F94B107882319F0E1
:108A5000169A10926F078AE50F94B107882319F0D0
:108A6000159A1092700785E40F94B107882309F4D2
:108A70001BCC0F94780618CCC757DF4F0FB6F8946D
:108A8000DEBF0FBECDBFDF91CF911F910F91FF9041
:108A9000EF90DF90CF90BF90AF909F908F907F909E
:108AA0006F905F904F903F902F9008950F93CF93CA
:108AB000DF93C82FD62F04E0262F41E3682F81EBE8
:108AC00091E10F94FD088823C9F02D2F41E36C2F0D
:108AD00081EB91E10E94D2B78C2F0E94B8928FEF68
:108AE0008D0F8C0F0E94B8922D2F44E36C2F81EBD9
:108AF00091E1DF91CF910F910C94D2B7DF91CF919B
:108B00000F9108957F928F929F92AF92BF92CF92D2
:108B1000DF92EF92FF920F931F93CF93DF93CDB726
:108B2000DEB72A970FB6F894DEBF0FBECDBF109206
:108B3000911180918911882351F00E94E5AC40E0A9
:108B400050E0BA0188E29CEE0E94ECA6C9C44091B4
:108B5000A6025091A70280918D1190918E11A09143
:108B60008F11B09190119A01280F391F4436510589
:108B700024F4253631053CF41CC04436510551F02F
:108B800024363105B4F484E690E09093A7028093F4
:108B9000A60213C08B309105A105B1051CF02A5027
:108BA000310907C0863F9F4FAF4FBF4F74F4265F18
:108BB0003F4F3093A7022093A60210928D1110927E
:108BC0008E1110928F11109290118091A6029091A7
:108BD000A7028A3091053CF0883E23E092072CF0F2
:108BE00087EE93E002C08AE090E09093A702809322
:108BF000A6020E9448A4782E0E94806F8091E51101
:108C0000853198F4772049F0809164119091651135
:108C1000892B19F00CEF11E102C00FED10E123E1F7
:108C20004FE061E089E00E944A928091E5118D3128
:108C300008F084C1883008F03FC08091760671103A
:108C400002C0811139C06091F60F7091F70F88272B
:108C500077FD8095982F0F94E91920E030E040E0EF
:108C60005FE30F94161E0F945A1F643671052CF49F
:108C70006A30710524F04CE003C042E101C046E0D7
:108C800022E130E0241B310937FF02C02F5F3F4F44
:108C9000359527953195219531092B5F2093E81162
:108CA00027E02093E911CB010E94759E0E94C96FB5
:108CB0008CED90E10E94BC6F8091E5118D31D0F573
:108CC0008091E7118531B0F120E030E040E05FE3D2
:108CD00060916406709165068091660690916706C2
:108CE0000F94161E0F945A1F9B01643671050CF0E9
:108CF000F4C22A3031050CF4EEC24CE022E130E03F
:108D0000241B310937FF02C02F5F3F4F3595279550
:108D10003195219531092B5F2093E8112CE12093A7
:108D2000E911CB010E94759E0E94C96F8CED90E104
:108D30000E94BC6F8091E511853140F58091E7116B
:108D4000813120F16091F60F7091F70F882777FD40
:108D50008095982F0F94E91920916406309165064B
:108D600040916606509167060F943C2018160CF04F
:108D7000B6C21092D11102E022E041E16DE081EB38
:108D800091E10E9452B881E08093D1118091E51168
:108D9000883008F03FC080918806711002C08111B0
:108DA00039C06091F20F7091F30F882777FD80959D
:108DB000982F0F94E91920E030E040E05FE30F9432
:108DC000161E0F945A1F643671052CF46A30710513
:108DD00024F04CE003C042E101C046E022E130E073
:108DE000241B310937FF02C02F5F3F4F3595279570
:108DF0003195219531092F5A2093E81127E02093CE
:108E0000E911CB010E94759E0E94C96F8CED90E123
:108E10000E94BC6F8091E5118D31D0F58091E711F2
:108E20008531B0F120E030E040E05FE3609168061A
:108E30007091690680916A0690916B060F94161ED8
:108E40000F945A1F9B01643671050CF053C22A30EF
:108E500031050CF44DC24CE022E130E0241B310915
:108E600037FF02C02F5F3F4F3595279531952195EC
:108E700031092F5A2093E8112CE12093E911CB01FD
:108E80000E94759E0E94C96F8CED90E10E94BC6F9C
:108E90008091E511853140F58091E711813120F114
:108EA0006091F20F7091F30F882777FD8095982FCE
:108EB0000F94E919209168063091690640916A067D
:108EC00050916B060F943C2018160CF015C21092AE
:108ED000D11102E022E042E168E581EB91E10E94DC
:108EE00052B881E08093D1118091E5118C3130F539
:108EF0008091E711843110F1809164119091651196
:108F0000019644E6489F9001499F300D112437FF98
:108F100002C021503F4F832F932F990F990B009739
:108F200069F028E62093E8112BE12093E9110E94D3
:108F3000759E0E94C96F85E20E949F6F8091E51126
:108F4000843328F48091E7118A3208F0DEC18091E1
:108F5000E511853328F48091E711813308F0FAC1D7
:108F600080916212882309F44DC08091E511843309
:108F700008F048C08091E711823308F443C0809123
:108F80005714882309F4EAC18091011590910215C4
:108F9000A0910315B09104150097A105B10509F43E
:108FA000DDC1BC01CD016D597F4F8F4F9F4F24E62E
:108FB00030E040E050E00F94B81D609105157091CD
:108FC000061580910715909108150F94B81D622F12
:108FD00048E4649FB0011124882777FD8095982F7D
:108FE0000F94E9192AE037ED43E25CE30F94481A45
:108FF0000F945F1F262F02E042E367E381EB91E1CC
:109000000E9452B88091E511813308F05DC08091D3
:10901000E711893208F458C00E945C776B017C012B
:109020008CE3882E912CA12CB12CC701B601A5018F
:1090300094010F94B81DCA01B901A50194010F94C0
:10904000B81DCA01962E872E59018E010F5F1F4F42
:1090500041E8C41641E5D40641E0E406F10408F411
:109060007FC1B90128E130E040E050E00F94B81D25
:1090700079018F929F92C50168E170E00F94DE2024
:109080009F938F933F932F932CE136E03F932F9341
:109090001F930F930F947D190FB6F894DEBF0FBE88
:1090A000CDBF9AE0E916F10408F489C198E0892F50
:1090B000880F890F8195855A8093E81180E380930A
:1090C000E911C8010E94C96FE091AB11F091AC1198
:1090D00084818111CCC0609180077091810780915B
:1090E0008207909183070F945A1FCB010E940C9E18
:1090F000BC018EE996E00F9456216091840770912F
:10910000850780918607909187070F945A1FCB019E
:109110000E940C9EBC0189E996E00F9456212CEA2E
:1091200035EC47E257E36091880770918907809199
:109130008A0790918B070F94161E20E030E048ECD0
:1091400052E40F94481A0F945A1F6B017C0197FD4B
:1091500019C090E1C91697E2D906E104F104E4F0E0
:10916000C701B60120E137E240E050E00F94DA1D7C
:10917000CA01B9012AE030E040E050E00F94DA1D66
:10918000605D0BC0F094E094D094C094C11CD11CDD
:10919000E11CF11C6DE201C060E260938A0628EEDA
:1091A000C21623E0D206E104F10494F0C701B6012F
:1091B00028EE33E040E050E00F94DA1DCA01B90117
:1091C0002AE030E040E050E00F94DA1D605D01C01D
:1091D00060E260938B06C701B60124E630E040E010
:1091E00050E00F94DA1D9AE0892E912CA12CB12C1D
:1091F000CA01B901A50194010F94DA1D605D609365
:109200008C06C701B601A50194010F94DA1D162F33
:10921000662381F08EE280938D06CA01B901A50113
:1092200094010F94DA1D605D60938E06105D1093BB
:109230008F0617C0CA01B901A50194010F94DA1D68
:10924000662339F08EE280938D06605D60938E0612
:1092500005C080E280938E0680938D0680E2809325
:109260008F066AE876E082E996E00F9456218091B5
:10927000E5118632A8F48091E7118E3188F008E07C
:1092800020E84EE160E081EB91E10E9452B88091CC
:10929000E511863228F48091E7118F3108F091C0F2
:1092A0008091E511823328F48091E7118C3208F027
:1092B000F8C08091E5118F3308F012C18091E71159
:1092C000883308F40DC11092E8118EE38093E91100
:1092D0000E941D7005C146E011CD42E10FCD02E0B4
:1092E00022E041E16DE081EB91E10E9452B84ECD68
:1092F00046E0B2CD42E1B0CD02E022E042E168E5D5
:1093000081EB91E10E9452B8EFCD07E028E04AE2FC
:109310006AE281EB91E10E9452B805E022E04CE262
:1093200062E381EB91E10E9452B86AE08AE2BEDB1F
:109330006091B3117091B41182E38093CD118BE2EF
:109340008093CE112DEC31E142E381EB91E10F945A
:109350001F09FDCD6AE486E3A9DB02CE60E038CECA
:1093600044E6A416B104C0F48F929F92C50168E14F
:1093700070E00F94DE209F938F9382E196E09F939D
:109380008F931F930F930F947D190FB6F894DEBF40
:109390000FBECDBF95E08BCE8F929F923F932F93C0
:1093A0008AE096E09F938F931F930F930F947D19FC
:1093B0000FB6F894DEBF0FBECDBF96E078CE97E033
:1093C00076CE1092D11183E08093E81185E28093EC
:1093D000E911772029F08AED90E10E94BC6F0DC061
:1093E0008091A711811102C08FE305C080916E07A3
:1093F0008111F1CF80E20E949F6F8BE08093E81192
:1094000015E21093E9118EE996E00E94C96F8BE294
:109410008093E8111093E911772029F088ED90E10D
:109420000E94BC6F0DC08091A811811102C08FE312
:1094300005C080916F078111F1CF80E20E949F6F7C
:1094400083E38093E81115E21093E91189E996E02E
:109450000E94C96F83E58093E8111093E91177208A
:1094600029F086ED90E10E94BC6F0DC08091A9119A
:10947000811102C08FE305C0809170078111F1CF87
:1094800080E20E949F6F8BE58093E81185E28093D4
:10949000E91182E996E00E94C96F81E08093D111C1
:1094A000FFCE84E00E94876F83E08093E81112E38F
:1094B0001093E91186E00E94AA6F0E94806F8CE0F1
:1094C0008093E8111093E9118091A6029091A70270
:1094D0000E94759E0E94C96F85E20E949F6FE9CE2F
:1094E0002A960FB6F894DEBF0FBECDBFDF91CF91A5
:1094F0001F910F91FF90EF90DF90CF90BF90AF90B2
:109500009F908F907F9008951F93CF93DF93109239
:10951000911180918D1190918E11A0918F11B09128
:10952000901181309048A105B10540F010928D1145
:1095300010928E1110928F1110929011C0918D1176
:1095400040918606141604F5842F992787FD90957F
:1095500005972C2F332727FD309528173907A4F0BE
:1095600045301CF0CBEFC40F01C0C0E08C2F992711
:1095700087FD9095A92FB92F80938D1190938E110F
:10958000A0938F11B0939011C0938A11D0E012E094
:10959000C11109C08091A8028823D9F121E041E0DE
:1095A00067EC75E020C0C13049F48091A80288239F
:1095B00081F120E041E068EB75E015C0C23049F46C
:1095C0008091A802882329F120E041E068EA75E053
:1095D0000AC0C33061F48091A8028823D1F020E052
:1095E00041E061EA75E08D2F0E94A49412C0C4305E
:1095F00081F48091A802882351F021E040E066E9DF
:1096000075E08D2F0E94A4948D2F0E94D46F10932B
:10961000A802DF5FCF5FD53009F0BACFD0938606BE
:10962000DF91CF911F9108951F93CF93DF931092F5
:10963000911180918D1190918E11A0918F11B09107
:10964000901181309048A105B10540F010928D1124
:1096500010928E1110928F1110929011C0918D1155
:1096600040918506141604F5842F992787FD90955F
:1096700005972C2F332727FD309528173907A4F09D
:1096800045301CF0CBEFC40F01C0C0E08C2F9927F0
:1096900087FD9095A92FB92F80938D1190938E11EE
:1096A000A0938F11B0939011C0938A11D0E012E073
:1096B000C11109C08091A8028823D9F121E041E0BD
:1096C00069E875E020C0C13049F48091A802882380
:1096D00081F120E041E060E875E015C0C23049F456
:1096E0008091A802882329F120E041E060E775E03D
:1096F0000AC0C33061F48091A8028823D1F020E031
:1097000041E06EE675E08D2F0E94A49412C0C43033
:1097100081F48091A802882351F021E040E063E6C3
:1097200075E08D2F0E94A4948D2F0E94D46F10930A
:10973000A802DF5FCF5FD53009F0BACFD09385069E
:10974000DF91CF911F9108950F931F93CF93DF93D4
:109750001092911180918D1190918E11A0918F1185
:10976000B091901181309048A105B10540F0109260
:109770008D1110928E1110928F1110929011C09134
:109780008D11409187061416D4F4842F992787FDF4
:10979000909501972C2F332727FD309528173907EF
:1097A00074F0CFEFC40F8C2F90E0A0E0B0E0809376
:1097B0008D1190938E11A0938F11B09390111092F0
:1097C0008B1180918A11C81714F4C0938A1180916B
:1097D0008A11992787FD909504962C2F332727FD12
:1097E00030958217930724F48CEF8C0F80938A11A5
:1097F00010918A11D0E081E002E0111123C088238A
:10980000B9F01C16ACF040918D1150918E11609101
:109810008F11709190114F5F5F4F6F4F7F4F40934B
:109820008D1150938E1160938F1170939011CF5FB3
:109830008091A802882309F469C021E041E06BEF20
:1098400075E04EC0113019F58823B9F0C230ACF480
:1098500040918D1150918E1160918F1170919011E6
:109860004F5F5F4F6F4F7F4F40938D1150938E111D
:1098700060938F1170939011CF5F8091A80288231D
:1098800009F444C020E040E066EE75E029C01230E3
:10989000E9F480918911811105C08091A802882383
:1098A000A9F109C0C230C9F70E944AA780918B1163
:1098B000882399F333C081E0C23009F080E024E0CE
:1098C00041EE55E06D2F0E941EB920C0133061F4A7
:1098D0008091A8028823D1F020E041E06FED75E08F
:1098E0008D2F0E94A49412C0143081F48091A8029C
:1098F000882351F021E040E064ED75E08D2F0E9457
:10990000A4948D2F0E94D46F0093A802DF5F1F5F85
:10991000D53011F080E071CFD0938706DF91CF91E1
:109920001F910F910895AF92BF92CF92DF92EF9265
:10993000FF920F931F93CF93DF93CDB7DEB7A0971E
:109940000FB6F894DEBF0FBECDBF6115710581055E
:109950009105B1F1B12CC42ED12CE12CF12CAA240B
:10996000A394AB0C01E010E00C0F1D1F0B0D111D9B
:10997000B7FC1A95A70196010F94B81DF8016083F2
:10998000B901CA01611571058105910511F41B2DFD
:1099900012C0BA2CE4CFE1E0F0E0EC0FFD1FE10FC4
:1099A000F11D17FDFA9580818A3040F490E3890F0C
:1099B0000E94435911501F3F71F715C097E3F7CF2D
:1099C00080E3A0960FB6F894DEBF0FBECDBFDF9147
:1099D000CF911F910F91FF90EF90DF90CF90BF90AC
:1099E000AF900C944359A0960FB6F894DEBF0FBE0B
:1099F000CDBFDF91CF911F910F91FF90EF90DF903E
:109A0000CF90BF90AF900895CF92DF92EF92FF92E8
:109A10006B017C0197FF0BC08DE20E944359F094CB
:109A2000E094D094C094C11CD11CE11CF11C4AE00C
:109A3000C701B601FF90EF90DF90CF9074CF8F9267
:109A40009F92AF92BF92CF92DF92EF92FF92CF930D
:109A50006B017C01B42E20E030E0A9010F94E319E2
:109A600087FF07C08DE20E944359F7FAF094F7F898
:109A7000F094C0E060E070E080E09FE3CB1541F03F
:109A80002DEC3CEC4CEC5DE30F94481ACF5FF6CF25
:109A90009B01AC01C701B6010F94161E6B017C013E
:109AA0000F945F1F4B015C014AE03DDFCC2389F13D
:109AB000C501B4010F94E7199B01AC01C701B601C0
:109AC0000F94151E6B017C018EE20E94435920E029
:109AD00030E040E251E4C701B6010F94481A6B012F
:109AE0007C010F945A1F4B01AA2497FCA094BA2C16
:109AF000C501B40189DFC501B4010F94E9199B01C7
:109B0000AC01C701B6010F94151E6B017C01C15059
:109B1000F1F6CF91FF90EF90DF90CF90BF90AF9094
:109B20009F908F900895CF93DF930F94270AE09131
:109B30003209F0E0E057F84F8081882309F458C0DB
:109B4000EBECF3E18491EF012196882321F00E9450
:109B50004359FE01F7CFC091320980E6C89FE0016A
:109B60001124CE54D84F88818E3419F0E8ECF3E1FB
:109B700010C080E20E94435989910E944359899103
:109B800090ED980F9A30C8F38D32B9F38B32A9F368
:109B9000EDCF8491EF012196882321F00E94435953
:109BA000FE01F7CF0F9493086FE070E0681B710916
:109BB000882777FD8095982F27DFE5ECF3E18491E6
:109BC000EF012196882321F00E944359FE01F7CF2F
:109BD0008091330964E070E0681B7109882777FD84
:109BE0008095982F11DF8AE0DF91CF910C94435933
:109BF000DF91CF910895CF93DF938FB7F894909131
:109C0000BA0A9093B90A8FBFEEECF3E18491EF01A9
:109C10002196882321F00E944359FE01F7CF6091DD
:109C20005B0670915C0680915D0690915E066F5FA9
:109C30007F4F8F4F9F4FE8DE8AE00E944359DF91AC
:109C4000CF9171CFEF92FF920F931F93CF93DF933A
:109C50001F92CDB7DEB7082F162FE6E0F2E484910D
:109C60007F012FEFE21AF20A882331F099830E94D4
:109C70004359F7019981F3CFE02FF92F84917F01A8
:109C80009FEFE91AF90A882321F00E944359F7014E
:109C9000F5CF60915B0670915C0680915D069091B6
:109CA0005E06B2DE8AE00E9443591111A4DF1092D1
:109CB000C5101092C4100F90DF91CF911F910F919A
:109CC000FF90EF900895CF93DF93E7EBF3E184915A
:109CD000EF012196882321F00E944359FE01F7CF1E
:109CE000E3EBF3E18491EF012196882321F00E94B8
:109CF0004359FE01F7CF62B36695617070E080E072
:109D000090E082DE62B3617070E080E090E07CDE23
:109D10008AE00E944359EFEAF3E18491EF01219632
:109D2000882321F00E944359FE01F7CF609106017C
:109D3000772767FD7095872F972F662797FD639587
:109D400077278827992760DE62B362FB662760F970
:109D500070E080E090E058DE8AE00E944359EBEA30
:109D6000F3E18491EF012196882321F00E94435969
:109D7000FE01F7CF6091060166FB662760F970E08F
:109D800080E090E041DE6091060165FB662760F9A6
:109D900070E080E090E038DE8AE00E944359E6EA15
:109DA000F3E18491EF012196882321F00E94435929
:109DB000FE01F7CF6091060163FB662760F970E052
:109DC00080E090E021DE609106016295617070E0B4
:109DD00080E090E019DE8AE00E944359E1EAF3E175
:109DE0008491EF012196882321F00E944359FE01BE
:109DF000F7CF609106016695617070E080E090E0B9
:109E000003DE6091060162FB662760F970E080E086
:109E100090E0FADD8AE0DF91CF910C9443591F93D3
:109E2000CF93DF9383E50F94B107811104C0C8E29B
:109E3000D3E010E00DC0C0E00E941D5B682F8C2FA6
:109E4000D1D7CF5FC530C1F7F2CF1F5F143059F0C3
:109E500089910F94B1078823C1F30E941D5B682F7D
:109E6000812FC0D7F2CF82E40F94B107882329F065
:109E70000E941D5B682F84E0B5D7DF91CF911F91C1
:109E800022CF0F931F93CF93DF938B01FC0184911B
:109E9000EF012196882321F00E944359FE01F7CF5C
:109EA000B801882777FD8095982FDF91CF911F917A
:109EB0000F91AACDCF93DF9383E50F94B107C82FFD
:109EC000882371F00F9443060F945A1F70930B026E
:109ED00060930A0221E0672B09F020E020933A0406
:109EE00080E50F94B107882369F080910A02909170
:109EF0000B02892B19F00E94315B01C081E0809335
:109F00003A042CC0C1112AC0E1E4F2E48491EF01CB
:109F10002196882321F00E944359FE01F7CF8091BA
:109F20003A04882319F066EF72E002C06CE273E035
:109F30008EE893E10E94A49B60910A0270910B024B
:109F40008DE793E19EDFE9E7F3E18491EF0121964C
:109F5000882321F00E944359FE01F7CFDF91CF9172
:109F6000089590E0FC01EF51F04C2491FC01E95D73
:109F7000FF4B8491882399F090E0880F991FFC0192
:109F8000E953F04CA591B491875E9C4EFC018591FC
:109F900094919FB7F8948C91822B8C939FBF0895D6
:109FA0001F93CF93DF93182FEB01DBDF209711F482
:109FB00060E004C0CF3FD10539F461E0812FDF912B
:109FC000CF911F910D94E609E12FF0E0ED5CFC4E7E
:109FD000449150E0FA013197E231F10508F09BC05D
:109FE000EE58FF4F0D94052184B5806884BDC7BD30
:109FF00097C084B5806284BDC8BD92C08091800046
:10A00000806880938000D0938900C093880088C0C6
:10A0100080918000806280938000D0938B00C093F9
:10A020008A007EC080918000886080938000D093F9
:10A030008D00C0938C0074C08091B00080688093C4
:10A04000B000C093B3006CC08091B0008062809378
:10A05000B000C093B40064C0809190008068809389
:10A060009000D0939900C09398005AC080919000BE
:10A07000806280939000D0939B00C0939A0050C060
:10A0800080919000886080939000D0939D00C09351
:10A090009C0046C08091A00080688093A0008091C1
:10A0A000A0008F7B8093A000D093A900C093A8004C
:10A0B00037C08091A00080628093A000D093AB0055
:10A0C000C093AA002DC08091A00088608093A0005A
:10A0D000D093AD00C093AC0023C080912001806874
:10A0E00080932001D0932901C093280119C0809149
:10A0F0002001806280932001D0932B01C0932A011C
:10A100000FC080912001886080932001D0932D01A1
:10A11000C0932C0105C0C038D1050CF04ECF48CFFC
:10A12000DF91CF911F9108951F93CF93DF93E0911B
:10A13000BF11F091C011309719F081EB91E11995A1
:10A14000C091B311D091B411E091E211F091E311FB
:10A1500082E01995E091E211F091E31181E0199507
:10A1600020E030E045E1BE0181EB91E10F941F0951
:10A17000182F882341F024EE31E147E1BE0181EB45
:10A1800091E10F941F09E091E211F091E31180E059
:10A190001995812FDF91CF911F910895CF93C82FEB
:10A1A0008FEF8C0F893060F48AE296E00E94336F63
:10A1B0008C2F0E949F6F809191060E94876F03C031
:10A1C0008C2F0E949F6F81E0CF910895CF93DF93F2
:10A1D0002FB7F89494E08902E0011124FE01EF54B6
:10A1E000F04F60817181828193812FBF0F94E919B3
:10A1F000CB56D84F288139814A815B810F94481A08
:10A20000DF91CF9108952FB7F894909105019B7F2E
:10A21000909305012FBF87FD96C0A3982FB7F894A0
:10A22000909105019460909305012FBF880F2FB77F
:10A23000F894909105019B7F909305012FBF87FDB6
:10A240008EC0A3982FB7F8949091050194609093D5
:10A2500005012FBF880F2FB7F894909105019B7FC0
:10A26000909305012FBF87FD78C0A3982FB7F8946E
:10A27000909105019460909305012FBF880F2FB72F
:10A28000F894909105019B7F909305012FBF87FD66
:10A2900062C0A3982FB7F8949091050194609093B1
:10A2A00005012FBF880F2FB7F894909105019B7F70
:10A2B000909305012FBF87FD4CC0A3982FB7F8944A
:10A2C000909105019460909305012FBF880F2FB7DF
:10A2D000F894909105019B7F909305012FBF87FD16
:10A2E00036C0A3982FB7F89490910501946090938D
:10A2F00005012FBF982F990F2FB7F8948091050172
:10A300008B7F809305012FBF97FD1FC0A3982FB7A8
:10A31000F894809105018460809305012FBF2FB7C9
:10A32000F894809105018B7F809305012FBF96FDE6
:10A3300018C0A3989FB7F89480910501846080931A
:10A3400005019FBF0895A39A69CFA39AE0CFA39A6E
:10A35000C9CFA39AB3CFA39A9DCFA39A87CFA39A2D
:10A3600071CFA39AE7CFFC0120E03EE2DB014C91E4
:10A37000403241F0283011F430833196DB014C91AA
:10A38000408331962F5F6F5F7F4F2B3079F71082BC
:10A390000895CF92DF92EF92FF92C0906806D0901E
:10A3A0006906E0906A06F0906B066091F20F70917A
:10A3B000F30F68507109882777FD8095982F0F94C7
:10A3C000E9199B01AC01C701B6010F94E31987FF9E
:10A3D0001DC020E030E040E050E4C701B6010F941A
:10A3E000161E0F945F1F7093E5066093E4060F94AA
:10A3F0001B0A605A75418F4F9F4F6093E60670931A
:10A40000E7068093E8069093E90608C01092E606F6
:10A410001092E7061092E8061092E906FF90EF907E
:10A42000DF90CF900895CF92DF92EF92FF92C0908D
:10A430006406D0906506E0906606F090670660912D
:10A44000F60F7091F70F65517109882777FD809598
:10A45000982F0F94E9199B01AC01C701B6010F9425
:10A46000E31987FF1DC020E030E040E251E4C7015E
:10A47000B6010F94161E0F945F1F7093EB06609346
:10A48000EA060F941B0A605C73468F4F9F4F6093E0
:10A49000EC067093ED068093EE069093EF0608C0ED
:10A4A0001092EC061092ED061092EE061092EF0656
:10A4B000FF90EF90DF90CF9008954F925F926F9250
:10A4C0007F928F929F92AF92BF92CF92DF92EF9244
:10A4D000FF920F931F93CF93DF932C0121E736E177
:10A4E00081E090E0F90145915491441655060CF035
:10A4F00062C0AC0141505109DA01AA0FBB1FAA0F7B
:10A50000BB1FA159B94EFD0165917491440F551FB0
:10A51000440F551F4359594EFA0165907490FC0140
:10A52000EE0FFF1FEE0FFF1FE159F94EA590B490FB
:10A53000FD0105911491F901C591D491FA0185901D
:10A540009490882777FD8095982F0F94E9196B01D7
:10A550007C01B20166197709882777FD8095982FCD
:10A560000F94E9192B013C01B501601B710B882781
:10A5700077FD8095982F0F94E9199B01AC01C301D9
:10A58000B2010F94481A2B013C01BE0168197909E8
:10A59000882777FD8095982F0F94E9199B01AC01CE
:10A5A000C301B2010F94F21E9B01AC01C701B601B9
:10A5B0000F94161E11C001962C5F3F4F8A339105F0
:10A5C00009F090CFE3E5F7E165917491882777FD75
:10A5D0008095982F0F94E919DF91CF911F910F91DA
:10A5E000FF90EF90DF90CF90BF90AF909F908F90B3
:10A5F0007F906F905F904F9008954F925F926F920F
:10A600007F928F929F92AF92BF92CF92DF92EF9202
:10A61000FF92CF93DF93CDB7DEB72C970FB6F894A8
:10A62000DEBF0FBECDBF8091680690916906A091F4
:10A630006A06B0916B0689839A83AB83BC83609171
:10A64000F20F7091F30F882777FD8095982F0F9464
:10A65000E91929813A814B815C810F94151E6B01A8
:10A660007C016093D2067093D3068093D4069093B6
:10A67000D5062091591030915A1040915B1050919D
:10A680005C100F94481A6D837E838F839887609344
:10A69000CE067093CF068093D0069093D10620917A
:10A6A000CA063091CB064091CC065091CD06C70129
:10A6B000B6010F94161E4B015C016093CA0670939D
:10A6C000CB068093CC069093CD0620915510309107
:10A6D000561040915710509158100F94481A69879E
:10A6E0007A878B879C876093C6067093C706809392
:10A6F000C8069093C90620ED3CEC4CE45DE3609104
:10A7000051107091521080915310909154100F94E9
:10A71000481A2B013C012091C2063091C30640919A
:10A72000C4065091C50669817A818B819C810F9402
:10A73000151E9B01AC01C301B2010F94481A2B01F5
:10A740003C0123E333E343E75FE36091BE0670918E
:10A75000BF068091C0069091C1060F94481A9B01D4
:10A76000AC01C301B2010F94161E2B013C01609392
:10A77000BE067093BF068093C0069093C106898180
:10A780009A81AB81BC818093C2069093C306A0934B
:10A79000C406B093C50629853A854B855C856D81D5
:10A7A0007E818F8198850F94161EA30192010F94CC
:10A7B000151E2B013C0120E030E04EE453E40F94E1
:10A7C0003C2020E030E0A9011816ACF4C701B60126
:10A7D0000F943C2018166CF5A7019601C501B40131
:10A7E0000F94151E6093CA067093CB068093CC0617
:10A7F0009093CD061EC0C301B2010F94E31987FFE9
:10A8000022C020E030E0A901C701B6010F94E3198E
:10A8100087FF16C0A7019601C501B4010F94151E4C
:10A820006093CA067093CB068093CC069093CD06B6
:10A8300007C0412C512C8EE4682E83E4782E03C08F
:10A84000412C512C3201C301B2012C960FB6F89461
:10A85000DEBF0FBECDBFDF91CF91FF90EF90DF90B5
:10A86000CF90BF90AF909F908F907F906F905F90B0
:10A870004F9008954F925F926F927F928F929F9226
:10A88000AF92BF92CF92DF92EF92FF920F931F93FE
:10A89000CF93DF9300D01F92CDB7DEB70091F60FB4
:10A8A0001091F70F8090640690906506A090660660
:10A8B000B0906706B801882777FD8095982F0F9490
:10A8C000E919A50194010F94151E6B017C01609399
:10A8D000BA067093BB068093BC069093BD0620ED2C
:10A8E0003CEC4CE45DE36091451070914610809122
:10A8F0004710909148100F94481A2B013C01209169
:10A90000B6063091B7064091B8065091B906C50118
:10A91000B4010F94151E9B01AC01C301B2010F9449
:10A92000481A2B013C0123E333E343E75FE36091E3
:10A93000B2067091B3068091B4069091B5060F945B
:10A94000481A9B01AC01C301B2010F94161E698322
:10A950007A838B839C836093B2067093B306809353
:10A96000B4069093B5068092B6069092B706A09270
:10A97000B806B092B90680917606882321F081E06E
:10A980008093B106B9C020E030E040E251E4C70155
:10A99000B6010F943C20181624F481E08093B10690
:10A9A000A4C020E030E040E251ECC701B6010F94B2
:10A9B000E31987FDE4CF012B11F38091B1068823C1
:10A9C00051F01092AD061092AE061092AF061092A2
:10A9D000B0061092B10620914D1030914E1040916A
:10A9E0004F1050915010C701B6010F94481A2B0117
:10A9F0003C016093A9067093AA068093AB069093DE
:10AA0000AC062091AD063091AE064091AF06509154
:10AA1000B006C701B6010F94161E4B015C0160938E
:10AA2000AD067093AE068093AF069093B00620916A
:10AA3000491030914A1040914B1050914C100F9496
:10AA4000481A9B01AC016093A5067093A6068093FB
:10AA5000A7069093A806C301B2010F94161E298180
:10AA60003A814B815C810F94151E2B013C0120E043
:10AA700030E04FE753E40F943C2020E030E0A901A0
:10AA80001816ACF4C701B6010F943C2018166CF5EB
:10AA9000A7019601C501B4010F94151E6093AD0680
:10AAA0007093AE068093AF069093B0061EC0C301AC
:10AAB000B2010F94E31987FF22C020E030E0A90122
:10AAC000C701B6010F94E31987FF16C0A7019601CD
:10AAD000C501B4010F94151E6093AD067093AE06C8
:10AAE0008093AF069093B00607C0412C512C9FE78E
:10AAF000692E93E4792E03C0412C512C3201C301FD
:10AB0000B2010F900F900F900F90DF91CF911F9196
:10AB10000F91FF90EF90DF90CF90BF90AF909F90FC
:10AB20008F907F906F905F904F900895609168062E
:10AB30007091690680916A0690916B0608954F9214
:10AB40005F926F927F928F929F92AF92BF92CF92BD
:10AB5000DF92EF92FF920F931F93CF93DF932C011D
:10AB60002BED33E181E090E0F901459154914416D9
:10AB700055060CF062C0AC0141505109DA01AA0F30
:10AB8000BB1FAA0FBB1FA752BC4EFD01659174915C
:10AB9000440F551F440F551F49525C4EFA016590F2
:10ABA0007490FC01EE0FFF1FEE0FFF1FE752FC4EEB
:10ABB000A590B490FD0105911491F901C591D4912E
:10ABC000FA0185909490882777FD8095982F0F94AF
:10ABD000E9196B017C01B20166197709882777FDB5
:10ABE0008095982F0F94E9192B013C01B501601B4A
:10ABF000710B882777FD8095982F0F94E9199B0199
:10AC0000AC01C301B2010F94481A2B013C01BE01F3
:10AC100068197909882777FD8095982F0F94E9198D
:10AC20009B01AC01C301B2010F94F21E9B01AC0168
:10AC3000C701B6010F94161E11C001962C5F3F4F3D
:10AC40008032910509F090CFE5E5F4E165917491CA
:10AC5000882777FD8095982F0F94E919DF91CF9180
:10AC60001F910F91FF90EF90DF90CF90BF90AF902A
:10AC70009F908F907F906F905F904F90089560911C
:10AC80006406709165068091660690916706089546
:10AC900067FD5CC0823021F128F4882349F08130BF
:10ACA00069F054C0833071F1843009F43DC04EC066
:10ACB000662311F0A19A8FC0A1988DC09FB766231B
:10ACC00029F0F89480910801806804C0F89480917C
:10ACD00008018F77809308019FBF47FF4CC07FC05A
:10ACE0009FB7662329F0F89480910801806404C01E
:10ACF000F894809108018F7B809308019FBF47FFE4
:10AD000040C06FC09FB7662329F0F8948091080176
:10AD1000886004C0F89480910801877F80930801BF
:10AD20009FBF47FF3EC05AC09FB7662329F0F894E3
:10AD300080910801826004C0F894809108018D7FA1
:10AD4000809308019FBF47FF39C04AC047FD49C0F3
:10AD50008230B9F028F4882341F0813061F0089501
:10AD60008330F9F0843051F10895442311F0A09A12
:10AD70000895A0980895442311F0A29A0895A298E6
:10AD800008959FB7442329F0F894809108018062C8
:10AD900004C0F894809108018F7D809308019FBFC3
:10ADA00008959FB7442329F0F894809108018061A9
:10ADB000F4CFF894809108018F7EEFCF9FB74423A2
:10ADC00029F0F894809108018460E7CFF89480918D
:10ADD00008018B7FE2CF47FFC8CF089508950895FB
:10ADE00008950895643079F028F4613041F06230BC
:10ADF00041F00895683051F0603141F0089540E02D
:10AE000003C040E004C041E060E002C041E061E016
:10AE10003FCF24E08202C0011124FC01EF54F04F27
:10AE20004081518162817381FC01EB55F84F408371
:10AE3000518362837383E091E40FF091E50F82897F
:10AE40009389A489B5898093C10F9093C20FA09371
:10AE5000C30FB093C40F089580E0B8D960930B0777
:10AE600070930C0780930D0790930E0781E0AED985
:10AE700060930F0770931007809311079093120748
:10AE800082E0A4D960931307709314078093150789
:10AE90009093160708958091E30F9FB780FF09C034
:10AEA000F89480910B018D7F80930B019FBF8FEFF2
:10AEB00008C0F89480910B01826080930B019FBFC2
:10AEC00081E080938A028091E30F9FB781FF09C0E0
:10AED000F89480910B01816080930B019FBF8FEFED
:10AEE00008C0F89480910B018E7F80930B019FBF67
:10AEF00081E080938B028091E30F9FB782FF09C0AE
:10AF0000F89480910B018B7F80930B019FBF8FEF93
:10AF100008C0F89480910B01846080930B019FBF5F
:10AF200081E080938C028091E30F9FB783FF09C07B
:10AF3000F89480910B01806480930B019FBF8FEF89
:10AF400008C0F89480910B018F7B80930B019FBF09
:10AF500081E080938D0208954F925F926F927F926D
:10AF6000AF92BF92CF92DF92EF92FF920F931F9317
:10AF7000CF93DF938C01EB01FC0147A050A461A4A7
:10AF800072A4AFA0B8A4C9A4DAA49501A601C30114
:10AF9000B2010F94E31987FF40C0A3019201C301DE
:10AFA000B2010F94481A2B013C01F80183A994A91E
:10AFB000A5A9B6A9BC01CD0190589B01AC010F9485
:10AFC000161EF80127A530A941A952A90F94481AC5
:10AFD0009B01AC01C301B2010F94151E0F94812097
:10AFE0007B018C019B01AC01B501C6010F94E319F3
:10AFF00087FF02C0750186019701A801B501C6014E
:10B000000F94E319882349F0A701B8014FA358A76B
:10B0100069A77AA7888181608883DF91CF911F918A
:10B020000F91FF90EF90DF90CF90BF90AF907F9007
:10B030006F905F904F9008958F929F92AF92BF92C2
:10B04000CF92DF92EF92FF920F931F93CF93DF93F4
:10B0500000D01F92CDB7DEB71DE6812E11E1912EF3
:10B060000EEFA02E00E1B02E08E311E1C12CD12C8F
:10B070007601C394F40161917191819191914F0195
:10B08000F50121913191419151915F0129833A83D9
:10B090004B835C830F94E71929813A814B815C8152
:10B0A0000F94481A0F945F1FF80161937193819375
:10B0B00091938F01C616D706E806F90610F46B01C6
:10B0C0007C01FDE78F16F1E19F06A1F66FEF7FEFA0
:10B0D000CB01A70196010F94B81D20931210309355
:10B0E000131040931410509315100F900F900F9061
:10B0F0000F90DF91CF911F910F91FF90EF90DF9014
:10B10000CF90BF90AF909F908F9008950F931F9313
:10B11000CF93DF93C8E2D3E00DE611E189910F945C
:10B12000B107882349F00F9443060F945F1FF8017D
:10B1300060837183828393830C5F1F4FF3E0CC3273
:10B14000DF0761F7DF91CF911F910F9175CF61E01C
:10B15000FC0180810D94E6098EBD0DB407FEFDCF84
:10B1600008958FEF8EBD0DB407FEFDCF8EB5089507
:10B170000F931F93CF93DF93EB010F941B0A8B0167
:10B18000F0DF8F3F49F00F941B0A601B710B6C17A7
:10B190007D07B0F380E001C081E0DF91CF911F9186
:10B1A0000F910895CF92DF92FF920F931F93CF9349
:10B1B000DF9300D01F92CDB7DEB76C01F62EFC01F5
:10B1C0008281982F906A96959CBD80FD06C091E083
:10B1D000863009F490E0892F01C080E08DBD60E0E9
:10B1E000F601808129833A834B835C830F94E609BF
:10B1F0006CE271E0C601BCDF8F2D8064ADDF08E139
:10B2000010E05C814B813A812981DA01C901002E6D
:10B2100004C0B695A795979587950A94D2F7298388
:10B220003A834B835C8398DF0850110929813A8166
:10B230004B815C81083FFFEF1F0739F7FF2029F0A2
:10B2400088E0F81621F08FEF03C085E901C087E898
:10B2500083DFECE0FE1201C084DF10E082DFF60144
:10B26000838387FF04C01F3F11F01F5FF7CF0F904C
:10B270000F900F900F90DF91CF911F910F91FF9042
:10B28000DF90CF9008959091C00095FFFCCF809300
:10B29000C6000895EF92FF921F93CF93DF931F9202
:10B2A000CDB7DEB7182FE5E6F6E184917F012FEFE9
:10B2B000E21AF20A882329F09983E5DFF7019981E0
:10B2C000F4CFE12FF92F84917F019FEFE91AF90A5A
:10B2D000882319F0D8DFF701F6CFECE4F6E184918A
:10B2E0007F01AFEFEA1AFA0A882319F0CCDFF701E1
:10B2F000F6CF0F90DF91CF911F91FF90EF900895BF
:10B30000CF93DF9383E50F941208882319F00F94ED
:10B31000330602C060E070E0EB01DD27C230D105EA
:10B32000A8F0E6E0F2E48491EF012196882319F079
:10B33000AADFFE01F8CFEAE2F6E18491EF0121965F
:10B34000882309F44DC09FDFFE01F7CF88E40F94F6
:10B3500012088823A9F00F943306683771053CF072
:10B36000633281E078072CF062E271E002C068E7A6
:10B3700070E0FE01EE0FFF1FEA5AFE4E71836083FC
:10B3800086E40F941208882399F00F9433066F3FD8
:10B39000710519F014F06FEF70E0FE01EE0FFF1F62
:10B3A000E25BFE4E77FF02C060E070E07183608375
:10B3B00082E40F941208882399F00F9433066530C5
:10B3C000710534F0683871052CF067E870E002C050
:10B3D00065E070E0CC0FDD1FCE5ADE4E79836883C6
:10B3E000DF91CF910895CF93DF93E2E3F5E184916C
:10B3F000EF012196882319F046DFFE01F8CFE4E241
:10B40000F5E18491EF012196882319F03CDFFE01DC
:10B41000F8CFEDE0F5E18491EF012196882319F052
:10B4200032DFFE01F8CFEDEFF4E18491EF012196D8
:10B43000882319F028DFFE01F8CFECEEF4E18491C7
:10B44000EF012196882319F01EDFFE01F8CFEBED06
:10B45000F4E18491EF012196882319F014DFFE01B5
:10B46000F8CFECECF4E18491EF012196882319F0F8
:10B470000ADFFE01F8CFE7EBF4E18491EF012196BA
:10B48000882319F000DFFE01F8CFE1EAF4E18491AE
:10B49000EF012196882319F0F6DEFE01F8CFECE8E3
:10B4A000F4E18491EF012196882319F0ECDEFE018E
:10B4B000F8CFEFE6F4E18491EF012196882319F0AB
:10B4C000E2DEFE01F8CFE7E5F4E18491EF01219699
:10B4D000882319F0D8DEFE01F8CFDF91CF910895CF
:10B4E0003FB7F8942091BA0A8091B90A821759F0AF
:10B4F000E22FF0E0E75CF54F808190E02F5F2F773F
:10B500002093BA0A02C08FEF9FEF3FBF0895CF93F9
:10B51000FC01C62F80818B33A1F0809133098430E8
:10B5200080F420915E1030E6239FC0011124BF01FA
:10B530008E54984F0F9456218C2F0F949C0781E0C6
:10B5400001C080E0CF9108958091A3069091A40658
:10B55000009731F04AE050E060E070E00D9423186D
:10B5600060E070E0CB01089583E50F94B107882374
:10B5700051F00F9443066093E6107093E7108093A8
:10B58000E8109093E91084E50F94B107882351F0F7
:10B590000F9443066093E2107093E3108093E410DD
:10B5A0009093E51082E40F94B107882349F0CCDF33
:10B5B00060935A1170935B1180935C1190935D11AD
:10B5C00088E50F94B107882351F00F9443066093E8
:10B5D0001B1170931C1180931D1190931E1189E50E
:10B5E0000F94B107882351F00F94430660931F1105
:10B5F0007093201180932111909322118AE50F946A
:10B60000B107882351F00F94430660932311709380
:10B610002411809325119093261185E40F94B1078E
:10B62000882351F00F9443066093271170932811DB
:10B630008093291190932A1108950F94330697FD52
:10B640000EC00F9433066F3F71058105910509F017
:10B650001CF40F94330601C06FEF862F089580E02D
:10B6600008958091A3069091A406892B39F0E5DF17
:10B6700091E0811101C090E0892F089581E0089543
:10B6800083E50F94B107882319F0EBDF80939407CB
:10B690000895CF93DF93C0912C14CC23C1F0C150F7
:10B6A000C0932C148FE1C89FE0011124CA50DD4ED5
:10B6B0008BE1FE013496ABEDB2E101900D928A95DB
:10B6C000E1F78A819B819093DA128093D9121092CC
:10B6D0008A1181E080938B1183E08093A802DF912F
:10B6E000CF9108955F988EBD00000DB407FEFDCF89
:10B6F0008EB56EBD00000DB407FEFDCF8EB55F9A0E
:10B700000895CF92DF92EF92FF920F931F93CF9302
:10B71000DF93EC010F941B0A0E811F812885398568
:10B72000011511052105310559F53C853323A9F192
:10B730002A8531503C8731E0320F3A874D853413EA
:10B7400001C01A86FE0134E0239FE00DF11D112493
:10B7500006851785208931890A831B832C833D83C5
:10B760006B017C01C00ED11EE11CF11CCE82DF8278
:10B77000E886F9868C819D81892B79F0769A0DC0B7
:10B780006B017C01C01AD10AE20AF30AF7FC05C07A
:10B7900076981E821F8218861986DF91CF911F919D
:10B7A0000F91FF90EF90DF90CF9008950F931F932C
:10B7B000CF93DF938C01EB01DC0113968C918823EE
:10B7C000C1F18250823028F48FE28883198281E0AF
:10B7D00031C0F801648575858685978540E00E94B3
:10B7E000D670882339F1D8015096EC91B0E2EB9FE6
:10B7F000F0011124E55AFB4F3097D9F090E020E09A
:10B800003EE24081403269F0283029F4DE01A90F80
:10B81000B11D3C939F5F4081DE01A90FB11D4C9388
:10B820009F5F2F5F31962B3061F7C90FD11D1882B2
:10B8300001C080E0DF91CF911F910F910895CF93C8
:10B84000DF938091EA11811107C081E08093EA11B2
:10B8500081EB91E10F942309C091B311D091B41100
:10B86000E091E211F091E31182E01995E091E2118B
:10B87000F091E31181E0199520E030E044E1BE0150
:10B8800081EB91E10F941F0924EE31E147E1BE0104
:10B8900081EB91E10F941F09E091E211F091E31126
:10B8A00080E0DF91CF9119941092F70F1092F60F6C
:10B8B00080E00E9413521092F30F1092F20F0E9438
:10B8C000C9510E9447771092F70F1092F60F80E04F
:10B8D0000E94135210920C109FB7F894E2E0F1E02E
:10B8E00080818F7B80839FBF1092F30F1092F20FA5
:10B8F00010920A10759808951092651110926411B3
:10B900001092671110926611CFDF0C9444A79091AA
:10B91000331280913412981731F0809134128F5F76
:10B920008F708093341208950F931F93CF93DF93FA
:10B93000EC01FC01E65AFF4F108213823497138208
:10B94000128280E293E091838083B5961082138205
:10B95000349713821282918380838E010A561F4F7F
:10B960009E0124533E4FF801B8016C5F7F4FAC013C
:10B97000CF01801B910B860F971FDC011C92139641
:10B980001C9213821282518340837F96E217F30741
:10B9900079F7CE0183539E4F29E1DC0111962C9358
:10B9A000119714961C920596DC0157961C9282966C
:10B9B000DC011C9213961C920497DC0113961C92D6
:10B9C0001E92129720E233E02D933C931982188245
:10B9D0001B821A828F549F4FDC011D921D921D9273
:10B9E0001C9213970496DC011D921D921D921C92CD
:10B9F00013971082FE01E15FFD4F108286E391E014
:10BA0000F8019C01119221503040E1F7FE01E3550D
:10BA1000FD4F81E08083E955F240118210820F943E
:10BA20001B0AC755DD4F68577C4E8F4F9F4F688369
:10BA300079838A839B83DF91CF911F910F91089522
:10BA40002F923F924F925F926F927F928F929F922E
:10BA5000AF92BF92CF92DF92EF92FF920F931F931C
:10BA6000CF93DF93CDB7DEB768970FB6F894DEBFFC
:10BA70000FBECDBF1C015B018A01DC01D7966D9121
:10BA80007D918D919C91DA970F94E7196B017C0160
:10BA9000F50120813181428153810F94481A0F941E
:10BAA000DC1E0F945F1F69877A878B879C87D8017C
:10BAB0002D913D914D915C91C701B6010F94481AAB
:10BAC0000F94DC1E0F945F1F6D877E878F87988B86
:10BAD00029853A854B855C85283731054105510517
:10BAE00040F488E790E0A0E0B0E089879A87AB87D0
:10BAF000BC872D853E854F855889283731054105FE
:10BB0000510540F488E790E0A0E0B0E08D879E8783
:10BB1000AF87B88B91012D5B3F4FD9018D919D91DE
:10BB20000D90BC91A02D8D839E83AF83B887BC01FF
:10BB3000CD010F94E91969837A838B839C8369858E
:10BB40007A858B859C850F94E719698B7A8B8B8B13
:10BB50009C8B20E030E0A90169817A818B819C81F6
:10BB60000F94E319882339F1A7019601C701B601A3
:10BB70000F94481A4B015C0129893A894B895C89E9
:10BB8000CA01B9010F94481A9B01AC01C501B40167
:10BB90000F94151E4B015C0129813A814B815C8118
:10BBA000CA01B9010F94161E9B01AC01C501B40175
:10BBB0000F94F21E03C060E070E0CB010F94DC1E16
:10BBC0000F945A1F2B013C016D817E818F819885D6
:10BBD00090958095709561957F4F8F4F9F4F0F94F3
:10BBE000E9194B015C016D857E858F8598890F94DD
:10BBF000E7196D837E838F83988720E030E0A90169
:10BC0000C501B4010F94E319882349F12D813E81C8
:10BC10004F815885CA01B9010F94481A6D8B7E8BEC
:10BC20008F8B988FA7019601C701B6010F94481A10
:10BC30009B01AC016D897E898F89988D0F94151EAB
:10BC40006B017C01A5019401C501B4010F94161E7E
:10BC50009B01AC01C701B6010F94F21E03C060E066
:10BC600070E0CB010F948B1FF10182889388A48828
:10BC7000B58875016401C418D508E608F7080F9463
:10BC80005A1FC61AD70AE80AF90AF7FE6BC020E065
:10BC900030E0A90169817A818B819C810F94E3193D
:10BCA000882309F447C029813A814B815C81CA010C
:10BCB000B9010F94161E6B017C01C501B4010F94EC
:10BCC000E7199B01AC01C701B6010F94481A6B013B
:10BCD0007C0129893A894B895C89CA01B9010F9491
:10BCE000481A9B01AC01C701B6010F94151E6B01E8
:10BCF0007C012D813E814F815885CA01B9010F9485
:10BD0000481A9B01AC01C701B6010F94161E6B01C6
:10BD10007C0120E030E040E850E469817A818B8149
:10BD20009C810F94481A9B01AC01C701B6010F9486
:10BD3000F21E03C060E070E0CB010F94DC1E0F9494
:10BD40005A1F2B013C0197FF03C0412C512C32019B
:10BD5000481459046A047B0410F024013501C12CF5
:10BD6000D12C76018FB7F894D1019C9193FD22C01C
:10BD7000F101468A578A608E718EC40CD51CE61C70
:10BD8000F71C5A96CD92DD92ED92FC925D97298533
:10BD90003A854B855C85DB962D933D934D935C9363
:10BDA000DE97FF962D853E854F8558892083318308
:10BDB000428353838FBF68960FB6F894DEBF0FBEE1
:10BDC000CDBFDF91CF911F910F91FF90EF90DF904A
:10BDD000CF90BF90AF909F908F907F906F905F902B
:10BDE0004F903F902F900895CF93DF9383E50F946A
:10BDF0001208882321F00F943306EB0102C0C0E043
:10BE0000D0E080E50F941208882321F00F943306C8
:10BE1000CB0102C080E090E0BE01DF91CF9162CC07
:10BE2000CF93DF9300D01F921F92CDB7DEB795E07E
:10BE3000E9EAF2E0DE01119601900D929A95E1F7A0
:10BE4000E1E0F0E0EC0FFD1FE80FF11D808190E0D4
:10BE50000F900F900F900F900F90DF91CF9142CCE9
:10BE60001F93CF93DF93C8E2D3E010E089910F9442
:10BE7000B107882321F00F943306812FD1DF1F5F94
:10BE80001430A1F782E40F94B107882321F00F94B6
:10BE9000330684E0C5DF83E50F94B107882341F0C2
:10BEA000C0E00F9433068C2FBBDFCF5FC530C9F7DE
:10BEB000DF91CF911F9108958F929F92AF92BF9281
:10BEC000CF92DF92EF92FF92CF93C82FC09058028B
:10BED000D0905902E0905A02F0905B02A7019601BF
:10BEE000C701B6010F94C2208090FE069090FF0615
:10BEF000A0900007B0900107811129C0C11127C08F
:10BF000080916F06882319F1A7019601C501B4013C
:10BF10000F94151E209106113091071140910811C0
:10BF2000509109110F94481A0F944720719561950B
:10BF3000710980917007882351F08091F00F9091E2
:10BF4000F10F860F971F9093F10F8093F00F80925F
:10BF5000580290925902A0925A02B0925B02CF917D
:10BF6000FF90EF90DF90CF90BF90AF909F908F9019
:10BF70000895CF92DF92EF92FF92E1E4F2E4849190
:10BF80007F019FEFE91AF90A882319F07CD9F7019C
:10BF9000F6CFE7EFF9E184917F019FEFE91AF90A03
:10BFA000882319F070D9F701F6CF8AE50F94B1070D
:10BFB0008823C1F10F9443066B017C0120E030E03F
:10BFC00040E050EC0F943C2087FD20C020E030E0A2
:10BFD00040EA50E4C701B6010F94E3191816B4F013
:10BFE000C092FE06D092FF06E0920007F092010791
:10BFF00080E062DF6091FE067091FF06809100078D
:10C000009091010742E00E941F4D18C0E2EEF9E155
:10C0100084917F019FEFE91AF90A882379F033D9D7
:10C02000F701F6CF4091FE065091FF0660910007A0
:10C03000709101078FED99E10E946ABD8AE0FF903F
:10C04000EF90DF90CF901FC9AF92BF92CF92DF9257
:10C05000EF92FF920F931F93CF93C82F882319F06D
:10C06000E7ECF9E10BC0E1E4F2E484918F010F5FAA
:10C070001F4F8823A9F307D9F801F7CF84918F01C7
:10C080000F5F1F4F882319F0FED8F801F7CFCC239C
:10C0900019F0EAEAF9E10BC0E1E4F2E484918F01DE
:10C0A0000F5F1F4F8823A9F3EED8F801F7CF8491D3
:10C0B0008F010F5F1F4F882319F0E5D8F801F7CFE4
:10C0C0008AE0E1D8C11129C0E1E4F2E484918F0152
:10C0D0000F5F1F4F882319F0D6D8F801F7CFE7E993
:10C0E000F9E184918F010F5F1F4F882319F0CBD89E
:10C0F000F801F7CF80914D11882319F08AE0C3D859
:10C10000BCC3ECE8F9E184918F010F5F1F4F8823D6
:10C1100009F4B3C3B8D8F801F6CF40914911509152
:10C120004A1160914B1170914C1183E899E10E9482
:10C130006ABD8AE0A8D880914D11811119C0CC2325
:10C1400019F0E8E7F9E10BC0E1E4F2E484918F0132
:10C150000F5F1F4F8823A9F396D8F801F7CF84917A
:10C160008F010F5F1F4F882319F08DD8F801F7CF8B
:10C17000C11121C0E1E4F2E484918F010F5F1F4FF0
:10C18000882319F080D8F801F7CFE7E6F9E1849128
:10C190008F010F5F1F4F882319F075D8F801F7CF73
:10C1A000E1E4F2E484918F010F5F1F4F882319F0BF
:10C1B0006AD8F801F7CF4091FE105091FF106091BE
:10C1C0000011709101118FE599E10E946ABD4091C3
:10C1D00002115091031160910411709105118CE5C9
:10C1E00099E10E946ABD409106115091071160913A
:10C1F00008117091091189E599E10E946ABD409189
:10C200000A1150910B1160910C1170910D1186E57E
:10C2100099E10E946ABD8AE036D8C11121C0E1E4EB
:10C22000F2E484918F010F5F1F4F882319F02BD800
:10C23000F801F7CFE8E3F9E184918F010F5F1F4F19
:10C24000882319F020D8F801F7CFE1E4F2E48491D3
:10C250008F010F5F1F4F882319F015D8F801F7CF12
:10C260004091EA105091EB106091EC107091ED103C
:10C270008FE299E10E946ABD4091EE105091EF105B
:10C280006091F0107091F1108CE299E10E946ABD0A
:10C290004091F2105091F3106091F4107091F510EC
:10C2A00089E299E10E946ABD4091F6105091F71021
:10C2B0006091F8107091F91086E299E10E946ABDD0
:10C2C0008AE00E944359C11124C0E1E4F2E4849160
:10C2D0008F010F5F1F4F882321F00E944359F801FF
:10C2E000F6CFE4E0F9E184918F010F5F1F4F8823BF
:10C2F00021F00E944359F801F6CFE1E4F2E4849181
:10C300008F010F5F1F4F882321F00E944359F801CE
:10C31000F6CF40916D1150916E1160916F11709137
:10C3200070118BEF98E10E9466C14091711150919C
:10C330007211609173117091741188EF98E10E94ED
:10C3400066C140917511509176116091771170918D
:10C35000781185EF98E10E9466C140917911509162
:10C360007A1160917B1170917C1182EF98E10E94AB
:10C3700066C18AE00E944359C11124C0E1E4F2E49D
:10C3800084918F010F5F1F4F882321F00E94435932
:10C39000F801F6CFE8EAF8E184918F010F5F1F4FB3
:10C3A000882321F00E944359F801F6CFE1E4F2E43A
:10C3B00084918F010F5F1F4F882321F00E94435902
:10C3C000F801F6CF40918511509186116091871147
:10C3D000709188118FE998E10E946ABD40918111A6
:10C3E0005091821160918311709184118CE998E1D0
:10C3F0000E946ABD40917D1150917E1160917F1124
:10C400007091801189E998E10E946ABD8AE00E94DA
:10C410004359C11124C0E1E4F2E484918F010F5F1C
:10C420001F4F882321F00E944359F801F6CFE5E21F
:10C43000F8E184918F010F5F1F4F882321F00E9444
:10C440004359F801F6CFE1E4F2E484918F010F5FE4
:10C450001F4F882321F00E944359F801F6CF4091E5
:10C46000E6105091E7106091E8107091E9108CE1AE
:10C4700098E10E946ABD4091E2105091E3106091F2
:10C48000E4107091E51089E198E10E946ABD409145
:10C490005A1150915B1160915C1170915D1186E1B0
:10C4A00098E10E9466C140911B1150911C1160914E
:10C4B0001D1170911E1183E198E10E946ABD4091A7
:10C4C0001F1150912011609121117091221180E172
:10C4D00098E10E946ABD409123115091241160910E
:10C4E0002511709126118DE098E10E946ABD40915E
:10C4F0002711509128116091291170912A118AE019
:10C5000098E10E946ABD8AE00E944359C11124C08B
:10C51000E1E4F2E484918F010F5F1F4F882321F043
:10C520000E944359F801F6CFECEFF7E184918F01B7
:10C530000F5F1F4F882321F00E944359F801F6CF67
:10C54000E1E4F2E484918F010F5F1F4F882321F013
:10C550000E944359F801F6CF409174075091750736
:10C56000609176077091770783EF97E10E946ABD2B
:10C57000409178075091790760917A0770917B0715
:10C5800080EF97E10E946ABD40917C0750917D0742
:10C5900060917E0770917F078DEE97E10E946ABDE2
:10C5A0008AE00E944359C11124C0E1E4F2E484917D
:10C5B0008F010F5F1F4F882321F00E944359F8011C
:10C5C000F6CFE9EDF7E184918F010F5F1F4F8823CC
:10C5D00021F00E944359F801F6CFE1E4F2E484919E
:10C5E0008F010F5F1F4F882321F00E944359F801EC
:10C5F000F6CF60916F0670E080ED97E10E94414FA9
:10C600008AE00E944359CC2379F086E5A82E81E187
:10C61000B82E92E5C92E91E1D92E2EE4E22E21E129
:10C62000F22E00E010E024C0E1E4F2E484918F01F6
:10C630000F5F1F4F882321F00E944359F801F6CF66
:10C64000E3EBF7E184918F010F5F1F4F882321F007
:10C650000E944359F801F6CFE1E4F2E484918F019E
:10C660000F5F1F4F882389F20E944359F801F6CFCC
:10C67000B8018AEA97E10E94414FF50161917191F9
:10C680005F0187EA97E10E94414FF6016191719144
:10C690006F0184EA97E10E94414FF7016191719126
:10C6A0007F0181EA97E10E94414F8AE00E9443594D
:10C6B0000F5F1F4F02301105D9F6C11124C0E1E40C
:10C6C000F2E484918F010F5F1F4F882321F00E94B5
:10C6D0004359F801F6CFE2E9F7E184918F010F5F4A
:10C6E0001F4F882321F00E944359F801F6CFE1E45F
:10C6F000F2E484918F010F5F1F4F882321F00E9485
:10C700004359F801F6CF40914D1050914E10609171
:10C710004F107091501089E897E10E946ABD2CEA91
:10C7200035EC47E25EE36091491070914A108091C8
:10C730004B1090914C100F94F21EAB01BC0186E897
:10C7400097E10E944DBD2CEA35EC47E25EE3609133
:10C7500045107091461080914710909148100F94A9
:10C76000481AAB01BC0183E897E10E944DBD8AE005
:10C770000E944359C1110CC0E1E4F2E484918F019D
:10C780000F5F1F4F882321F00E944359F801F6CF15
:10C790004091591050915A1060915B1070915C104B
:10C7A0008AE797E10E946ABD2CEA35EC47E25EE336
:10C7B00060915510709156108091571090915810BB
:10C7C0000F94F21EAB01BC0187E797E10E944DBDBB
:10C7D0002CEA35EC47E25EE3609151107091521003
:10C7E00080915310909154100F94481AAB01BC01E2
:10C7F00084E797E10E944DBD8AE00E944359C11130
:10C8000024C0E1E4F2E484918F010F5F1F4F88237D
:10C8100021F00E944359F801F6CFEEE5F7E184914B
:10C820008F010F5F1F4F882321F00E944359F801A9
:10C83000F6CFE1E4F2E484918F010F5F1F4F88236C
:10C8400021F00E944359F801F6CF4091FE06509125
:10C85000FF06609100077091010785E597E10E944E
:10C860006ABD8AE0CF911F910F91FF90EF90DF900A
:10C87000CF90BF90AF900C944359E1E4F2E48491DF
:10C880008F010F5F1F4F882309F447CC0E94435943
:10C89000F801F5CF83E50F94B107882319F00E94C2
:10C8A000315B01C081E091E08927CECBCF92DF924E
:10C8B000EF92FF921F93CF93DF9300D01F92CDB7DB
:10C8C000DEB780918D1190918E11A0918F11B09152
:10C8D0009011B7FF08C010928D1110928E11109216
:10C8E0008F111092901180910F1190911011A091C1
:10C8F0001111B091121140918D1150918E116091D2
:10C900008F117091901184179507A607B70744F40B
:10C9100080938D1190938E11A0938F11B0939011ED
:10C920008091A802882359F160918D1170918E1128
:10C9300080918F1190919011C0901311D09014118B
:10C94000E0901511F09016116C0D7D1D8E1D9F1D30
:10C950000F94E71920E030E048EC52E40F94481AB5
:10C9600069837A838B839C83CE0101960E94229DEA
:10C97000BC018091191190911A110E94A0A8809178
:10C9800089111091FB10811106C01123C1F1809112
:10C99000A8028823A1F160918D1170918E11809170
:10C9A0008F1190919011C0901311D0901411E090BC
:10C9B0001511F09016116C0D7D1D8E1D9F1D0F948D
:10C9C000E71920E030E048EC52E40F94481A0F9445
:10C9D0005F1FE0911711F0911811309721F06083DB
:10C9E000718382839383112329F0E091FC10F091ED
:10C9F000FD1019958091891181110E944AA780919B
:10CA00008911882329F0E091FC10F091FD1019950F
:10CA10000F900F900F900F90DF91CF911F91FF908B
:10CA2000EF90DF90CF900895CF92DF92EF92FF9238
:10CA30001F93CF93DF9300D01F92CDB7DEB78091C5
:10CA40008D1190918E11A0918F11B0919011B7FF1F
:10CA500008C010928D1110928E1110928F111092A9
:10CA6000901180910F1190911011A0911111B0911E
:10CA7000121140918D1150918E1160918F11709112
:10CA8000901184179507A607B70744F480938D117A
:10CA900090938E11A0938F11B09390118091A80262
:10CAA000882359F160918D1170918E1180918F11B1
:10CAB00090919011C0901311D0901411E090151125
:10CAC000F09016116C0D7D1D8E1D9F1D0F94E919A0
:10CAD00020E030E048EC52E40F94481A69837A83EE
:10CAE0008B839C83CE0101960E94229DBC01809184
:10CAF000191190911A110E94A0A88091891110918A
:10CB0000FB10811106C01123B1F18091A802882386
:10CB100091F160918D1170918E1180918F11909192
:10CB20009011C0901311D0901411E0901511F09055
:10CB300016116C0D7D1D8E1D9F1D0F94E91920E0AF
:10CB400030E048EC52E40F94481AE0911711F0914C
:10CB50001811309721F060837183828393831123AE
:10CB600029F0E091FC10F091FD1019958091891148
:10CB700081110E944AA70F900F900F900F90DF91A4
:10CB8000CF911F91FF90EF90DF90CF900895CF92BB
:10CB9000DF92EF92FF921F93CF93DF9300D01F920B
:10CBA000CDB7DEB780918D1190918E11A0918F112C
:10CBB000B0919011B7FF08C010928D1110928E1194
:10CBC00010928F111092901180910F11909110116D
:10CBD000A0911111B091121140918D1150918E11AF
:10CBE00060918F117091901184179507A607B70770
:10CBF00044F480938D1190938E11A0938F11B09374
:10CC000090118091A802882359F160918D11709143
:10CC10008E1180918F1190919011C0901311D0902E
:10CC20001411E0901511F09016116C0D7D1D8E1DE4
:10CC30009F1D0F94E9192AE037ED43E25CE30F945E
:10CC4000481A69837A838B839C83CE0101960E9464
:10CC5000EC9BBC018091191190911A110E94A0A81F
:10CC6000809189111091FB10811106C01123B1F13F
:10CC70008091A802882391F160918D1170918E119D
:10CC800080918F1190919011C0901311D090141138
:10CC9000E0901511F09016116C0D7D1D8E1D9F1DDD
:10CCA0000F94E9192AE037ED43E25CE30F94481A48
:10CCB000E0911711F0911811309721F06083718382
:10CCC00082839383112329F0E091FC10F091FD10F1
:10CCD00019958091891181110E944AA7809189112B
:10CCE000882329F0E091FC10F091FD1019950F9028
:10CCF0000F900F900F90DF91CF911F91FF90EF90C9
:10CD0000DF90CF900895CF92DF92EF92FF921F9322
:10CD1000CF93DF9300D01F92CDB7DEB780918D11F6
:10CD200090918E11A0918F11B0919011B7FF08C012
:10CD300010928D1110928E1110928F1110929011ED
:10CD400080910F1190911011A0911111B0911211B9
:10CD500040918D1150918E1160918F1170919011B1
:10CD600084179507A607B70744F480938D11909315
:10CD70008E11A0938F11B09390118091A8028823F7
:10CD800059F160918D1170918E1180918F11909158
:10CD90009011C0901311D0901411E0901511F090E3
:10CDA00016116C0D7D1D8E1D9F1D0F94E9192AE033
:10CDB00037ED43E25CE30F94481A69837A838B83EF
:10CDC0009C83CE0101960E94A19CBC018091191107
:10CDD00090911A110E94A0A8809189111091FB10C6
:10CDE000811106C01123B1F18091A802882391F12D
:10CDF00060918D1170918E1180918F119091901191
:10CE0000C0901311D0901411E0901511F0901611EC
:10CE10006C0D7D1D8E1D9F1D0F94E9192AE037EDC5
:10CE200043E25CE30F94481AE0911711F091181156
:10CE3000309721F06083718382839383112329F0DB
:10CE4000E091FC10F091FD101995809189118111EC
:10CE50000E944AA70F900F900F900F90DF91CF91F3
:10CE60001F91FF90EF90DF90CF9008950F931F9345
:10CE7000CF9380918D1190918E11A0918F11B091CF
:10CE80009011B7FF08C010928D1110928E11109260
:10CE90008F111092901180910F1190911011A0910B
:10CEA0001111B091121140918D1150918E1160911C
:10CEB0008F117091901184179507A607B70744F456
:10CEC00080938D1190938E11A0938F11B093901138
:10CED0008091A802882311F160918D1170918E11BB
:10CEE00080918F1190919011009113111091141154
:10CEF0002091151130911611600F711F821F931F21
:10CF00000F94E9190F945A1FCB010E94759EBC0122
:10CF10008091191190911A110E94A0A880918911F5
:10CF2000C091FB10811106C0CC2381F18091A80231
:10CF3000882361F160918D1170918E1180918F1114
:10CF400090919011009113111091141120911511CD
:10CF500030911611600F711F821F931F0F94E919F2
:10CF6000E0911711F0911811309721F060837183CF
:10CF700082839383CC2329F0E091FC10F091FD1083
:10CF800019958091891181110E944AA78091891178
:10CF9000CF911F910F91089569DF882329F0E091C7
:10CFA000FC10F091FD101994089560CF0E942BA9F8
:10CFB000882329F0E091FC10F091FD101994089558
:10CFC0000C942BA9EC01E6E0F2E484918F010F5F51
:10CFD0001F4F882321F00E944359F801F6CFEDE15D
:10CFE000FAE184918F010F5F1F4F882321F00E9487
:10CFF0004359F801F6CF0E94545C0F947A060E94C0
:10D0000007AD61E0CE010E942BA40E9444A70E94BC
:10D010001F5C84E07CD78091B21186958695109232
:10D02000E8118093E9110E941D708091B2118695DC
:10D030008695880F1092E8118093E9118EE09AE1AD
:10D040009BD78091B21186958695982F990F980F4E
:10D050001092E8119093E91181E09AE18DD70E9436
:10D0600094508111D6CF2FEF8BE49DE12150804069
:10D070009040E1F700C00000F8942FEF84E39CE0BB
:10D08000215080409040E1F700C000000E94545CB5
:10D09000A895FECF6F927F928F929F92AF92BF9290
:10D0A000DF92EF92FF920F931F93CF93DF93CDB751
:10D0B000DEB7AD970FB6F894DEBF0FBECDBF7C01D3
:10D0C000D62E80916312882309F4F7C180915714FA
:10D0D000882309F49DC0442309F4C4C180916F14CE
:10D0E000882321F1E6E0F2E484918F010F5F1F4F66
:10D0F000882321F00E944359F801F6CFE0EAFBE1D2
:10D1000084918F010F5F1F4F882321F00E944359A4
:10D11000F801F6CF61E070E080E090E00E94044DFD
:10D120008AE00E94435987E99BE14CDF8FE28093BC
:10D130007414B12C21E005E714E19FE1A92E809140
:10D140002C14B816B8F4AB9CC0011124B801865059
:10D150009D4E2DA70E94D65BC8012DA58C0101967E
:10D16000F8013081332321F02D3810F42F5FF6CFF2
:10D17000B394E5CF27FD06C0B80184E594E10E9491
:10D18000D65B02C0F8011082E1E4F2E484918F01E1
:10D190000F5F1F4F882321F00E944359F801F6CFFB
:10D1A000B7018EE79BE10E94A49B60916F14FDE89C
:10D1B0006F9FB00111246C587B4E83E79BE10E9466
:10D1C000A49B40910515509106156091071570912B
:10D1D00008158DE69BE10E9466C18AE00E944359D2
:10D1E00080916F1494E0899FF0011124E059FB4E67
:10D1F000409105155091061560910715709108151D
:10D2000040835183628373838F5F80936F140DC05B
:10D2100010926F1482E0B82E27C1B70180E69BE11F
:10D220000E94A49B8AE00E9443590E9430901D8274
:10D2300018861C821B8280E293E09A83898386EBA6
:10D2400092E19093D6128093D512F70180818F32AC
:10D2500009F06DC087010F5F1F4FCE0101963C01A1
:10D260000115110509F469C06FE270E0C8010F945F
:10D270004B215C01009709F461C00817190708F0F9
:10D280005DC04C01801A910AA401B801CE018096BC
:10D290000F946B21E0E2F0E0EC0FFD1FE80DF91DAB
:10D2A00010828E01005E1F4FF80181918F0188234B
:10D2B00019F00E944359F8CF8AE00E9443596091C7
:10D2C000D5127091D6126115710519F06C5F7F4F00
:10D2D00002C060E070E021E0AE01405E5F4FCE0131
:10D2E00005960E942EAD81111AC0ECE4FBE18491F9
:10D2F0008F010F5F1F4F811104C08E01005E1F4F11
:10D3000004C00E944359F801F2CFF80181918F01C6
:10D31000882319F00E944359F8CF8EE28CC0709296
:10D32000D6126092D51285010F5F1F4F99CF87EDFE
:10D3300092E19093D6128093D51287016091D51215
:10D340007091D612DD2009F45DC06115710519F0E8
:10D350006C5F7F4F02C060E070E021E0A80184E5CF
:10D3600094E10E942EAD882309F448C08091651491
:10D3700090916614A0916714B09168148093011580
:10D3800090930215A0930315B0930415B8018EE392
:10D390009BE10E94A49B4091011550910215609160
:10D3A00003157091041586E39BE10E9466C18AE033
:10D3B0000E944359109205151092061510920715F8
:10D3C00010920815E7E2FBE184917F019FEFE91AD3
:10D3D000F90A882321F00E944359F701F5CFB801DB
:10D3E00080E090E00E94E8AF80917212811102C04B
:10D3F000C80102C082E792E160E02DC0B80183E17C
:10D400009BE113C06115710519F06C5F7F4F02C07D
:10D4100060E070E026E5A80184E594E10E942EAD6D
:10D4200081110CC0B8018FEF9AE10E94A49B8EE29B
:10D430000E9443598AE00E9443590FC081E08093C3
:10D440006012B7018DEE9AE10E94A49B8AE00E94CF
:10D45000435960E0C8010E941BA4CE0101960E94BE
:10D4600087912BC0BB24B394E1E4F2E484918F0153
:10D470000F5F1F4F882321F00E944359F801F6CF18
:10D48000E8E6FBE184918F010F5F1F4F882321F0B5
:10D490000E944359F801F6CFE1E0BE1203C006E353
:10D4A00013E002C000E313E0F80181918F018823AB
:10D4B00009F4B3CE0E944359F7CFAD960FB6F89456
:10D4C000DEBF0FBECDBFDF91CF911F910F91FF90B7
:10D4D000EF90DF90BF90AF909F908F907F906F9074
:10D4E000089560E08091F80F9091F90F0E949F5588
:10D4F0006093640670936506809366069093670652
:10D500008091F40F9091F50F0E945D526093680630
:10D510007093690680936A0690936B06A8958FB7FF
:10D52000F8941092FA0F8FBF0895CF92DF92FF9276
:10D530000F931F93CF93DF931F921F92CDB7DEB748
:10D54000F82E6A0180915702882309F441C0E6E071
:10D55000F2E484918F010F5F1F4F882341F06983AC
:10D560007A830E944359F80169817A81F2CFFB01E5
:10D5700084918F010F5F1F4F882321F00E94435930
:10D58000F801F6CFE2E4FAE184918F010F5F1F4FBB
:10D59000882321F00E944359F801F6CFF7FC0CC014
:10D5A0006F2D772767FD7095872F972F0E94044D69
:10D5B0008AE00E9443590CC0EDE3FAE184918F01A7
:10D5C0000F5F1F4F882321F00E944359F801F6CFC7
:10D5D0008091D606811107C01092570281E0809396
:10D5E000D606C601EFDC0F900F90DF91CF911F910F
:10D5F0000F91FF90DF90CF900C94545C2F923F924C
:10D600004F925F926F927F928F929F92AF92BF9252
:10D61000CF92DF92EF92FF920F931F93CF93DF93FE
:10D6200000D01F92CDB7DEB74C011B0129833A838E
:10D630004B835C8327013801D7FE12C08091880696
:10D64000882309F4A7C0F40110821092DB0610921F
:10D65000DC061092DD061092DE0601E010E015C037
:10D66000F601EA58F94F8081882309F4BEC0F4011D
:10D670001082F601EE0FFF1FEE0FFF1FE952F94F68
:10D6800010821182128213828601F401808182301D
:10D69000E1F0833009F455C0813009F0A8C0F801E9
:10D6A000EE0FFF1FEE0FFF1FE952F94F208131816E
:10D6B0004281538169817A818B819C810F94E31926
:10D6C00087FD95C082E0F4018083000F111F000FD9
:10D6D000111F0952194FB501882777FD8095982FA2
:10D6E0000F94E9199B01AC01F8016081718182817D
:10D6F00093810F94151E9B01AC0169817A818B8106
:10D700009C810F943C2087FD0CC00F941B0A685627
:10D71000754C8F4F9F4FF101608371838283938398
:10D7200066C00F941B0AF1010081118122813381AF
:10D73000601B710B820B930B97FD59C083E0F401C2
:10D740008083FFEFCF16DF0631F0C114D10431F42E
:10D7500047E95AE105C040E65AE102C044E85AE10F
:10D7600064E77AE18C2D0F900F900F900F90DF916E
:10D77000CF911F910F91FF90EF90DF90CF90BF90CE
:10D78000AF909F908F907F906F905F904F903F9061
:10D790002F90CBCE01E010E07801EE0CFF1CEE0CD8
:10D7A000FF1CC7018952994F7C01A3019201FC0122
:10D7B00060817181828193810F94E319882309F438
:10D7C00064CFF7014082518262827382FF24F39416
:10D7D00020E030E0A901C301B2010F943C201816EB
:10D7E0000CF0F12CF401F08250CF8601D5CF0F90D0
:10D7F0000F900F900F90DF91CF911F910F91FF909D
:10D80000EF90DF90CF90BF90AF909F908F907F90E0
:10D810006F905F904F903F902F9008958F3F29F029
:10D82000811106C048E95CE405C045E65CE402C03D
:10D8300048E85CE466E77CE478CE8F3F29F081110C
:10D8400006C04BED5CE405C048EA5CE402C04BEC6A
:10D850005CE469EB7CE469CE4F925F926F927F92B9
:10D86000AF92BF92CF92DF92EF92FF920F931F93EE
:10D87000CF93DF9300D01F92CDB7DEB78091FA0F20
:10D88000811113C00F900F900F900F90DF91CF91E7
:10D890001F910F91FF90EF90DF90CF90BF90AF90CE
:10D8A0007F906F905F904F9008951BDE0F941B0A3E
:10D8B00069837A838B839C8380915C0290915D0263
:10D8C000181619060CF026C1019790935D028093FB
:10D8D0005C02409064065090650660906606709009
:10D8E000670680917606811119C080917206909129
:10D8F0007306A0917406B09175060097A105B10555
:10D9000069F029813A814B815C81281B390B4A0BD4
:10D910005B0B57FD03C081E0809376066091F60FA4
:10D920007091F70F882777FD8095982F0F94E9194C
:10D930001EE1A12EB12CC12CD12C7B018C01A301A5
:10D94000920161EF76E080EF96E058DE4090640649
:10D9500050906506609066067090670660916B0750
:10D9600070916C07882777FD8095982F0F94E9199F
:10D970009B01AC01C301B2010F943C201816D4F4F2
:10D980006091680270916902882777FD8095982FD1
:10D990000F94E9199B01AC01C301B2010F94E31983
:10D9A00087FF08C080E00E943A540F945A1F759573
:10D9B000679501C060E060930C108091EC06909137
:10D9C000ED06A091EE06B091EF060097A105B10516
:10D9D00021F129813A814B815C81281B390B4A0B4B
:10D9E0005B0B57FD1AC00E943F562B013C01609112
:10D9F000EA067091EB0680E090E00F94E7199B0136
:10DA0000AC01C301B2010F94E31987FFA5C04BED30
:10DA10005AE16CEC7AE180E088DD8091E606909135
:10DA2000E706A091E806B091E9060097A105B105C7
:10DA300021F129813A814B815C81281B390B4A0BEA
:10DA40005B0B57FD1AC00E9496552B013C0160915B
:10DA5000E4067091E50680E090E00F94E7199B01E1
:10DA6000AC01C301B2010F94E31987FF72C04AEA07
:10DA70005AE16DEB7AE18FEF58DD6091F20F709112
:10DA8000F30F882777FD8095982F0F94E91920913F
:10DA900068063091690640916A0650916B06FAE07B
:10DAA000AF2EB12CCC24CA94DC2C7B018C016FED01
:10DAB00076E083EE96E0A2DD80918806811127C092
:10DAC000409068065090690660906A0670906B06F8
:10DAD00020E030E040EA50E4C301B2010F943C2062
:10DAE00087FF04C060E060930A10CCCE20E030E0F5
:10DAF00046E153E4C301B2010F94E319181694F3FD
:10DB00000E94FD520F945A1F75956795ECCF1092A5
:10DB10000A10B8CE40906406509065066090660684
:10DB20007090670620E030E848E953E4C301B20191
:10DB30000F943C201816A4F020E030E040EA50E4B6
:10DB4000C301B2010F94E31987FFCBCE80E066DEFC
:10DB5000C0CE0E94C95191CF80E00E9413525DCF88
:10DB600080E06BDE4090640650906506609066062B
:10DB700070906706E1CF0F931F93CF93DF93EC0173
:10DB80008B016091411240914212641306C085E3FB
:10DB900092E10E94815B60DEF4CF28813981F80137
:10DBA000808191815091401274E0579FF0011124BF
:10DBB000E75CFD4E33872287958784876F5F60938C
:10DBC000411281E0850F841719F08093401202C042
:10DBD00010924012DF91CF911F910F9108950F93F2
:10DBE0001F93CF93DF93CDB7DEB728970FB6F89486
:10DBF000DEBF0FBECDBF8823C1F083E992E09887D6
:10DC00008F8304E610E01A830983BE01695F7F4FAA
:10DC1000CE010196B0DF8AEB92E09E838D831A835A
:10DC20000983BE016B5F7F4F0BC088EB91E09C8343
:10DC30008B8384E190E09A838983BE016D5F7F4F7F
:10DC4000CE01019698DF28960FB6F894DEBF0FBE7E
:10DC5000CDBFDF91CF911F910F9108950E9483C195
:10DC6000BECFAF92BF92CF92DF92FF920F931F93DE
:10DC7000CF93DF9300D01F92CDB7DEB7F82E662387
:10DC800051F01092F9061092F5061092F6061092D5
:10DC9000F7061092F8060F941B0A0091F5061091F2
:10DCA000F6062091F7063091F8065B016C01A01A88
:10DCB000B10AC20AD30AD7FC3DC0F7FE05C004EC86
:10DCC00019E020E030E015C0E091F9062F2D332750
:10DCD00027FD30952C5F3F4F4E2F552747FD509520
:10DCE000241735073CF1EF1554F300E911E020E06B
:10DCF00030E0DC01CB01800F911FA21FB31F809386
:10DD0000F5069093F606A093F706B093F80680ED1B
:10DD100097E09C838B838CE291E09A838983BE0198
:10DD20006D5F7F4FCE01019626DF8091F9068F5FF0
:10DD30008093F9060F900F900F900F90DF91CF9185
:10DD40001F910F91FF90DF90CF90BF90AF900895FB
:10DD5000CF92DF92EF92FF926B017C0183E3C816B2
:10DD6000D104E104F10468F082E3C81AD108E108A3
:10DD7000F10862E370E080E090E00F9488096CDDC8
:10DD8000EDCFC701B6010F948809FF90EF90DF90A7
:10DD9000CF9062CDEF92FF920F931F93CF93DF93BB
:10DDA000EC0189018C81833039F089E0440F551FE3
:10DDB000661F771F8A95D1F79A01AB0161E1CE0109
:10DDC0000E94D258882331F084E08983CE010E94DA
:10DDD000A75841C00F941B0A7B010E94B1588B8346
:10DDE0008F3F49F40F941B0A6E197F096D32714001
:10DDF000A0F381E103C08E3F49F08FE08983CE011B
:10DE00000E94A7588FEF0E94AC5825C08FEF8EBD9F
:10DE1000F80180E090E02FEF0DB407FEFDCF3EB596
:10DE200031932EBD01968F3F31E09307A9F70DB4D2
:10DE300007FEFDCF8EB5F801E150FE4F80830E94B2
:10DE4000B1580E94B158CE010E94A7588FEF0E948E
:10DE5000AC5881E001C080E0DF91CF911F910F911C
:10DE6000FF90EF9008952091B5113091B6112817C9
:10DE7000390709F444C09093B6118093B511009707
:10DE800009F437C02091C811FC01211107C0359653
:10DE9000E491E093C911FC013C960FC0213039F4A4
:10DEA0003F96E491E093C911FC01709606C03D963F
:10DEB000E491E093C911FC013E9684918093CA11CC
:10DEC0008091C911992787FD90952091CA11821BD5
:10DED000910927FD93952091CB11203441F0829F29
:10DEE000C001112426E0969587952A95E1F7809345
:10DEF000CC118CEE90E09093C7118093C6110895D9
:10DF000083E29CE1B0DF81E0809391060895CF9396
:10DF1000C82F823051F020F4813079F4CF91F0CFC6
:10DF2000833031F0843021F008C08AE296E002C0EC
:10DF300086EB96E098DFC0939106CF910895E0912B
:10DF4000AD11F091AE110190F081E02D682F8DEAB6
:10DF500091E11994CF93C82F8FEF8C0F893048F43B
:10DF60008AE296E080DF8C2FEADF80919106CF91E4
:10DF7000CECF8C2FCF91E3CFCF93DF93EC01FE0177
:10DF80008491882319F0E6DF2196F9CFDF91CF91B4
:10DF90000895CF93DF93EC018991882311F0DADFA4
:10DFA000FBCFDF91CF9108959CE0899F802D1124B4
:10DFB00041E0480F4093DF10845F8093E010609150
:10DFC000E51170E0282F30E02E5F3F4F261737070E
:10DFD0009CF150E02091E71130E04217530764F5BF
:10DFE0009EE39093E8118093E91185E4B3DF80917B
:10DFF00079068F5CAFDF80E2ADDF609164067091DF
:10E00000650680916606909167060F945A1FCB01B2
:10E010000E94759EBEDF8FE29DDF0E9448A48111A1
:10E0200004C080917606811107C08091F60F90910F
:10E03000F70F0E94759EADCF0895CF93DF93C0E197
:10E04000D2E08991882329F07ADF82E0C632D807AE
:10E05000C1F7DF91CF9108950F931F93CF93DF9373
:10E06000EC0189018C81833039F039E0440F551F70
:10E07000661F771F3A95D1F79A01AB0168E1CE018F
:10E080000E94D258882311F086E034C08EEF8EBDF6
:10E0900080E090E00DB407FEFDCFF801E80FF91F16
:10E0A00020812EBD0DB407FEFDCF21812EBD02962D
:10E0B000811522E0920771F70DB407FEFDCF8FEFB7
:10E0C0000E94AC588FEF0E94AC580E94B1588B83CD
:10E0D0008F71853031F083E18983CE010E94A7588A
:10E0E0000AC068E572E0CE010E94B858182F81116D
:10E0F00007C087E18983CE010E94A75810E012C0B3
:10E1000020E030E0A9016DE0CE010E94D2588111DB
:10E1100004C00E94B158882311F086E1EBCFCE01F4
:10E120000E94A758812FDF91CF911F910F910895E1
:10E13000CF93809119078823A9F140911A07509134
:10E140001B0760911C0770911D072BE534E080913F
:10E1500017079091180780DFC82F882321F140917D
:10E16000FA065091FB066091FC067091FD06411580
:10E1700051056105710589F02BE534E080911707A1
:10E180009091180769DF882359F01092FA061092CF
:10E19000FB061092FC061092FD06109219078C2FB8
:10E1A000C82F01C0C1E08C2FCF910895CF92DF928C
:10E1B000EF92FF92CF936B017C01C42F80911A07DD
:10E1C00090911B07A0911C07B0911D078C159D0510
:10E1D000AE05BF05C1F0ACDF811102C080E017C001
:10E1E0002BE534E0B701A60180911707909118073D
:10E1F000D1DD882399F3C0921A07D0921B07E092D1
:10E200001C07F0921D0781E0C11180931907CF917F
:10E21000FF90EF90DF90CF9008958F929F92AF92F2
:10E22000BF92CF92DF92EF92FF921F93CF93DF9333
:10E23000C82F2DE234E1309318072093170710926E
:10E24000491442E050E060E070E040933214509393
:10E25000331460933414709335141092190710928C
:10E26000FA061092FB061092FC061092FD064FEF84
:10E270005FEFBA0140931A0750931B0760931C0786
:10E2800070931D07882349F1853008F0F6C040E0FF
:10E2900060E070E0CB018ADF882309F4EEC020E162
:10E2A000C29FF0011124E75FF94F80818F7709F059
:10E2B000E4C04485558566857785443651056105FA
:10E2C000710508F4DAC0C084D184E284F384C114F7
:10E2D000D104E104F10421F4D0C0C12CD12C760189
:10E2E00040E0C701B60162DF182F882309F4C5C0DA
:10E2F00080916604909167048115924009F0BDC039
:10E30000A0916B04AA2309F4B8C08091690490918C
:10E310006A04009709F4B1C040916804442309F4E9
:10E32000ACC0A093441440933614E0E050E061E0A8
:10E3300070E0CE2F9B010E2E02C0220F331F0A94D5
:10E34000E2F74217530749F021E02E0FE83018F0AA
:10E3500020933F1492C0E22FECCFE0933F14209122
:10E360007104309172042115310519F040E050E03C
:10E3700008C020917F043091800440918104509125
:10E3800082042093371430933814409339145093F7
:10E390003A1446015701880E991EA11CB11C8092A7
:10E3A000451490924614A0924714B0924814E091FC
:10E3B0006C04F0916D04F0934B14E0934A14B0E0B8
:10E3C0000F94F61D680D791D8A1D9B1D60934C14DA
:10E3D00070934D1480934E1490934F1445E0EE0FBC
:10E3E000FF1F4A95E1F7E150FE4FEF2FFF27E6951B
:10E3F000DC01CB018E0F9F1FA11DB11D8093401426
:10E4000090934114A0934214B093431480906E04EF
:10E4100090906F048114910419F0A12CB12C08C0C4
:10E4200080907B0490907C04A0907D04B0907E044A
:10E43000A7019601281B390B4A0B5B0BDA01C901B6
:10E44000880D991DAA1DBB1D0C2E04C0B695A7955D
:10E45000979587950A94D2F780933B1490933C1438
:10E46000A0933D14B0933E14853F4FE09407A1055F
:10E47000B10528F48CE08093491410E01AC0853F60
:10E480009F4FA105B10510F480E111C08091870470
:10E4900090918804A0918904B0918A0480934C14CF
:10E4A00090934D14A0934E14B0934F1480E2809338
:10E4B0004914812FDF91CF911F91FF90EF90DF9052
:10E4C000CF90BF90AF909F908F9008958F929F9222
:10E4D000AF92BF92CF92DF92EF92FF920F931F9372
:10E4E000CF93DF93EC016A017B01890189859A85CD
:10E4F000AB85BC850196A11DB11D84179507A607A4
:10E50000B70710F480E054C08F89803129F499272F
:10E51000872F762F652F0BC08032A1F7CB01BA0170
:10E52000E7E09695879577956795EA95D1F78B887B
:10E530009C88AD88BE88680D791D8A1D9B1D8090C2
:10E540001A0790901B07A0901C07B0901D07681534
:10E5500079058A059B0581F48F89803191F4DD244A
:10E56000EE24FF24F601EE0FFF1FE55AFB4F8081DA
:10E570009181A0E0B0E016C040E018DE8111ECCF40
:10E58000C1CFE894C7F8DD24EE24FF24F601EE0F96
:10E59000FF1FEE0FFF1FE55AFB4F80819181A28183
:10E5A000B381BF70F80180839183A283B38381E03C
:10E5B000DF91CF911F910F91FF90EF90DF90CF905F
:10E5C000BF90AF909F908F9008952F923F924F925F
:10E5D0005F926F927F928F929F92AF92BF92CF92F3
:10E5E000DF92EF92FF920F931F93CF93DF93EC0193
:10E5F0005B016A018B81811103C08FEF9FEFC6C061
:10E60000898180FFFACF49895A896B897C898885FD
:10E610009985AA85BB852601612C712C8A019B01F5
:10E62000081B190B2A0B3B0B04151505260537058E
:10E6300018F46A01C81AD90A76013E0124E0620E74
:10E64000711CE114F10409F476C0488559856A8586
:10E650007B854A0181E098222B811A012B01A9E0D8
:10E660005694479437942794AA95D1F7898D9A8D1B
:10E67000FC01223049F4628D738D848D958D620D7D
:10E68000731D841D951D3CC01481115012218114ED
:10E690009104C1F4111116C0452B462B472B49F4A8
:10E6A0008D899E89AF89B88D8C839D83AE83BF830E
:10E6B00009C04C815D816E817F81930107DF8823D2
:10E6C00009F49BCFE98DFA8D6C817D818E819F81CC
:10E6D0006250710981099109058404C0660F771F92
:10E6E000881F991F0A94D2F726853785408951895A
:10E6F000620F731F841F951F610F711D811D911D76
:10E7000020E032E02819390987012E153F0508F469
:10E7100089010115F2E01F0761F520911A07309178
:10E720001B0740911C0750911D0762177307840750
:10E73000950719F41EC0C60129C09501AB01BC01A3
:10E74000809117079091180725DB882309F455CF8E
:10E75000A00EB11E88859985AA85BB85800F911F63
:10E76000A11DB11D88879987AA87BB87E01AF10A86
:10E7700068CF40E01BDD882309F43FCFB401655A20
:10E780007B4FA801C5010F942421E2CFDF91CF91E7
:10E790001F910F91FF90EF90DF90CF90BF90AF90BF
:10E7A0009F908F907F906F905F904F903F902F90B1
:10E7B0000895AF92BF92CF92DF92EF92FF920F93A4
:10E7C0001F93CF93DF936C01EB017A01DC01139669
:10E7D0008C911397823070F018960D911D912D91A8
:10E7E0003C911B970F71112722273327012B022BF6
:10E7F000032B11F08FEF58C04115510511F0F701AF
:10E8000010821DE040E250E0BE01C601DEDE9C0148
:10E810008032910531F081E0232B09F480E081956D
:10E8200043C088818823C1F1853E61F38E3251F364
:10E83000E114F10461F19B859F739F3041F54A8D8E
:10E840005B8D452B21F58F719FEF980F9530F8F474
:10E8500090E00197189F9001199F300D1124FE013F
:10E8600080E090E05701A20EB31E8530B8F46181BC
:10E87000A501480F591FDA016C93019632968D302D
:10E88000910599F7888186FF02C0F50115868B8571
:10E8900083FDB8CF822F08C080E006C08B3010F413
:10E8A0006481E6CF6681E4CFDF91CF911F910F9114
:10E8B000FF90EF90DF90CF90BF90AF9008954F9270
:10E8C0005F926F927F92AF92BF92CF92DF92EF9260
:10E8D000FF920F931F93CF93DF93EC016A017B01AB
:10E8E0002B81222349F089899A89AB89BC898417B5
:10E8F0009507A607B70710F480E06BC0223009F433
:10E9000063C0C114D104E104F10449F41C821D82E6
:10E910001E821F82188619861A861B8659C0888512
:10E920009985AA85BB85E98DFA8DE585F0E0399654
:10E93000AC01BD0141505109610971090E2E04C09D
:10E9400076956795579547950A94D2F79701860172
:10E95000015011092109310904C0369527951795F1
:10E960000795EA95D2F7041715072607370720F011
:10E97000892B8A2B8B2B49F48D899E89AF89B88D81
:10E980008C839D83AE83BF8304C0041B150B260BB1
:10E99000370B280139015E0184E0A80EB11C411437
:10E9A00051046104710481F04C815D816E817F812D
:10E9B0009501898D9A8D8ADD91E0491A5108610887
:10E9C00071088111ECCF05C0C886D986EA86FB861E
:10E9D00081E0DF91CF911F910F91FF90EF90DF9039
:10E9E000CF90BF90AF907F906F905F904F900895C1
:10E9F0004F925F926F927F92AF92BF92CF92DF92CF
:10EA0000EF92FF920F931F93CF93DF9300D01F924B
:10EA1000CDB7DEB78C0149835A836B837C83590160
:10EA2000C12CD12C7601412CB2E05B2E612C712CD3
:10EA300049815A816B817C819E012F5F3F4FC801C4
:10EA400045DD882341F1D301C201F801058404C0EA
:10EA5000880F991FAA1FBB1F0A94D2F7C80ED91E90
:10EA6000EA1EFB1E49815A816B817C818789803136
:10EA700039F481E0483F5F4F6105710538F4D8CF24
:10EA800081E0483F5F4F6F4F7F4090F2F501C082B9
:10EA9000D182E282F3820F900F900F900F90DF915E
:10EAA000CF911F910F91FF90EF90DF90CF90BF908B
:10EAB000AF907F906F905F904F9008950F931F934A
:10EAC000CF93DF93EC018B018B81882311F080E0E1
:10EAD00041C0FB018789803131F18032C1F783E089
:10EAE0008B83F801428D538D648D758D4D8B5E8BBC
:10EAF0006F8B788F9E012F5E3F4FC80179DF88238F
:10EB000031F31A8F098F81E089831C821D821E8256
:10EB10001F82188619861A861B861C861D861E86ED
:10EB20001F86188A17C082E08B831D8A1E8A1F8A5F
:10EB3000188EFB01408D518D60E070E085E0440F40
:10EB4000551F661F771F8A95D1F7498B5A8B6B8BA0
:10EB50007C8BD7CFDF91CF911F910F9108954F926A
:10EB60005F926F927F928F929F92AF92BF92CF925D
:10EB7000DF92EF92FF920F931F93CF93DF93EC01FD
:10EB80004A015B01280139014230510561057105D7
:10EB900008F462C049855A856B857C854F5F5F4F5D
:10EBA0006F4F7F4F481559056A057B0508F454C01F
:10EBB0008F89803129F4FF24EB2CDA2CC92C0CC06E
:10EBC000803209F049C07501640137E0F694E7949A
:10EBD000D794C7943A95D1F74B895C896D897E8922
:10EBE000C40ED51EE61EF71E41E0C701B601DEDAEF
:10EBF000882391F19F89903159F49924AA24BB2448
:10EC0000F401EE0FFF1FE55AFB4F5182408210C006
:10EC1000E89487F89924AA24BB24F401EE0FFF1F7F
:10EC2000EE0FFF1FE55AFB4F4082518262827382D2
:10EC30009A89923090F04D815E816F8178854C0D7C
:10EC40005D1D6E1D7F1D4093FA065093FB06609379
:10EC5000FC067093FD0601C080E0DF91CF911F910B
:10EC60000F91FF90EF90DF90CF90BF90AF909F906B
:10EC70008F907F906F905F904F900895AF92BF926A
:10EC8000CF92DF92EF92FF920F931F93CF93DF9378
:10EC900000D01F92CDB7DEB75C016A017B0182E034
:10ECA00090E0A0E0B0E0F50180839183A283B3837C
:10ECB0009E012F5F3F4FB701A601C50107DC8111FF
:10ECC00002C080E023C000E010E09801B701A60177
:10ECD000C50145DF8823A9F3C980DA80EB80FC8079
:10ECE000F5018789803149F481E0F8EFCF16FFEF15
:10ECF000DF06E104F10450F4DBCF81E098EFC916A0
:10ED00009FEFD906E9069FE0F90690F20F900F9069
:10ED10000F900F90DF91CF911F910F91FF90EF9087
:10ED2000DF90CF90BF90AF900895CF93DF93CDB792
:10ED3000DEB780917806811110C09E01275F3F4F9A
:10ED40004F81588562E470E080E192E00F94AB1946
:10ED50000E94FCA383E08093A802DF91CF910895E5
:10ED6000FF920F931F93CF93DF93C091A71181E080
:10ED7000C827D091A811D827F090A911F826C11161
:10ED800002C0DD2319F0E1E4F2E404C0F110FBCF8E
:10ED900080E077C084918F010F5F1F4F882321F09F
:10EDA0000E944359F801F6CFEDE1FCE184918F0117
:10EDB0000F5F1F4F882321F00E944359F801F6CFBF
:10EDC000CC2361F0EBE1FCE184918F010F5F1F4FD9
:10EDD000882321F00E944359F801F6CFDD2361F02A
:10EDE000E9E1FCE184918F010F5F1F4F882321F03F
:10EDF0000E944359F801F6CFF11003C0EFE0FCE1A7
:10EE00000CC0E7E1FCE184918F010F5F1F4F882365
:10EE1000A9F30E944359F801F6CF84918F010F5F47
:10EE20001F4F882321F00E944359F801F6CFFF209D
:10EE300019F04CE353E002C040EC53E0DD2319F03D
:10EE40002EE333E002C020EC33E0CC2319F080E461
:10EE500093E002C080EC93E05F934F933F932F9336
:10EE60009F938F938DEF9BE19F938F931F925DDF15
:10EE70008DB79EB709960FB6F8949EBF0FBE8DBF93
:10EE800081E0DF91CF911F910F91FF9008958091C4
:10EE900053128150823010F080E008951092531286
:10EEA0000F941B0A60935C1270935D1280935E1244
:10EEB00090935F1281E008950F931F9380915312F6
:10EEC000813019F40F941B0A08C060915C12709194
:10EED0005D1280915E1290915F1200915812109114
:10EEE000591220915A1230915B12601B710B820BE8
:10EEF000930B28EE33E040E050E00F94B81D809172
:10EF0000541290915512A0915612B0915712280F99
:10EF1000391F4A1F5B1FCA01B9011F910F91089544
:10EF200080915312813099F1823051F4C5DF6093A2
:10EF3000541270935512809356129093571218C022
:10EF4000109258121092591210925A1210925B128B
:10EF500010925C1210925D1210925E1210925F126B
:10EF6000109254121092551210925612109257127B
:10EF700081E0809353120F941B0A60935812709390
:10EF8000591280935A1290935B1281E0089580E0A9
:10EF90000895CF92DF92EF92FF92C0908C07D090AD
:10EFA0008D07E0908E07F0908F0720910A11309125
:10EFB0000B1140910C1150910D11C701B6010F9426
:10EFC000481A0F94472060932F1270933012809349
:10EFD000311290933212C701B6010F945A1F2FB706
:10EFE000F8946093BD0F7093BE0F8093BF0F909302
:10EFF000C00F2FBF10921F121092201210922112D8
:10F0000010922212FF90EF90DF90CF9008958091A0
:10F010005312813079F482E0809353120F941B0ACB
:10F0200060935C1270935D1280935E1290935F12F6
:10F0300081E0089580E00895E82FF0E0ED5CFC4E5B
:10F04000849190E0FC013797EC30F105F8F4EC572F
:10F05000FF4F0D9405218091B100887F84608093DB
:10F06000B100089580919100887F84608093910021
:10F0700008958091A100887F84608093A100089505
:10F0800080912101887F84608093210108958F926F
:10F090009F92AF92BF92CF92DF92EF92FF920F9327
:10F0A0001F93CF93DF931F921F92CDB7DEB77C01E2
:10F0B000490180914811811148C08B015B01A40E68
:10F0C000B51E0A151B0509F440C0F701C080D180A8
:10F0D000F80161918F016983C6016A830F94991CBD
:10F0E0006A81681729F1C6010F94A11CC6010F940B
:10F0F000991C99818917E1F0E1E4F2E484918F0190
:10F100000F5F1F4F882321F00E944359F801F6CF6B
:10F11000E3EEFBE184918F010F5F1F4F882321F005
:10F120000E944359F801F6CF81E0809348110DC049
:10F13000BE016F5F7F4FC4010E94DA9AF7018081A0
:10F140009181019691838083BCCF0F900F90DF91C6
:10F15000CF911F910F91FF90EF90DF90CF90BF90D4
:10F16000AF909F908F9008952F923F924F925F9211
:10F170006F927F928F929F92AF92BF92CF92DF92C7
:10F18000EF92FF920F931F93CF93DF93CDB7DEB72C
:10F190006B970FB6F894DEBF0FBECDBF9F8B8E8BE3
:10F1A0001B01488F298FFC016081718182819381CD
:10F1B000698B7A8B8B8B9C8BF101C080D180E28034
:10F1C000F380CD86DE86EF86F88A40904F0450901B
:10F1D0005004609051047090520420914B0430917F
:10F1E0004C0440914D0450914E040F94151E4B0158
:10F1F0005C012CE032E040EA51EC0F943C2087FDAA
:10F2000024C021E230E046E953E4C501B4010F9483
:10F21000E3191816D4F0A3019201C701B6010F94A7
:10F22000151E6B017C012CE032E040EA51EC0F949A
:10F230003C2087FD0AC021E230E847E953E4C701DA
:10F24000B6010F94E31918162CF4612C712C00EC04
:10F250001FE74AC3C0900C02D0900D02E0900E024E
:10F26000F0900F0280910307811107C080915E0228
:10F270008093020781E08093030780915F02909161
:10F280006002A0916102B091620280930C0290939F
:10F290000D02A0930E02B0930F020E94B0EA1982F1
:10F2A0001A821B821C82AE014F5F5F4FBE01635FFB
:10F2B0007F4FCE0141960E949CE881E00E940AEBBC
:10F2C000811197C20F94270A04E010E0812C912C41
:10F2D000A12CE1E4BE2E412C512CF0E26F2EF1E482
:10F2E0007F2E60E070E080EF93E40E944FEB882374
:10F2F00009F401C1015011090115110509F0C1C03E
:10F30000E0E9F5E284918F010F5F1F4F882321F020
:10F310000E944359F801F6CF60E081E895E20E942F
:10F320002BA450E7C52E53E0D52EDE82CD8269E1B5
:10F33000E62EF12CFA82E982BE016B5F7F4FCE018F
:10F3400001960E94BB6D1E821D8202E310E01A83AB
:10F350000983BE016B5F7F4FCE0101960E94BB6D9A
:10F36000DE82CD82FA82E982BE016B5F7F4FCE01E1
:10F3700001960E94BB6D1E821D821A830983BE0105
:10F380006B5F7F4FCE0101960E94BB6DDE82CD8206
:10F39000FA82E982BE016B5F7F4FCE0101960E9427
:10F3A000BB6D1E821D821A830983BE016B5F7F4F76
:10F3B000CE0101960E94BB6D80E090E0A0E0B1E438
:10F3C0008D839E83AF83B88780E090E0A8ECB2E4A1
:10F3D00089839A83AB83BC83BE016B5F7F4FCE0171
:10F3E00001960E94A0E810928C0710928D0710924F
:10F3F0008E0710928F07C0907906809188079091B0
:10F400008907A0918A07B0918B074091840750919A
:10F41000850760918607709187070091800710919A
:10F420008107209182073091830709831A832B83F8
:10F430003C834D835E836F83788789879A87AB8708
:10F44000BC87AE01475F5F4FBE016B5F7F4FCE0150
:10F4500001960E94D4A2E12CF12C00EA1FE32CE8D3
:10F4600037E0AE01475F5F4FBE016B5F7F4FCE015C
:10F4700001960E943DCF8DDD0E947DFB82E795E2E3
:10F480001EC1E9EAF5E284919F012F5F3F4F882377
:10F4900041F02A8F3B8F0E9443592A8D3B8DF90101
:10F4A000F2CF60E089E695E20E942BA48D829E82D5
:10F4B000AF82B88649825A826B827C82BE016B5FC2
:10F4C0007F4FCE0101960E94A0E81D8A19821A8200
:10F4D0001B821C82FCE0F9871D829E012B5E3F4F40
:10F4E000AE014F5F5F4FBE01675F7F4FCE01059654
:10F4F0000E94A7E8F6CE80E090E0A0E0B1E48D8322
:10F500009E83AF83B88720E030E040EA50E460910A
:10F5100088077091890780918A0790918B070F94D3
:10F52000161E69837A838B839C83BE016B5F7F4F3A
:10F53000CE0101960E94A0E804E010E0812C912CFD
:10F5400030E8A32E3FE3B32E412C512C40E2642E31
:10F5500041E4742EDFC060E087E395E20E942BA4B3
:10F5600080E7C82E83E0D82EDE82CD8299E1E92E95
:10F57000F12CFA82E982BE016B5F7F4FCE010196CA
:10F580000E94BB6D1E821D8202E310E01A83098374
:10F59000BE016B5F7F4FCE0101960E94BB6DDE8284
:10F5A000CD82FA82E982BE016B5F7F4FCE01019668
:10F5B0000E94BB6D1E821D821A830983BE016B5F90
:10F5C0007F4FCE0101960E94BB6DDE82CD82FA8212
:10F5D000E982BE016B5F7F4FCE0101960E94BB6D39
:10F5E0001E821D821A830983BE016B5F7F4FCE018D
:10F5F00001960E94BB6D80E090E0A0E0B1E48D83B5
:10F600009E83AF83B88780E090E0A8ECB2E4898362
:10F610009A83AB83BC83BE016B5F7F4FCE010196A3
:10F620000E94A0E810928C0710928D0710928E070E
:10F6300010928F07C0907906809188079091890772
:10F64000A0918A07B0918B0740918407509185075C
:10F65000609186077091870700918007109181075C
:10F66000209182073091830709831A832B833C837F
:10F670004D835E836F83788789879A87AB87BC8742
:10F68000AE01475F5F4FBE016B5F7F4FCE010196BA
:10F690000E94D4A2E12CF12C00EA1FE32CE837E011
:10F6A000AE01475F5F4FBE016B5F7F4FCE0101969A
:10F6B0000E943DCF6EDC0E947DFB88E295E20E94B5
:10F6C000E26760E08FE195E20E942BA48D829E822A
:10F6D000AF82B88649825A826B827C82BE016B5FA0
:10F6E0007F4FCE0101960E94A0E81D8A19821A82DE
:10F6F0001B821C828CE089871D829E012B5E3F4FFE
:10F70000AE014F5F5F4FBE01675F7F4FCE01059631
:10F710000E94A7E860E070E080E792E40E944FEB6F
:10F72000882319F1015011090115110569F4E6E466
:10F73000F5E284918F010F5F1F4F882309F40BCFEF
:10F740000E944359F801F5CFEFE5F5E284919F015E
:10F750002F5F3F4F882309F4B4CF2A8F3B8F0E943D
:10F7600043592A8D3B8DF901F1CF80908807909005
:10F770008907A0908A07B0908B072091530430919D
:10F7800054044091550450915604C501B4010F949E
:10F79000151E2091FE063091FF0640910007509102
:10F7A00001070F94161E3B018C01988D91111CC00E
:10F7B00080E090E0A0E0B1E489839A83AB83BC83CE
:10F7C00020E030E040EA50E4C501B4010F94161E79
:10F7D0006D837E838F839887BE016F5F7F4FCE01DD
:10F7E00005960E94A0E809C080E00E940AEB8823E9
:10F7F00021F0612C712C00EC1FE7809102078093AF
:10F800005E02E98DE33008F440C0ECEDF5E284914E
:10F810005F019FEFA91AB90A882321F00E9443597A
:10F82000F501F5CFEE89FF89608171818281938135
:10F8300043E00E941F4DE7EDF5E284915F019FEFE9
:10F84000A91AB90A882321F00E944359F501F5CF7E
:10F85000F101608171818281938143E00E941F4D9B
:10F86000E2EDF5E284915F019FEFA91AB90A8823BE
:10F8700021F00E944359F501F5CF43E0B301C801DF
:10F880000E941F4D8AE00E944359C0920C02D09200
:10F890000D02E0920E02F0920F029301A801B30153
:10F8A000C8010F94C2208823F9F060E083EC95E250
:10F8B0000E942BA4E6E0F2E484917F019FEFE91A15
:10F8C000F90A882321F00E944359F701F5CFE3EBB1
:10F8D000F5E284917F019FEFE91AF90A882321F06C
:10F8E0000E944359F701F5CFB301C8016B960FB6DB
:10F8F000F894DEBF0FBECDBFDF91CF911F910F9166
:10F90000FF90EF90DF90CF90BF90AF909F908F903F
:10F910007F906F905F904F903F902F9008952F921F
:10F920003F924F925F926F927F928F929F92AF928F
:10F93000BF92CF92DF92EF92FF920F931F93CF93DC
:10F94000DF93CDB7DEB7CF5FD1090FB6F894DEBF36
:10F950000FBECDBF05DA81110C940A8BFE013196E2
:10F960008CE3DF011D928A95E9F7C0906F06C652BD
:10F97000DF4FC882CA5DD0408AE40F94B107882364
:10F9800021F00E94FB910C940A8B86E50F941208DB
:10F99000882349F00F943306CC52DF4F7983688374
:10F9A000C45DD04006C0CC52DF4F19821882C45DBE
:10F9B000D040CC52DF4F28813981C45DD040253002
:10F9C000310570F0E1EBF7E284918F010F5F1F4F7B
:10F9D000882311F40C940A8B0E944359F801F4CF48
:10F9E00084E40F94B107882341F00E94315BC15237
:10F9F000DF4F8883CF5DD04005C0C152DF4F1882F2
:10FA0000CF5DD040CC52DF4F48815981C45DD0409A
:10FA1000433051056CF484E50F94B107882379F0E5
:10FA20000E94315BC352DF4F8883CD5DD0400CC054
:10FA300051E0C352DF4F5883CD5DD04005C0C35263
:10FA4000DF4F1882CD5DD04088E50F9412088823DF
:10FA500021F00F943306162F01C012E089E50F94B0
:10FA60001208882321F00F943306062F01C002E00C
:10FA700080E50F941208811107C0CD52DF4F188323
:10FA8000C35DD040202E08C00F943306CD52DF4F07
:10FA90006883C35DD040262ECD52DF4F8881C35D81
:10FAA000D040823018F4ECE7F7E204C091E0921500
:10FAB00068F0F9CF84918F010F5F1F4F882311F4F5
:10FAC0000C940A8B0E944359F801F4CF83E50F94FC
:10FAD0001208882319F00F94430604C060E070E810
:10FAE0008BEB95E420E030E040E752E40F94F21E07
:10FAF00060935F0270936002809361029093620250
:10FB0000C0904B04D0904C04E0904D04F0904E0413
:10FB10008CE40F941208811109C020E030E040E12C
:10FB200051E4C701B6010F94151E02C00F9443069D
:10FB30000F945A1F6B017C01CA52DF4F798368838F
:10FB4000C65DD04080904B0490904C04A0904D0432
:10FB5000B0904E0482E50F941208811109C020E094
:10FB600030E040E953E4C501B4010F94161E02C011
:10FB70000F9443060F945A1F4B015C01C553DF4F8E
:10FB800079836883CB5CD04040904F045090500400
:10FB9000609051047090520486E40F941208811111
:10FBA00009C020E030E040E151E4C301B2010F940C
:10FBB000151E02C00F9443060F945A1FC954DF4FFD
:10FBC000688379838A839B83C75BD040C954DF4FA6
:10FBD000A881B981C75BD040C052DF4FB983A883E9
:10FBE000C05ED04040904F0450905004609051044B
:10FBF0007090520482E40F941208811109C020E031
:10FC000030E840E953E4C301B2010F94161E02C06C
:10FC10000F9443060F945A1FC554DF4F68837983AE
:10FC20008A839B83CB5BD040C554DF4FE881F98149
:10FC3000CB5BD040C153DF4FF983E883CF5CD0402A
:10FC4000B601882777FD8095982F0F94E919CA513E
:10FC5000DF4F688379838A839B83C65ED040409060
:10FC60004B0450904C0460904D0470904E0420E082
:10FC700030E040EA51E4C301B2010F94151E9B012C
:10FC8000AC01CA51DF4F688179818A819B81C65E50
:10FC9000D0400F94E31987FD13C021E0C4010997F8
:10FCA000CA52DF4F48815981C65DD0404817590775
:10FCB0000CF420E0C154DF4F2883CF5BD04006C056
:10FCC00051E0C154DF4F5883CF5BD040B401882747
:10FCD00077FD8095982F0F94E9194B015C0120E086
:10FCE00030E046E953E4C301B2010F94161E9B01B4
:10FCF000AC01C501B4010F943C20181684F089E0D2
:10FD0000C80ED11C81E0C553DF4FE880F980CB5C81
:10FD1000D040CE14DF040CF480E0382E02C033242F
:10FD20003394C954DF4F28813981C75BD040B90172
:10FD3000882777FD8095982F0F94E9192B013C01B6
:10FD4000C0904F04D0905004E0905104F0905204C1
:10FD500020E030E040EA51E4C701B6010F94151EDF
:10FD60009B01AC01C301B2010F94E31901E087FDCF
:10FD700011C0C554DF4F88819981CB5BD040099772
:10FD8000C052DF4F48815981C05ED04048175907A3
:10FD90000CF400E0C554DF4FA881B981CB5BD040A3
:10FDA000BD01882777FD8095982F0F94E9194B01A5
:10FDB0005C0120E030E847E953E4C701B6010F9445
:10FDC000161E9B01AC01C501B4010F943C2018160E
:10FDD0009CF0C954DF4F88819981C75BD040099658
:10FDE00011E0C153DF4FC880D980CF5CD0408C1563
:10FDF0009D051CF410E001C011E0C154DF4FD88014
:10FE0000CF5BD040D1100CC0332029F08DE697E2B3
:10FE10000E944A590BC0011109C011110DC016C032
:10FE200085E797E20E944A593110F0CF002321F074
:10FE300085E697E20E944A59112311F40C940A8B2B
:10FE40008EE597E20E944A590C940A8BCC52DF4F00
:10FE5000E880F980C45DD040EF28F9F0E7E4F7E2EC
:10FE600084918F010F5F1F4F882321F00E94435917
:10FE7000F801F6CFC152DF4FF880CF5DD040FF20B0
:10FE800061F0EEE2F7E284918F010F5F1F4F88234C
:10FE900021F00E944359F801F6CF0E947DFB109299
:10FEA0006F06C152DF4FC880CF5DD040C1100AC07D
:10FEB0000E942C578BE097E00E945CA10F949A0857
:10FEC0000F94A40381E00E940AEB882349F0C652F4
:10FED000DF4FD880CA5DD040D0926F060C940A8B59
:10FEE0000F944A0A85E40F94B107882341F00E94D9
:10FEF000315BC451DF4F8883CC5ED04005C0C45114
:10FF0000DF4F1882CC5ED040CD52DF4FF880C35D0A
:10FF1000D040EF2CF12CC251DF4FF982E882CE5E47
:10FF2000D040C22CD12CC051DF4FD982C882C05FD3
:10FF3000D040CD52DF4FF880C35DD040F29C7001BD
:10FF40001124C552DF4FF982E882CB5DD040C22C2C
:10FF5000C0942C2D2170CD53DF4F2883C35CD0403B
:10FF6000EE0CFF1CC651DF4FF982E882CA5ED0401A
:10FF70002CEFA70124036001259FD00C1124CC5045
:10FF8000DF4FD982C882C45FD040C552DF4FE880BE
:10FF9000F980CB5DD040EE0CFF1CEE0CFF1CCE5068
:10FFA000DF4FF982E882C25FD040C554DF4F19822B
:10FFB0001882CB5BD0402FEF3FEFC954DF4F39831E
:10FFC0002883C75BD040C553DF4FC880D980CB5C46
:10FFD000D040CA52DF4FE880F980C65DD040CE18CD
:10FFE000DF08C553DF4FD982C882CB5CD040C153F4
:10FFF000DF4FC880D980CF5CD040C052DF4FE8804F
:020000021000EC
:10000000F980C05ED040CE18DF08C153DF4FD982DF
:10001000C882CF5CD040C953DF4F288139814A81E3
:100020005B81C75CD040CA01B9010F94C220811125
:1000300016C3CD53DF4FC880C35CD040CC2091F0B5
:10004000CD52DF4FF880C35DD040CA52DF4FF882F7
:10005000C65DD04021E0C052DF4F2883C05ED04053
:10006000312C12C0CD52DF4F3880C35DD0403A945E
:100070003FEFC052DF4F3883C05ED0404FEFCA52CF
:10008000DF4F4883C65DD04081E0CD53DF4FC8804D
:10009000C35CD040C826CD53DF4FC882C35CD0407C
:1000A0009E01235C3F4FC954DF4F88819981C75B14
:1000B000D0400196C651DF4FC880D980CA5ED0407B
:1000C0008C0D9D1D880F991F880F991F280F391FB0
:1000D000C154DF4F39832883CF5BD040C251DF4FFB
:1000E00028813981CE5ED04021503109CA50DF4F7E
:1000F00039832883C65FD040C051DF4F4881598182
:10010000C05FD04041505109C850DF4F59834883E8
:10011000C85FD040C554DF4FC880D980CB5BD0408A
:10012000EE24D7FCE094FE2CC650DF4FC882D98263
:10013000EA82FB82CA5FD040CA52DF4FD880C65DD8
:10014000D0403D1409F47AC2C553DF4F88819981AC
:10015000CB5CD040CA50DF4F68817981C65FD04008
:100160000F94F220882777FD8095982F0F94E91936
:100170006B017C01632D772767FD7095872F972F83
:100180000F94E9199B01AC01C701B6010F94481AFD
:100190009B01AC01CA51DF4F688179818A819B81C3
:1001A000C65ED0400F94161E4B015C01C153DF4F59
:1001B00088819981CF5CD040C850DF4F68817981B8
:1001C000C85FD0400F94F220882777FD8095982F44
:1001D0000F94E9196B017C01C650DF4F688179816A
:1001E0008A819B81CA5FD0400F94E9199B01AC01C1
:1001F000C701B6010F94481A9B01AC01C301B201BB
:100200000F94161E6B017C0120E030E0A901C501AE
:10021000B4010F94E31987FF04C020E030E0A90186
:1002200004C020E030E040E05FE3C501B4010F947A
:10023000161E0F948B1FC355DF4F688379838A8303
:100240009B83CD5AD04020E030E0A901C701B60120
:100250000F94E31987FF04C020E030E0A90104C037
:1002600020E030E040E05FE3C701B6010F94161EC6
:100270000F948B1FC755DF4F688379838A839B83D5
:10028000C95AD040C954DF4F28813981C75BD0405B
:100290002F5F3F4FC954DF4F39832883C75BD0405E
:1002A000E32DEE0FFF0BC554DF4FC880D980CB5B29
:1002B000D040EC0DFD1DEE0FFF1FA1EAEA2EF12C40
:1002C000EC0EFD1EEE0DFF1D31832083CC52DF4F5F
:1002D0002881C45DD040C451DF4F4881CC5ED040FE
:1002E000BE0167557F4FCE0183559F4F0E94B47862
:1002F000C953DF4F688379838A839B83C75CD0406F
:100300009B01AC010F94C220882341F0C652DF4FFD
:10031000F880CA5DD040F0926F0690C1C953DF4F9C
:10032000288139814A815B81C75CD040CE51DF4F43
:10033000688179818A819B81C25ED0400F94161EAC
:10034000CE51DF4F688379838A839B83C25ED0401E
:10035000C954DF4FE881F981C75BD040EE0FFF1F22
:10036000EE0FFF1F2DE630E02C0F3D1FE20FF31FB5
:10037000C953DF4FC880D980EA80FB80C75CD0407A
:10038000C082D182E282F382C355DF4F8880998098
:10039000AA80BB80CD5AD040C154DF4FE881F9819B
:1003A000CF5BD040CC50DF4FE880F980C45FD040B5
:1003B000EE0DFF1D80829182A282B382C755DF4F6E
:1003C000C880D980EA80FB80C95AD040CE50DF4F28
:1003D00028813981C25FD040E20FF31FC082D182F1
:1003E000E282F382C154DF4FE881F981CF5BD040D4
:1003F00080E090E0A0E8BFE381939193A193B19353
:10040000C154DF4FF983E883CF5BD040A50194014D
:1004100069817A818B819C810F94161E69837A830E
:100420008B839C83A70196016D817E818F81988546
:100430000F94161E6D837E838F839887C953DF4F79
:10044000288139814A815B81C75CD04069857A8582
:100450008B859C850F94161E69877A878B879C876E
:10046000A5019401C501B4010F94481A9B01AC0188
:100470006D857E858F8598890F94161E6D877E8782
:100480008F87988BA7019601C701B6010F94481A70
:100490009B01AC0169897A898B899C890F94161E0E
:1004A000698B7A8B8B8B9C8BC953DF4F2881398169
:1004B0004A815B81C75CD040CA01B9010F94481AD8
:1004C0009B01AC016D897E898F89988D0F94161ED2
:1004D0006D8B7E8B8F8B988FA7019601C501B40120
:1004E0000F94481A9B01AC01698D7A8D8B8D9C8D80
:1004F0000F94161E698F7A8F8B8F9C8FC953DF4F95
:10050000288139814A815B81C75CD040C501B40133
:100510000F94481A9B01AC016D8D7E8D8F8D98A133
:100520000F94161E6D8F7E8F8F8F98A3C953DF4F48
:10053000288139814A815B81C75CD040C701B601FF
:100540000F94481A9B01AC0169A17AA18BA19CA1CF
:100550000F94161E69A37AA38BA39CA3E894B7F803
:100560001DA10EA1FFA1C652DF4FF883CA5DD04086
:1005700028A5C351DF4F2883CD5ED040212F302FD7
:100580004F2FC351DF4F5881CD5ED040C501B4011C
:100590000F943C2018162CF4182D092D3A2D2B2DD4
:1005A0000AC0C652DF4F3881CA5DD040C351DF4F09
:1005B0002881CD5ED040812F902FA32FB22F8DA305
:1005C0009EA3AFA3B8A746015701E894B7F819A5B1
:1005D0000AA5FBA4ECA4212F302F4F2D5E2DC501C1
:1005E000B4010F943C20181624F4182D092DFA2C70
:1005F000EB2C812F902FAF2DBE2D89A79AA7ABA7EB
:10060000BCA720E030E040E85FE369AD7AAD8BAD98
:100610009CAD0F94161E69AF7AAF8BAF9CAF80E094
:100620000E9454F1C052DF4FC880C05ED0403C0CE5
:10063000C652DF4F1882CA5DD0407ECDC554DF4F11
:1006400028813981CB5BD0402F5F3F4FC554DF4FAE
:1006500039832883CB5BD040221508F4DCCC80E0C2
:100660000E940AEB882341F0C652DF4FC880CA5D62
:10067000D040C0926F06C5C7C953DF4F288139816A
:100680004A815B81C75CD040CA01B9010F94C22086
:100690008111B7C789AC9AACABACBCAC20E030E000
:1006A000A901C501B4010F94E319882309F408C214
:1006B000A501940169817A818B819C810F94F21E3E
:1006C000C954DF4F688379838A839B83C75BD0409B
:1006D00069837A838B839C83A50194016D817E81DC
:1006E0008F8198850F94F21EC554DF4F68837983FC
:1006F0008A839B83CB5BD0406D837E838F83988777
:10070000A501940169857A858B859C850F94F21EDD
:10071000C154DF4F688379838A839B83CF5BD0404A
:1007200069877A878B879C87A50194016D857E8573
:100730008F8598890F94F21E6B017C01C954DF4F9D
:10074000288139814A815B81C75BD040CA01B901E8
:100750000F94481A9B01AC01C701B6010F94151EF6
:10076000C553DF4F688379838A839B83CB5CD040FA
:100770006D877E878F87988BA501940169897A8917
:100780008B899C890F94F21E6B017C01C554DF4F4D
:10079000288139814A815B81CB5BD040CA01B90194
:1007A0000F94481A9B01AC01C701B6010F94151EA6
:1007B000C153DF4F688379838A839B83CF5CD040AA
:1007C000698B7A8B8B8B9C8BA50194016D897E89BB
:1007D0008F89988D0F94F21E6B017C01C154DF4FFD
:1007E000288139814A815B81CF5BD040CA01B90140
:1007F0000F94481A9B01AC01C701B6010F94151E56
:100800006D8B7E8B8F8B988FA5019401698D7A8D6E
:100810008B8D9C8D0F94F21E6B017C01C554DF4FB4
:10082000288139814A815B81CB5BD040C954DF4F3D
:10083000688179818A819B81C75BD0400F94481A77
:100840009B01AC01C701B6010F94151ECD53DF4FBC
:10085000688379838A839B83C35CD040698F7A8F56
:100860008B8F9C8FA501940169A17AA18BA19CA17A
:100870000F94F21E6B017C01C154DF4F2881398136
:100880004A815B81CF5BD040C554DF4F688179815D
:100890008A819B81CB5BD0400F94481A9B01AC01AD
:1008A000C701B6010F94151E6B017C0169A37AA3E1
:1008B0008BA39CA3A50194016D8D7E8D8F8D98A136
:1008C0000F94F21E4B015C01C154DF4F2881398126
:1008D0004A815B81CF5BD040C954DF4F6881798109
:1008E0008A819B81C75BD0400F94481A9B01AC0161
:1008F000C501B4010F94151E4B015C016D8F7E8FF5
:100900008F8F98A3C153DF4F288139814A815B8142
:10091000CF5CD040C553DF4F688179818A819B814C
:10092000CB5CD0400F94481A2B013C01CD53DF4FD4
:10093000288139814A815B81C35CD040CA01B901F9
:100940000F94481A9B01AC01C301B2010F94151E0C
:10095000CA52DF4F688379838A839B83C65DD04008
:100960002B013C01E89477F829A53AA54BA55CA595
:100970006DA17EA18FA198A50F94161E2FEF36EEC4
:100980004BED5EE20F94481A9B01AC01C301B2012A
:100990000F94E31918160CF093C0CD53DF4F288144
:1009A00039814A815B81C35CD040C701B6010F9495
:1009B000481A2B013C01C153DF4F288139814A81FC
:1009C0005B81CF5CD040C501B4010F94481A9B01F4
:1009D000AC01C301B2010F94151ECA52DF4F28812A
:1009E00039814A815B81C65DD0400F94F21E2B0194
:1009F0003C016DA77EA78FA798ABCD53DF4F288111
:100A000039814A815B81C35CD040C501B4010F9438
:100A1000481A4B015C01C553DF4F288139814A8157
:100A20005B81CB5CD040C701B6010F94481A9B0193
:100A3000AC01C501B4010F94151ECA52DF4F2881C5
:100A400039814A815B81C65DD0400F94F21E6B01F3
:100A50007C0169AB7AAB8BAB9CABC954DF4F28816F
:100A600039814A815B81C75BD040C301B2010F94D9
:100A7000481A9B01AC01C154DF4F688179818A819A
:100A80009B81CF5BD0400F94161E4B015C01C55477
:100A9000DF4F288139814A815B81CB5BD040C70120
:100AA000B6010F94481A9B01AC01C501B4010F9423
:100AB000161EDC01CB01B0588DAB9EABAFABB8AF0F
:100AC000CDA4DEA4EFA4F8A82601370177FA70942C
:100AD00077F8709489A89AA8ABA8BCA82DA93EA9BC
:100AE0004FA958ADC954DF4F288339834A835B83AC
:100AF000C75BD040C552DF4F48815981CB5DD040A4
:100B0000BA01882777FD8095982F0F94E9199B01EA
:100B1000AC01CE51DF4F688179818A819B81C25EB1
:100B2000D0400F94F21EC153DF4F688379838A83CC
:100B30009B83CF5CD040CC52DF4F88819981C45DCC
:100B4000D040892B09F460C0E8E1F7E284918F017D
:100B50000F5F1F4F882321F00E944359F801F6CF01
:100B600048E0C301B2010E941F4DE3E1F7E2849126
:100B70008F010F5F1F4F882321F00E944359F80116
:100B8000F6CF48E0C501B40190580E941F4DEEE039
:100B9000F7E284918F010F5F1F4F882321F00E949D
:100BA0004359F801F6CFC954DF4F688179818A81B2
:100BB0009B81C75BD040905848E00E941F4D8AE05F
:100BC0000E944359CC52DF4FA881B981C45DD04007
:100BD0001397D4F0E5EFF6E284918F010F5F1F4F7A
:100BE000882321F00E944359F801F6CF48E0C15311
:100BF000DF4F688179818A819B81CF5CD0400E94E0
:100C00001F4D8AE00E944359C152DF4FB881CF5D2A
:100C1000D040B111D1C1CB56DF4FC882D982EA8210
:100C2000FB82C559D040C756DF4F88829982AA827D
:100C3000BB82C959D040C12CD12C50E8E52E5FE3CE
:100C4000F52EC356DF4FC882D982EA82FB82CD5986
:100C5000D040CE018B569F4F0E94E29FC757DF4F77
:100C6000C882D982EA82FB82C958D040C357DF4F7D
:100C7000188219821A821B82CD58D040CF56DF4F7E
:100C8000488259826A827B82C159D040CE018757FF
:100C90009F4F0E94E29FCB56DF4FC880D980EA80E9
:100CA000FB80C559D040C954DF4FC882D982EA823F
:100CB000FB82C75BD040C756DF4F488059806A80AF
:100CC0007B80C959D040C356DF4F88809980AA8065
:100CD000BB80CD59D040C757DF4FC880D980EA804C
:100CE000FB80C958D040C554DF4FC882D982EA8200
:100CF000FB82CB5BD040C357DF4FC880D980EA80EE
:100D0000FB80CD58D040C154DF4FC882D982EA82DF
:100D1000FB82CF5BD040CF56DF4FC880D980EA80BE
:100D2000FB80C159D040A7019601C301B2010F94C5
:100D3000481ACD53DF4F688379838A839B83C35CD2
:100D4000D040C154DF4F288139814A815B81CF5B1C
:100D5000D040C501B4010F94481A9B01AC01CD539A
:100D6000DF4F688179818A819B81C35CD0400F9479
:100D7000151EC358DF4F688379838A839B83CD57C1
:100D8000D040C554DF4F288139814A815B81CB5BDC
:100D9000D040C501B4010F94481A4B015C01A70172
:100DA0009601C954DF4F688179818A819B81C75B35
:100DB000D0400F94481A9B01AC01C501B4010F94B7
:100DC000151ECF57DF4F688379838A839B83C15871
:100DD000D040C154DF4F288139814A815B81CF5B8C
:100DE000D040C954DF4F688179818A819B81C75B7C
:100DF000D0400F94481A6B017C01C554DF4F288105
:100E000039814A815B81CB5BD040C301B2010F9431
:100E1000481A9B01AC01C701B6010F94151ECB57B0
:100E2000DF4F688379838A839B83C558D040CE0186
:100E300083589F4F0E94E29FC757DF4F8880998059
:100E4000AA80BB80C958D040C357DF4FC880D98023
:100E5000EA80FB80CD58D040CF56DF4F4880598084
:100E60006A807B80C159D040C358DF4F28813981C7
:100E70004A815B81CD57D040C954DF4F28833983E5
:100E80004A835B83C75BD040CF57DF4F888199810E
:100E9000AA81BB81C158D040C554DF4F8883998354
:100EA000AA83BB83CB5BD040CB57DF4F28813981EE
:100EB0004A815B81C558D040C154DF4F28833983B4
:100EC0004A835B83CF5BD040CB56DF4F08811981CB
:100ED0002A813B81C559D040C756DF4F488159818F
:100EE0006A817B81C959D040C356DF4F888199817F
:100EF000AA81BB81CD59D0408092EB119092EC1128
:100F0000A092ED11B092EE11C092EF11D092F011BB
:100F1000E092F111F092F2114092F3115092F4111B
:100F20006092F5117092F611C954DF4FC880D980D4
:100F3000EA80FB80C75BD040C092F711D092F811D5
:100F4000E092F911F092FA11C554DF4FC880D980B0
:100F5000EA80FB80CB5BD040C092FB11D092FC11A9
:100F6000E092FD11F092FE11C154DF4FC880D9808C
:100F7000EA80FB80CF5BD040C092FF11D09200127C
:100F8000E0920112F09202120093031210930412E5
:100F900020930512309306124093071250930812C3
:100FA0006093091270930A1280930B1290930C12A3
:100FB000A0930D12B0930E12C352DF4FD880CD5DB7
:100FC000D040DD2009F47EC2E2E3F6E284918F0195
:100FD0000F5F1F4F882321F00E944359F801F6CF7D
:100FE00044244A94420C542CC554DF4F1882CB5BE6
:100FF000D04020ECC154DF4F2883CF5BD04039E78D
:10100000CD53DF4F3883C35CD04044E4C553DF4F3A
:101010004883CB5CD040CE018B569F4FCF54DF4FDF
:1010200099838883C15BD040DE01A757BF4FCD5461
:10103000DF4FB983A883C35BD040FE01E358FF4F65
:10104000CB54DF4FF983E883C55BD04057FC29C1FF
:10105000652C660C770821EAE22EF12CEC0EFD1EC1
:101060006E0C7F1C212C312CC954DF4F1882C75BBA
:10107000D040F301E20DF31DC080D180C352DF4F99
:10108000D982C882CD5DD0408601000F111F000FAC
:10109000111FEDE6F0E0EC0FFD1FE00FF11F808067
:1010A0009180A280B380C153DF4F288139814A816A
:1010B0005B81CF5CD040C501B4010F94151E6B015C
:1010C0007C01E1E0F0E0EC0FFD1FE00FF11F84ADCB
:1010D00095ADA6ADB7ADCB56DF4F88839983AA8374
:1010E000BB83C559D040C352DF4FE881F981CD5D44
:1010F000D040C552DF4F28813981CB5DD040E20F0F
:10110000F31FEE0FFF1FEE0FFF1F41E050E04C0FEB
:101110005D1FE40FF51F84AD95ADA6ADB7ADC75704
:10112000DF4F88839983AA83BB83C958D040C358B3
:10113000DF4F188219821A821B82CD57D040CA54C1
:10114000DF4F5881C65BD0405F93CB54DF4F88811F
:10115000C55BD0408F93CC54DF4F9881C45BD040A7
:101160009F93CD54DF4FA881C35BD040AF93CE5443
:10117000DF4FB881C25BD040BF93CF54DF4FE881CF
:10118000C15BD040EF932DB73EB7245231090FB663
:10119000F8943EBF0FBE2DBFADB7BEB71196EBEEB4
:1011A000F1E184E201900D928A95E1F70E9477A027
:1011B000C358DF4F288139814A815B81CD57D040A8
:1011C000C501B4010F94151E5B018C010FB6F89494
:1011D000DEBF0FBECDBF9B01AC01C554DF4F6881A0
:1011E000CB5BD040C154DF4F7881CF5BD040CD5333
:1011F000DF4F8881C35CD040C553DF4F9881CB5C03
:10120000D0400F943C201816A4F4C554DF4FA88298
:10121000CB5BD040C154DF4FB882CF5BD040CD53C1
:10122000DF4F0883C35CD040C553DF4F1883CB5CCE
:10123000D04020E030E0A901C701B6010F943C2066
:1012400087FD0CC0EFE2F6E284918F010F5F1F4F24
:10125000882339F00E944359F801F6CF80E20E94BA
:10126000435945E0C701B6010E941F4DC954DF4FE5
:101270005881C75BD0405F5FC954DF4F5883C75B5D
:10128000D04084E0280E311CCD52DF4FC880C35DB2
:10129000D0405C1508F4EDCE8AE00E9443595A9480
:1012A000D5CE8AE00E944359CC52DF4F2881398144
:1012B000C45DD0402430310509F004C1E6E0F6E217
:1012C00084918F010F5F1F4F811112C0AE014B56E9
:1012D0005F4FCF54DF4F59834883C15BD0401E011D
:1012E00059E8250E311C3E018DE7680E711C1AC0AD
:1012F0000E944359F801E4CF80E20E94435945E03F
:10130000C501B4010E941F4DD3940C5F1F4FCD52F5
:10131000DF4FF881C35DD040DF16A8F08AE00E945D
:1013200043594A9447FCCAC0E42CEE0CFF08A1EADA
:10133000CA2ED12CCC0EDD1EEC0CFD1C00E010E002
:10134000D12CB4E2CB2EF701E00FF11F0190F08118
:10135000E02D5F01AA0CBB1CAA0CBB1CA1E0B0E0F5
:10136000AC0FBD1FAA0DBB1DDC968D919D910D90FC
:10137000BC91A02DCB56DF4F88839983AA83BB8372
:10138000C559D040C552DF4FA881B981CB5DD0404F
:10139000EA0FFB1FEE0FFF1FEE0FFF1F21E030E0F3
:1013A0002C0F3D1FE20FF31F84AD95ADA6ADB7AD79
:1013B000F10180839183A283B383D3011D921D9297
:1013C0001D921C9213977F926F923F922F92CE5450
:1013D000DF4FB881C25BD040BF93CF54DF4FE8816D
:1013E000C15BD040EF932DB73EB7245231090FB601
:1013F000F8943EBF0FBE2DBFADB7BEB71196EBEE52
:10140000F1E18C2D01900D928A95E1F70E9477A071
:10141000EDE6F0E0EC0FFD1FEA0DFB1DD3012D9171
:101420003D914D915C9160817181828193810F9496
:10143000151EC554DF4F2881CB5BD040C154DF4F10
:101440003881CF5BD040CD53DF4F4881C35CD04063
:10145000C553DF4F5881CB5CD0400F94151E4B0114
:101460005C010FB6F894DEBF0FBECDBF20E030E0C8
:10147000A9010F943C2087FD3FCFE3E0F6E2849181
:101480009F012F5F3F4F882309F439CFC250DF4FB0
:101490002883CE5FD040C150DF4F3883CF5FD0402C
:1014A0000E944359C250DF4F2881CE5FD040C150C7
:1014B000DF4F3881CF5FD040F901E1CF8AE00E9451
:1014C000435908C0CC52DF4FE880F980C45DD0405A
:1014D000EF2821F084EE95E20E9451C0C152DF4F07
:1014E000F880CF5DD040F11085C08CE0E0E8F7E0F7
:1014F000DE01A358BF4F01900D928A95E1F781E07C
:1015000080936F06CE0183589F4F0E945CA1C35504
:10151000DF4F288139814A815B81CD5AD04060916B
:1015200080077091810780918207909183070F94C3
:10153000151E6B017C012DEB37E346E855EB0F944C
:101540003C2087FD4BC02DEB37E346E855E3C70150
:10155000B6010F94E31918160CF440C0C755DF4FBD
:10156000288139814A815B81C95AD04060918407C2
:101570007091850780918607909187070F94151EBB
:101580006B017C012DEB37E346E855EB0F943C20D3
:1015900087FD24C02DEB37E346E855E3C701B601CC
:1015A0000F94E3191816D4F0C953DF4F28813981FD
:1015B0004A815B81C75CD040609188077091890740
:1015C00080918A0790918B070F94151ECB57DF4FA0
:1015D000688379838A839B83C558D0408CE0FE0161
:1015E000E358FF4FA0E8B7E001900D928A95E1F72C
:1015F00081E005C0C652DF4F8881CA5DD04080932C
:101600006F060F94310A0E9492BF80916F0681117C
:101610000F94A403C150DF4F0FB6F894DEBF0FBE86
:10162000CDBFDF91CF911F910F91FF90EF90DF9091
:10163000CF90BF90AF909F908F907F906F905F9072
:101640004F903F902F9008952F923F924F925F922C
:101650006F927F928F929F92AF92BF92CF92DF92C2
:10166000EF92FF920F931F93CF93DF93CDB7DEB727
:101670002B970FB6F894DEBF0FBECDBF9E838D8330
:10168000DC0159962D903C905A97F1014184528487
:1016900063847484FFEF4F1A5F0A6F0A7F0A1496FF
:1016A000CD90DD90ED90FC901797C114D104E1042A
:1016B000F10439F02FEFC21AD20AE20AF20A1B86AD
:1016C00007C0D101CD90DD90ED90FC90B1E0BB87DB
:1016D000460157011F82188619861A86F1018185F5
:1016E0009285A385B4852F81388549855A85281729
:1016F00039074A075B0708F08DC04C145D046E047F
:101700007F0450F482E0C82ED12CE12CF12C92E021
:10171000892E912CA12CB12C9E012F5F3F4FB70138
:10172000A601C1010E946672882309F473C08981F1
:101730009A81AB81BC81892B8A2B8B2B41F046018E
:1017400057013FEF831A930AA30AB30A05C0C814CE
:10175000D904EA04FB0489F08F819885A985BA85AC
:101760000196A11DB11D8F839887A987BA879FEF26
:10177000C91AD90AE90AF90AB1CF0FEF1FEF2FEF03
:101780003FE0B501A401C1010E94AF75F82E882386
:1017900009F440C0ED81FE814481558166817781E5
:1017A000411551056105710539F095018401C101AB
:1017B0000E94AF75882371F1AD81BE8114968D9220
:1017C0009D92AD92BC921797BB85BB2351F0D5017A
:1017D000C4010196A11DB11DF10180839183A283F3
:1017E000B383ED81FE8185899689A789B08D892B88
:1017F0008A2B8B2B81F4AD81BE8155968D929D9263
:10180000AD92BC92589711968C9111978068119661
:101810008C9301C0F12C8F2D2B960FB6F894DEBF60
:101820000FBECDBFDF91CF911F910F91FF90EF9031
:10183000DF90CF90BF90AF909F908F907F906F90F0
:101840005F904F903F902F900895CF93DF93EC01DE
:101850008B81882391F1898187FF2BC06C857D85E1
:101860008E859F8541E00E94D670882331F1E889FA
:1018700080E2E89FF0011124E55AFB4F3097E9F030
:101880008081853ED1F08B81823040F449895A892C
:101890006B897C89448F558F668F778F4D895E89E0
:1018A0006F89788D538F428F758B648B89818F7789
:1018B0008983DF91CF910C94987081E0888380E0D8
:1018C000DF91CF910895CF93DF93EC018B8181302D
:1018D00099F4898181FF10C049895A896B897C8973
:1018E000452B462B472B59F140E050E0BA01CE0181
:1018F0000E945F74811102C080E022C04D895E8920
:101900006F89788D898D9A8D0E943E768823A1F308
:101910001D8A1E8A1F8A188E198A1A8A1B8A1C8A97
:10192000898180688983CE0190DF882329F340E094
:1019300050E0BA01CE01DF91CF910C945F7481E049
:10194000DF91CF9108956F927F928F929F92AF9285
:10195000BF92CF92DF92EF92FF920F931F93CF939C
:10196000DF931F92CDB7DEB78C015B014A01722E67
:10197000DB0159968D919C915A97F801928F818F36
:1019800040E050E0BA01C5010E945F74E12CF5010E
:1019900080859185A285B38541895289638974893F
:1019A00084179507A607B70708F0CEC035E0B695AF
:1019B000A795979587953A95D1F7F82FFF70FF2E49
:1019C000D50113968C91823008F49BC141E050E020
:1019D000BE016F5F7F4FC5010E94E572019719F448
:1019E000898190E002C08FEF9FEF019609F489C1D1
:1019F000F50180859185A285B3854F96A11DB11D06
:101A000080879187A287B387F0E2FF9EB0011124FF
:101A1000655A7B4F6115710509F473C1DB018C9127
:101A2000882311F0853EB9F4E1100EC080911A07A9
:101A300090911B07A0911C07B0911D07F8018487A6
:101A40009587A687B787F08ADB018C91EE24E39413
:101A500081119DCF79C04BE050E0C4010F94172154
:101A6000892B09F094CF77FC4CC120E2F29EF00163
:101A70001124E55AFB4F8385817121F0872D8271F6
:101A800009F05EC040911A0750911B0760911C0736
:101A900070911D07D8011C964D935D936D937C93B7
:101AA0001F975096FC924489558960E070E0BA0116
:101AB00055274427828D938DA0E0B0E0482B592B09
:101AC0006A2B7B2BD80155964D935D936D937C9338
:101AD00058978385887159F4848D958DA68DB78D1F
:101AE000F801818B928BA38BB48B81E010C0803185
:101AF00039F598012F5E3F4FD80159968D919C91F1
:101B00005A970E94F8748823D9F084E0F8018383FF
:101B1000872D8F70D80111968C931197F80114823C
:101B200015821682178218961D921D921D921C9284
:101B30001B9774FED9C0C801C6DE8111D5C0E2C0B2
:101B4000D80113961C92DDC0872D8274823409F06F
:101B5000D8C0EE20E1F0D8015096FC9050971C962A
:101B60006D917D918D919C911F9741E00E94D6705F
:101B7000882309F4C6C0F8018089F0E28F9FC00174
:101B80001124855A9B4F009709F08EC0BAC0D50129
:101B900013968C911397823009F4B3C051968D91AE
:101BA0009D910D90BC91A02D803E9F4FAF41B105FE
:101BB00008F0A7C0C50148DD882309F4A2C00E942F
:101BC0009870882309F49DC0D5015996ED91FC9138
:101BD0005A971496CD90DD90ED90FC901797B2E057
:101BE000CB1AD108E108F108058404C0CC0CDD1C37
:101BF000EE1CFF1C0A94D2F786859785A089B189CF
:101C0000C80ED91EEA1EFB1E81E080931907C09200
